Archive member included because of file (symbol)

c:/altera/11.1/nios2eds/bin/gnu/h-i686-mingw32/bin/../lib/gcc/nios2-elf/4.1.2/mhw-mulx\libgcc.a(_mul_df.o)
                              obj/HDMI_Lib/HDMI_RX/it6605.o (__muldf3)
c:/altera/11.1/nios2eds/bin/gnu/h-i686-mingw32/bin/../lib/gcc/nios2-elf/4.1.2/mhw-mulx\libgcc.a(_div_df.o)
                              obj/HDMI_Lib/HDMI_RX/it6605.o (__divdf3)
c:/altera/11.1/nios2eds/bin/gnu/h-i686-mingw32/bin/../lib/gcc/nios2-elf/4.1.2/mhw-mulx\libgcc.a(_si_to_df.o)
                              obj/HDMI_Lib/HDMI_RX/it6605.o (__floatsidf)
c:/altera/11.1/nios2eds/bin/gnu/h-i686-mingw32/bin/../lib/gcc/nios2-elf/4.1.2/mhw-mulx\libgcc.a(_thenan_df.o)
                              c:/altera/11.1/nios2eds/bin/gnu/h-i686-mingw32/bin/../lib/gcc/nios2-elf/4.1.2/mhw-mulx\libgcc.a(_mul_df.o) (__thenan_df)
c:/altera/11.1/nios2eds/bin/gnu/h-i686-mingw32/bin/../lib/gcc/nios2-elf/4.1.2/mhw-mulx\libgcc.a(lib2-divmod.o)
                              obj/HDMI_Lib/HDMI_RX/it6605.o (__divsi3)
c:/altera/11.1/nios2eds/bin/gnu/h-i686-mingw32/bin/../lib/gcc/nios2-elf/4.1.2/mhw-mulx\libgcc.a(_clzsi2.o)
                              c:/altera/11.1/nios2eds/bin/gnu/h-i686-mingw32/bin/../lib/gcc/nios2-elf/4.1.2/mhw-mulx\libgcc.a(_si_to_df.o) (__clzsi2)
c:/altera/11.1/nios2eds/bin/gnu/h-i686-mingw32/bin/../lib/gcc/nios2-elf/4.1.2/mhw-mulx\libgcc.a(_pack_df.o)
                              c:/altera/11.1/nios2eds/bin/gnu/h-i686-mingw32/bin/../lib/gcc/nios2-elf/4.1.2/mhw-mulx\libgcc.a(_mul_df.o) (__pack_d)
c:/altera/11.1/nios2eds/bin/gnu/h-i686-mingw32/bin/../lib/gcc/nios2-elf/4.1.2/mhw-mulx\libgcc.a(_unpack_df.o)
                              c:/altera/11.1/nios2eds/bin/gnu/h-i686-mingw32/bin/../lib/gcc/nios2-elf/4.1.2/mhw-mulx\libgcc.a(_mul_df.o) (__unpack_d)
c:/altera/11.1/nios2eds/bin/gnu/h-i686-mingw32/bin/../lib/gcc/nios2-elf/4.1.2/mhw-mulx\libgcc.a(_clz.o)
                              c:/altera/11.1/nios2eds/bin/gnu/h-i686-mingw32/bin/../lib/gcc/nios2-elf/4.1.2/mhw-mulx\libgcc.a(_clzsi2.o) (__clz_tab)
c:/altera/11.1/nios2eds/bin/gnu/h-i686-mingw32/bin/../lib/gcc/nios2-elf/4.1.2/../../../../nios2-elf/lib/mhw-mulx\libsmallc.a(lib_a-impure.o)
                              obj/HDMI_Lib/mcu.o (_impure_ptr)
c:/altera/11.1/nios2eds/bin/gnu/h-i686-mingw32/bin/../lib/gcc/nios2-elf/4.1.2/../../../../nios2-elf/lib/mhw-mulx\libsmallc.a(lib_a-memset.o)
                              obj/main.o (memset)
c:/altera/11.1/nios2eds/bin/gnu/h-i686-mingw32/bin/../lib/gcc/nios2-elf/4.1.2/../../../../nios2-elf/lib/mhw-mulx\libsmallc.a(lib_a-printf.o)
                              obj/HDMI_Lib/HDMI_TX/HDMI_TX.o (printf)
c:/altera/11.1/nios2eds/bin/gnu/h-i686-mingw32/bin/../lib/gcc/nios2-elf/4.1.2/../../../../nios2-elf/lib/mhw-mulx\libsmallc.a(lib_a-putchar.o)
                              obj/HDMI_Lib/HDMI_TX/it6613_drv.o (putchar)
c:/altera/11.1/nios2eds/bin/gnu/h-i686-mingw32/bin/../lib/gcc/nios2-elf/4.1.2/../../../../nios2-elf/lib/mhw-mulx\libsmallc.a(lib_a-puts.o)
                              obj/main.o (puts)
c:/altera/11.1/nios2eds/bin/gnu/h-i686-mingw32/bin/../lib/gcc/nios2-elf/4.1.2/../../../../nios2-elf/lib/mhw-mulx\libsmallc.a(lib_a-sprintf.o)
                              obj/terasic_lib/debug.o (sprintf)
c:/altera/11.1/nios2eds/bin/gnu/h-i686-mingw32/bin/../lib/gcc/nios2-elf/4.1.2/../../../../nios2-elf/lib/mhw-mulx\libsmallc.a(lib_a-strlen.o)
                              c:/altera/11.1/nios2eds/bin/gnu/h-i686-mingw32/bin/../lib/gcc/nios2-elf/4.1.2/../../../../nios2-elf/lib/mhw-mulx\libsmallc.a(lib_a-puts.o) (strlen)
c:/altera/11.1/nios2eds/bin/gnu/h-i686-mingw32/bin/../lib/gcc/nios2-elf/4.1.2/../../../../nios2-elf/lib/mhw-mulx\libsmallc.a(lib_a-vfprintf.o)
                              c:/altera/11.1/nios2eds/bin/gnu/h-i686-mingw32/bin/../lib/gcc/nios2-elf/4.1.2/../../../../nios2-elf/lib/mhw-mulx\libsmallc.a(lib_a-printf.o) (___vfprintf_internal_r)
c:/altera/11.1/nios2eds/bin/gnu/h-i686-mingw32/bin/../lib/gcc/nios2-elf/4.1.2/../../../../nios2-elf/lib/mhw-mulx\libsmallc.a(lib_a-vfprintf_1.o)
                              obj/HDMI_Lib/mcu.o (vfprintf)
c:/altera/11.1/nios2eds/bin/gnu/h-i686-mingw32/bin/../lib/gcc/nios2-elf/4.1.2/../../../../nios2-elf/lib/mhw-mulx\libsmallc.a(lib_a-vsnprintf.o)
                              obj/terasic_lib/debug.o (vsnprintf)
c:/altera/11.1/nios2eds/bin/gnu/h-i686-mingw32/bin/../lib/gcc/nios2-elf/4.1.2/../../../../nios2-elf/lib/mhw-mulx\libsmallc.a(lib_a-fvwrite_small_dev.o)
                              c:/altera/11.1/nios2eds/bin/gnu/h-i686-mingw32/bin/../lib/gcc/nios2-elf/4.1.2/../../../../nios2-elf/lib/mhw-mulx\libsmallc.a(lib_a-printf.o) (__sfvwrite_small_dev)
c:/altera/11.1/nios2eds/bin/gnu/h-i686-mingw32/bin/../lib/gcc/nios2-elf/4.1.2/../../../../nios2-elf/lib/mhw-mulx\libsmallc.a(lib_a-fvwrite_small_str.o)
                              c:/altera/11.1/nios2eds/bin/gnu/h-i686-mingw32/bin/../lib/gcc/nios2-elf/4.1.2/../../../../nios2-elf/lib/mhw-mulx\libsmallc.a(lib_a-sprintf.o) (__sfvwrite_small_str)
c:/altera/11.1/nios2eds/bin/gnu/h-i686-mingw32/bin/../lib/gcc/nios2-elf/4.1.2/../../../../nios2-elf/lib/mhw-mulx\libsmallc.a(lib_a-memmove.o)
                              c:/altera/11.1/nios2eds/bin/gnu/h-i686-mingw32/bin/../lib/gcc/nios2-elf/4.1.2/../../../../nios2-elf/lib/mhw-mulx\libsmallc.a(lib_a-fvwrite_small_str.o) (memmove)
c:/altera/11.1/nios2eds/bin/gnu/h-i686-mingw32/bin/../lib/gcc/nios2-elf/4.1.2/../../../../nios2-elf/lib/mhw-mulx\libsmallc.a(lib_a-putc.o)
                              c:/altera/11.1/nios2eds/bin/gnu/h-i686-mingw32/bin/../lib/gcc/nios2-elf/4.1.2/../../../../nios2-elf/lib/mhw-mulx\libsmallc.a(lib_a-putchar.o) (_putc_r)
c:/altera/11.1/nios2eds/bin/gnu/h-i686-mingw32/bin/../lib/gcc/nios2-elf/4.1.2/../../../../nios2-elf/lib/mhw-mulx\libsmallc.a(lib_a-writer.o)
                              c:/altera/11.1/nios2eds/bin/gnu/h-i686-mingw32/bin/../lib/gcc/nios2-elf/4.1.2/../../../../nios2-elf/lib/mhw-mulx\libsmallc.a(lib_a-fvwrite_small_dev.o) (_write_r)
c:/altera/11.1/nios2eds/bin/gnu/h-i686-mingw32/bin/../lib/gcc/nios2-elf/4.1.2/../../../../nios2-elf/lib/mhw-mulx\libsmallc.a(lib_a-int_errno.o)
                              c:/altera/11.1/nios2eds/bin/gnu/h-i686-mingw32/bin/../lib/gcc/nios2-elf/4.1.2/../../../../nios2-elf/lib/mhw-mulx\libsmallc.a(lib_a-writer.o) (errno)
../TR4_HDMI_TX_RX_bsp/\libhal_bsp.a(alt_irq_register.o)
                              obj/main.o (alt_irq_register)
../TR4_HDMI_TX_RX_bsp/\libhal_bsp.a(alt_irq_vars.o)
                              ../TR4_HDMI_TX_RX_bsp/\libhal_bsp.a(alt_irq_register.o) (alt_irq_active)
../TR4_HDMI_TX_RX_bsp/\libhal_bsp.a(alt_load.o)
                              ../TR4_HDMI_TX_RX_bsp//obj/HAL/src/crt0.o (alt_load)
../TR4_HDMI_TX_RX_bsp/\libhal_bsp.a(alt_main.o)
                              ../TR4_HDMI_TX_RX_bsp//obj/HAL/src/crt0.o (alt_main)
../TR4_HDMI_TX_RX_bsp/\libhal_bsp.a(alt_tick.o)
                              obj/HDMI_Lib/HDMI_RX/HDMI_RX.o (_alt_tick_rate)
../TR4_HDMI_TX_RX_bsp/\libhal_bsp.a(alt_usleep.o)
                              obj/HDMI_Lib/HDMI_RX/HDMI_RX.o (usleep)
../TR4_HDMI_TX_RX_bsp/\libhal_bsp.a(alt_write.o)
                              c:/altera/11.1/nios2eds/bin/gnu/h-i686-mingw32/bin/../lib/gcc/nios2-elf/4.1.2/../../../../nios2-elf/lib/mhw-mulx\libsmallc.a(lib_a-writer.o) (write)
../TR4_HDMI_TX_RX_bsp/\libhal_bsp.a(alt_sys_init.o)
                              ../TR4_HDMI_TX_RX_bsp/\libhal_bsp.a(alt_main.o) (alt_irq_init)
../TR4_HDMI_TX_RX_bsp/\libhal_bsp.a(altera_avalon_jtag_uart_fd.o)
                              ../TR4_HDMI_TX_RX_bsp/\libhal_bsp.a(alt_sys_init.o) (altera_avalon_jtag_uart_read_fd)
../TR4_HDMI_TX_RX_bsp/\libhal_bsp.a(altera_avalon_jtag_uart_read.o)
                              ../TR4_HDMI_TX_RX_bsp/\libhal_bsp.a(altera_avalon_jtag_uart_fd.o) (altera_avalon_jtag_uart_read)
../TR4_HDMI_TX_RX_bsp/\libhal_bsp.a(altera_avalon_jtag_uart_write.o)
                              ../TR4_HDMI_TX_RX_bsp/\libhal_bsp.a(altera_avalon_jtag_uart_fd.o) (altera_avalon_jtag_uart_write)
../TR4_HDMI_TX_RX_bsp/\libhal_bsp.a(altera_avalon_timer_sc.o)
                              ../TR4_HDMI_TX_RX_bsp/\libhal_bsp.a(alt_sys_init.o) (alt_avalon_timer_sc_init)
../TR4_HDMI_TX_RX_bsp/\libhal_bsp.a(alt_busy_sleep.o)
                              ../TR4_HDMI_TX_RX_bsp/\libhal_bsp.a(alt_usleep.o) (alt_busy_sleep)
../TR4_HDMI_TX_RX_bsp/\libhal_bsp.a(alt_close.o)
                              ../TR4_HDMI_TX_RX_bsp/\libhal_bsp.a(alt_main.o) (close)
../TR4_HDMI_TX_RX_bsp/\libhal_bsp.a(alt_dcache_flush_all.o)
                              ../TR4_HDMI_TX_RX_bsp/\libhal_bsp.a(alt_load.o) (alt_dcache_flush_all)
../TR4_HDMI_TX_RX_bsp/\libhal_bsp.a(alt_dev.o)
                              ../TR4_HDMI_TX_RX_bsp/\libhal_bsp.a(alt_sys_init.o) (alt_dev_list)
../TR4_HDMI_TX_RX_bsp/\libhal_bsp.a(alt_dev_llist_insert.o)
                              ../TR4_HDMI_TX_RX_bsp/\libhal_bsp.a(alt_sys_init.o) (alt_dev_llist_insert)
../TR4_HDMI_TX_RX_bsp/\libhal_bsp.a(alt_do_ctors.o)
                              ../TR4_HDMI_TX_RX_bsp/\libhal_bsp.a(alt_main.o) (_do_ctors)
../TR4_HDMI_TX_RX_bsp/\libhal_bsp.a(alt_do_dtors.o)
                              ../TR4_HDMI_TX_RX_bsp/\libhal_bsp.a(alt_main.o) (_do_dtors)
../TR4_HDMI_TX_RX_bsp/\libhal_bsp.a(alt_errno.o)
                              ../TR4_HDMI_TX_RX_bsp/\libhal_bsp.a(alt_write.o) (alt_errno)
../TR4_HDMI_TX_RX_bsp/\libhal_bsp.a(alt_icache_flush_all.o)
                              ../TR4_HDMI_TX_RX_bsp/\libhal_bsp.a(alt_load.o) (alt_icache_flush_all)
../TR4_HDMI_TX_RX_bsp/\libhal_bsp.a(alt_iic.o)
                              ../TR4_HDMI_TX_RX_bsp/\libhal_bsp.a(altera_avalon_timer_sc.o) (alt_ic_isr_register)
../TR4_HDMI_TX_RX_bsp/\libhal_bsp.a(alt_iic_isr_register.o)
                              ../TR4_HDMI_TX_RX_bsp/\libhal_bsp.a(alt_iic.o) (alt_iic_isr_register)
../TR4_HDMI_TX_RX_bsp/\libhal_bsp.a(alt_io_redirect.o)
                              ../TR4_HDMI_TX_RX_bsp/\libhal_bsp.a(alt_main.o) (alt_io_redirect)
../TR4_HDMI_TX_RX_bsp/\libhal_bsp.a(alt_irq_entry.o)
                              ../TR4_HDMI_TX_RX_bsp/\libhal_bsp.a(alt_irq_register.o) (alt_irq_entry)
../TR4_HDMI_TX_RX_bsp/\libhal_bsp.a(alt_irq_handler.o)
                              ../TR4_HDMI_TX_RX_bsp/\libhal_bsp.a(alt_irq_register.o) (alt_irq_handler)
../TR4_HDMI_TX_RX_bsp/\libhal_bsp.a(alt_open.o)
                              ../TR4_HDMI_TX_RX_bsp/\libhal_bsp.a(alt_io_redirect.o) (open)
../TR4_HDMI_TX_RX_bsp/\libhal_bsp.a(alt_release_fd.o)
                              ../TR4_HDMI_TX_RX_bsp/\libhal_bsp.a(alt_close.o) (alt_release_fd)
../TR4_HDMI_TX_RX_bsp/\libhal_bsp.a(altera_nios2_qsys_irq.o)
                              ../TR4_HDMI_TX_RX_bsp/\libhal_bsp.a(alt_sys_init.o) (altera_nios2_qsys_irq_init)
../TR4_HDMI_TX_RX_bsp/\libhal_bsp.a(alt_exception_entry.o)
                              ../TR4_HDMI_TX_RX_bsp/\libhal_bsp.a(alt_irq_entry.o) (alt_exception)
../TR4_HDMI_TX_RX_bsp/\libhal_bsp.a(alt_find_dev.o)
                              ../TR4_HDMI_TX_RX_bsp/\libhal_bsp.a(alt_open.o) (alt_find_dev)
../TR4_HDMI_TX_RX_bsp/\libhal_bsp.a(alt_find_file.o)
                              ../TR4_HDMI_TX_RX_bsp/\libhal_bsp.a(alt_open.o) (alt_find_file)
../TR4_HDMI_TX_RX_bsp/\libhal_bsp.a(alt_get_fd.o)
                              ../TR4_HDMI_TX_RX_bsp/\libhal_bsp.a(alt_open.o) (alt_get_fd)
../TR4_HDMI_TX_RX_bsp/\libhal_bsp.a(alt_icache_flush.o)
                              ../TR4_HDMI_TX_RX_bsp/\libhal_bsp.a(alt_icache_flush_all.o) (alt_icache_flush)
c:/altera/11.1/nios2eds/bin/gnu/h-i686-mingw32/bin/../lib/gcc/nios2-elf/4.1.2/../../../../nios2-elf/lib/mhw-mulx\libsmallc.a(lib_a-atexit.o)
                              ../TR4_HDMI_TX_RX_bsp/\libhal_bsp.a(alt_main.o) (atexit)
c:/altera/11.1/nios2eds/bin/gnu/h-i686-mingw32/bin/../lib/gcc/nios2-elf/4.1.2/../../../../nios2-elf/lib/mhw-mulx\libsmallc.a(lib_a-exit.o)
                              ../TR4_HDMI_TX_RX_bsp/\libhal_bsp.a(alt_main.o) (exit)
c:/altera/11.1/nios2eds/bin/gnu/h-i686-mingw32/bin/../lib/gcc/nios2-elf/4.1.2/../../../../nios2-elf/lib/mhw-mulx\libsmallc.a(lib_a-memcmp.o)
                              ../TR4_HDMI_TX_RX_bsp/\libhal_bsp.a(alt_find_dev.o) (memcmp)
c:/altera/11.1/nios2eds/bin/gnu/h-i686-mingw32/bin/../lib/gcc/nios2-elf/4.1.2/../../../../nios2-elf/lib/mhw-mulx\libsmallc.a(lib_a-__atexit.o)
                              c:/altera/11.1/nios2eds/bin/gnu/h-i686-mingw32/bin/../lib/gcc/nios2-elf/4.1.2/../../../../nios2-elf/lib/mhw-mulx\libsmallc.a(lib_a-atexit.o) (__register_exitproc)
c:/altera/11.1/nios2eds/bin/gnu/h-i686-mingw32/bin/../lib/gcc/nios2-elf/4.1.2/../../../../nios2-elf/lib/mhw-mulx\libsmallc.a(lib_a-__call_atexit.o)
                              c:/altera/11.1/nios2eds/bin/gnu/h-i686-mingw32/bin/../lib/gcc/nios2-elf/4.1.2/../../../../nios2-elf/lib/mhw-mulx\libsmallc.a(lib_a-exit.o) (__call_exitprocs)
../TR4_HDMI_TX_RX_bsp/\libhal_bsp.a(alt_exit.o)
                              c:/altera/11.1/nios2eds/bin/gnu/h-i686-mingw32/bin/../lib/gcc/nios2-elf/4.1.2/../../../../nios2-elf/lib/mhw-mulx\libsmallc.a(lib_a-exit.o) (_exit)

Allocating common symbols
Common symbol       size              file

alt_irq             0x100             ../TR4_HDMI_TX_RX_bsp/\libhal_bsp.a(alt_irq_handler.o)
AudioInfo           0xd               obj/HDMI_Lib/HDMI_TX/it6613_sys.o
errno               0x4               c:/altera/11.1/nios2eds/bin/gnu/h-i686-mingw32/bin/../lib/gcc/nios2-elf/4.1.2/../../../../nios2-elf/lib/mhw-mulx\libsmallc.a(lib_a-int_errno.o)
VideoPixelClock     0x4               obj/HDMI_Lib/HDMI_TX/it6613_sys.o
aspec               0x4               obj/HDMI_Lib/HDMI_TX/it6613_sys.o
RxCapability        0xf8              obj/HDMI_Lib/HDMI_TX/it6613_sys.o
Colorimetry         0x4               obj/HDMI_Lib/HDMI_TX/it6613_sys.o
pixelrep            0x1               obj/HDMI_Lib/HDMI_TX/it6613_sys.o
_atexit0            0x8c              c:/altera/11.1/nios2eds/bin/gnu/h-i686-mingw32/bin/../lib/gcc/nios2-elf/4.1.2/../../../../nios2-elf/lib/mhw-mulx\libsmallc.a(lib_a-atexit.o)
bHDMIMode           0x4               obj/HDMI_Lib/HDMI_TX/it6613_sys.o
bAudioEnable        0x4               obj/HDMI_Lib/HDMI_TX/it6613_sys.o
VIC                 0x1               obj/HDMI_Lib/HDMI_TX/it6613_sys.o
AviInfo             0x10              obj/HDMI_Lib/HDMI_TX/it6613_sys.o
Instance            0x10              obj/HDMI_Lib/HDMI_TX/it6613_drv.o

Memory Configuration

Name             Origin             Length             Attributes
reset            0x01020000         0x00000020
onchip_memory2   0x01020020         0x0001ffe0
*default*        0x00000000         0xffffffff

Linker script and memory map

LOAD ../TR4_HDMI_TX_RX_bsp//obj/HAL/src/crt0.o
LOAD obj/Beep.o
LOAD obj/HDMI_Lib/HDMI_RX/HDMI_RX.o
LOAD obj/HDMI_Lib/HDMI_RX/it6605.o
LOAD obj/HDMI_Lib/HDMI_TX/EDID.o
LOAD obj/HDMI_Lib/HDMI_TX/HDMI_TX.o
LOAD obj/HDMI_Lib/HDMI_TX/dss_sha.o
LOAD obj/HDMI_Lib/HDMI_TX/it6613_drv.o
LOAD obj/HDMI_Lib/HDMI_TX/it6613_sys.o
LOAD obj/HDMI_Lib/mcu.o
LOAD obj/main.o
LOAD obj/terasic_lib/I2C.o
LOAD obj/terasic_lib/debug.o
LOAD c:/altera/11.1/nios2eds/bin/gnu/h-i686-mingw32/bin/../lib/gcc/nios2-elf/4.1.2/../../../../nios2-elf/lib/mhw-mulx\libstdc++.a
LOAD c:/altera/11.1/nios2eds/bin/gnu/h-i686-mingw32/bin/../lib/gcc/nios2-elf/4.1.2/../../../../nios2-elf/lib/mhw-mulx\libm.a
LOAD c:/altera/11.1/nios2eds/bin/gnu/h-i686-mingw32/bin/../lib/gcc/nios2-elf/4.1.2/mhw-mulx\libgcc.a
START GROUP
LOAD c:/altera/11.1/nios2eds/bin/gnu/h-i686-mingw32/bin/../lib/gcc/nios2-elf/4.1.2/../../../../nios2-elf/lib/mhw-mulx\libsmallc.a
LOAD c:/altera/11.1/nios2eds/bin/gnu/h-i686-mingw32/bin/../lib/gcc/nios2-elf/4.1.2/mhw-mulx\libgcc.a
LOAD ../TR4_HDMI_TX_RX_bsp/\libhal_bsp.a
END GROUP
LOAD c:/altera/11.1/nios2eds/bin/gnu/h-i686-mingw32/bin/../lib/gcc/nios2-elf/4.1.2/mhw-mulx\libgcc.a
                0x01020000                __alt_mem_onchip_memory2 = 0x1020000

.entry          0x01020000       0x20
 *(.entry)
 .entry         0x01020000       0x20 ../TR4_HDMI_TX_RX_bsp//obj/HAL/src/crt0.o
                0x01020000                __reset

.exceptions     0x01020020      0x194
                0x01020020                PROVIDE (__ram_exceptions_start, ABSOLUTE (.))
                0x01020020                . = ALIGN (0x20)
 *(.irq)
 *(.exceptions.entry.label)
 .exceptions.entry.label
                0x01020020        0x0 ../TR4_HDMI_TX_RX_bsp/\libhal_bsp.a(alt_irq_entry.o)
                0x01020020                alt_irq_entry
 .exceptions.entry.label
                0x01020020        0x0 ../TR4_HDMI_TX_RX_bsp/\libhal_bsp.a(alt_exception_entry.o)
                0x01020020                alt_exception
 *(.exceptions.entry.user)
 *(.exceptions.entry)
 .exceptions.entry
                0x01020020       0x54 ../TR4_HDMI_TX_RX_bsp/\libhal_bsp.a(alt_exception_entry.o)
 *(.exceptions.irqtest.user)
 *(.exceptions.irqtest)
 .exceptions.irqtest
                0x01020074       0x10 ../TR4_HDMI_TX_RX_bsp/\libhal_bsp.a(alt_irq_entry.o)
 *(.exceptions.irqhandler.user)
 *(.exceptions.irqhandler)
 .exceptions.irqhandler
                0x01020084        0x4 ../TR4_HDMI_TX_RX_bsp/\libhal_bsp.a(alt_irq_entry.o)
 *(.exceptions.irqreturn.user)
 *(.exceptions.irqreturn)
 .exceptions.irqreturn
                0x01020088        0x4 ../TR4_HDMI_TX_RX_bsp/\libhal_bsp.a(alt_irq_entry.o)
 *(.exceptions.notirq.label)
 .exceptions.notirq.label
                0x0102008c        0x0 ../TR4_HDMI_TX_RX_bsp/\libhal_bsp.a(alt_irq_entry.o)
 *(.exceptions.notirq.user)
 *(.exceptions.notirq)
 .exceptions.notirq
                0x0102008c        0x8 ../TR4_HDMI_TX_RX_bsp/\libhal_bsp.a(alt_exception_entry.o)
 *(.exceptions.soft.user)
 *(.exceptions.soft)
 *(.exceptions.unknown.user)
 *(.exceptions.unknown)
 .exceptions.unknown
                0x01020094        0x4 ../TR4_HDMI_TX_RX_bsp/\libhal_bsp.a(alt_exception_entry.o)
 *(.exceptions.exit.label)
 .exceptions.exit.label
                0x01020098        0x0 ../TR4_HDMI_TX_RX_bsp/\libhal_bsp.a(alt_irq_entry.o)
 .exceptions.exit.label
                0x01020098        0x0 ../TR4_HDMI_TX_RX_bsp/\libhal_bsp.a(alt_exception_entry.o)
 *(.exceptions.exit.user)
 *(.exceptions.exit)
 .exceptions.exit
                0x01020098       0x54 ../TR4_HDMI_TX_RX_bsp/\libhal_bsp.a(alt_exception_entry.o)
 *(.exceptions)
 .exceptions    0x010200ec       0xc8 ../TR4_HDMI_TX_RX_bsp/\libhal_bsp.a(alt_irq_handler.o)
                0x010200ec                alt_irq_handler
                0x010201b4                PROVIDE (__ram_exceptions_end, ABSOLUTE (.))
                0x01020020                PROVIDE (__flash_exceptions_start, LOADADDR (.exceptions))

.text           0x010201b4    0x1318c
                0x010201b4                PROVIDE (stext, ABSOLUTE (.))
 *(.interp)
 *(.hash)
 *(.dynsym)
 *(.dynstr)
 *(.gnu.version)
 *(.gnu.version_d)
 *(.gnu.version_r)
 *(.rel.init)
 *(.rela.init)
 *(.rel.text .rel.text.* .rel.gnu.linkonce.t.*)
 *(.rela.text .rela.text.* .rela.gnu.linkonce.t.*)
 *(.rel.fini)
 *(.rela.fini)
 *(.rel.rodata .rel.rodata.* .rel.gnu.linkonce.r.*)
 *(.rela.rodata .rela.rodata.* .rela.gnu.linkonce.r.*)
 *(.rel.data .rel.data.* .rel.gnu.linkonce.d.*)
 *(.rela.data .rela.data.* .rela.gnu.linkonce.d.*)
 *(.rel.tdata .rel.tdata.* .rel.gnu.linkonce.td.*)
 *(.rela.tdata .rela.tdata.* .rela.gnu.linkonce.td.*)
 *(.rel.tbss .rel.tbss.* .rel.gnu.linkonce.tb.*)
 *(.rela.tbss .rela.tbss.* .rela.gnu.linkonce.tb.*)
 *(.rel.ctors)
 *(.rela.ctors)
 *(.rel.dtors)
 *(.rela.dtors)
 *(.rel.got)
 *(.rela.got)
 *(.rel.sdata .rel.sdata.* .rel.gnu.linkonce.s.*)
 *(.rela.sdata .rela.sdata.* .rela.gnu.linkonce.s.*)
 *(.rel.sbss .rel.sbss.* .rel.gnu.linkonce.sb.*)
 *(.rela.sbss .rela.sbss.* .rela.gnu.linkonce.sb.*)
 *(.rel.sdata2 .rel.sdata2.* .rel.gnu.linkonce.s2.*)
 *(.rela.sdata2 .rela.sdata2.* .rela.gnu.linkonce.s2.*)
 *(.rel.sbss2 .rel.sbss2.* .rel.gnu.linkonce.sb2.*)
 *(.rela.sbss2 .rela.sbss2.* .rela.gnu.linkonce.sb2.*)
 *(.rel.bss .rel.bss.* .rel.gnu.linkonce.b.*)
 *(.rela.bss .rela.bss.* .rela.gnu.linkonce.b.*)
 *(.rel.plt)
 *(.rela.plt)
 *(.rel.dyn)
 *(.init)
 *(.plt)
 *(.text .stub .text.* .gnu.linkonce.t.*)
 .text          0x010201b4       0x3c ../TR4_HDMI_TX_RX_bsp//obj/HAL/src/crt0.o
                0x010201b4                _start
 .text          0x010201f0        0x0 obj/Beep.o
 .text          0x010201f0      0xe64 obj/HDMI_Lib/HDMI_RX/HDMI_RX.o
                0x010201f0                EDID_WriteProtect
                0x01020220                HDMIRX_EnableEdid
                0x0102025c                HDMIRX_IsVideoOn
                0x010202a0                HDMIRX_WriteEeprom
                0x010203c4                HDMIRX_VerifyEeprom
                0x0102053c                HDMIRX_ShowInfo
                0x010209c4                HDMIRX_DevLoopProc
                0x01020b5c                HDMIRX_Init
                0x01020d1c                HDMIRX_ChipVerify
                0x01020dec                HDMIRX_GetAVIInfoFrame
                0x01020f08                HDMIRX_IsModeChange
                0x01020f28                HDMIRX_GetSourceColor
                0x01020fc4                HDMIRX_SetOutputColor
 .text          0x01021054     0x52cc obj/HDMI_Lib/HDMI_RX/it6605.o
                0x01021080                Check_HDMInterrupt
                0x010210a8                CheckHDMIRX
                0x0102125c                SelectHDMIPort
                0x010212c8                GetCurrentHDMIPort
                0x01021490                RxHDCPSetReceiver
                0x010214c0                RxHDCPSetRepeater
                0x010214f4                RxHDCPSetRdyTimeOut
                0x01021528                RxHDCPSetInvalidV
                0x0102155c                RxHDCPSetOverDownStream
                0x01021590                RxHDCPSetOverCascade
                0x010215c4                RxHDCPRepeaterCapabilitySet
                0x0102161c                RxHDCPRepeaterCapabilityClear
                0x01021678                RxGetKSVFifoList
                0x01021764                RxSetKSVFifoList
                0x01021850                RxHDCPGetM0
                0x01021908                RxHDCPGetBstatus
                0x010219a4                RxAuthSetBStatus
                0x01021a1c                RxHDCPWriteVR
                0x01021b78                RxAuthStartInt
                0x01021bb0                RxAuthDoneInt
                0x01021d5c                InitIT6605
                0x01021f6c                PowerDownHDMI
                0x01021fa8                getIT6605HorzTotal
                0x01022018                getIT6605HorzActive
                0x010220ec                getIT6605HorzFrontPorch
                0x01022164                getIT6605HorzSyncWidth
                0x010221d4                getIT6605HorzBackPorch
                0x01022230                getIT6605VertTotal
                0x010222f8                getIT6605VertActive
                0x010223cc                getIT6605VertFrontPorch
                0x01022434                getIT6605VertSyncToDE
                0x0102246c                getIT6605VertSyncWidth
                0x01022520                getIT6605VertSyncBackPorch
                0x01022564                getIT6605xCnt
                0x01022594                getIT6605AudioInfo
                0x01022664                GetAVIInfoFrame
                0x010226f8                GetAudioInfoFrame
                0x0102278c                GetMPEGInfoFrame
                0x01022820                GetVENDORSPECInfoFrame
                0x010228b4                GetACPPacket
                0x0102290c                getIT6605Regs
                0x01022a04                getIT6605OutputColorMode
                0x01022a2c                getIT6605OutputColorDepth
                0x01022b84                RDROM_Reset
                0x01022c24                Check_RDROM
                0x01022e40                SetDefaultRegisterValue
                0x01023004                CheckPlg5VPwr
                0x01023068                CheckHDCPFail
                0x010230a4                SetMUTE
                0x01023154                SetIntMask1
                0x010231c4                SetIntMask2
                0x01023234                SetIntMask3
                0x010232a4                SetIntMask4
                0x01023314                IsIT6605HDMIMode
                0x01023350                Interrupt_Handler
                0x010236ec                RXINT_5V_PwrOn
                0x01023744                RXINT_5V_PwrOff
                0x01023778                RXINT_SCDT_On
                0x010237bc                RXINT_SCDT_Off
                0x0102380c                RXINT_VideoMode_Chg
                0x0102387c                RXINT_HDMIMode_Chg
                0x010238ec                RXINT_AVMute_Set
                0x01023964                RXINT_AVMute_Clear
                0x01023a08                RXINT_SetNewAVIInfo
                0x01023a5c                RXINT_ResetAudio
                0x01023a9c                RXINT_ResetHDCP
                0x01023b0c                Timer_Handler
                0x01024400                AssignVideoTimerTimeout
                0x01024428                AssignAudioTimerTimeout
                0x01024450                SwitchVideoState
                0x01024760                SwitchAudioState
                0x01025378                Video_Handler
                0x010256b0                SetVideoInputFormatWithInfoFrame
                0x01025814                SetColorimetryByInfoFrame
                0x01025940                SetColorSpaceConvert
                0x01025e64                SetDVIVideoOutput
                0x01025e98                SetNewInfoVideoOutput
                0x01025f38                ResetAudio
                0x01025f7c                SetHWMuteCTRL
                0x010261e0                SetAudioMute
                0x01026230                CDR_Reset
 .text          0x01026320      0x950 obj/HDMI_Lib/HDMI_TX/EDID.o
                0x010263ac                ParseVESAEDID
                0x010264c0                ParseCEAEDID
 .text          0x01026c70      0xa10 obj/HDMI_Lib/HDMI_TX/HDMI_TX.o
                0x01026c70                HDMITX_ChipVerify
                0x01026d94                HDMITX_Init
                0x01026e00                HDMITX_HPD
                0x01026e3c                HDMITX_SetAVIInfoFrame
                0x0102700c                HDMITX_ChangeVideoTiming
                0x01027094                HDMITX_ChangeVideoTimingAndColor
                0x01027114                HDMITX_DisableVideoOutput
                0x0102713c                HDMITX_EnableVideoOutput
                0x01027164                HDMITX_SetColorSpace
                0x010271b0                HDMITX_IsSinkSupportYUV444
                0x01027240                HDMITX_IsSinkSupportYUV422
                0x010272d0                HDMITX_IsSinkSupportColorDepth36
                0x0102735c                HDMITX_IsSinkSupportColorDepth30
                0x010273e8                HDMITX_SetOutputColorDepth
                0x01027420                HDMITX_DevLoopProc
 .text          0x01027680        0x0 obj/HDMI_Lib/HDMI_TX/dss_sha.o
 .text          0x01027680     0x5814 obj/HDMI_Lib/HDMI_TX/it6613_drv.o
                0x01027680                HDMITX_InitInstance
                0x010277d4                InitIT6613
                0x010278e8                SetupVideoInputSignal
                0x0102791c                EnableVideoOutput
                0x01027a90                EnableAudioOutput
                0x01027c5c                GetEDIDData
                0x01027d34                EnableHDCP
                0x01027d90                CheckHDMITX
                0x010280c0                DisableIT6613
                0x01028104                DisableVideoOutput
                0x01028150                DisableAudioOutput
                0x01028190                EnableAVIInfoFrame
                0x010281fc                EnableAudioInfoFrame
                0x01028268                SetAVMute
                0x010282e8                SetOutputColorDepthPhase
                0x010283ac                Get6613Reg
                0x0102849c                ProgramDEGenModeByID
                0x01028704                ProgramSyncEmbeddedVideoMode
                0x0102b9f8                SHA_Simple
 .text          0x0102ce94      0xb74 obj/HDMI_Lib/HDMI_TX/it6613_sys.o
                0x0102ce94                HDMITX_SetOutput
                0x0102cfac                HDMITX_ChangeDisplayOption
                0x0102d47c                ConfigAVIInfoFrame
                0x0102d684                ConfigAudioInfoFrm
                0x0102d744                ParseEDID
 .text          0x0102da08      0xbbc obj/HDMI_Lib/mcu.o
                0x0102da08                OS_DelayMS
                0x0102da38                OS_GetTicks
                0x0102da60                OS_TicksPerSecond
                0x0102da88                DelayMS
                0x0102dac0                EnableDebugMessage
                0x0102dae8                ErrorF
                0x0102db4c                OS_PRINTF
                0x0102dc10                HDMITX_Reset
                0x0102dc78                HDMITX_DumpAllReg
                0x0102dce8                HDMITX_DumpReg
                0x0102dd84                HDMITX_ReadI2C_Byte
                0x0102ddc4                HDMITX_WriteI2C_Byte
                0x0102de00                HDMITX_ReadI2C_ByteN
                0x0102dea8                HDMITX_WriteI2C_ByteN
                0x0102df58                HDMIRX_Reset
                0x0102dfc0                HDMIRX_DumpReg
                0x0102e00c                HDMIRX_DumpAllReg
                0x0102e07c                HDMIRX_ReadI2C_Byte
                0x0102e0bc                HDMIRX_WriteI2C_Byte
                0x0102e0f8                HDMIRX_ReadI2C_ByteN
                0x0102e1a0                HDMIRX_WriteI2C_ByteN
                0x0102e250                ReadRXIntPin
                0x0102e290                I2C_Read_Byte
                0x0102e2d8                I2C_Write_Byte
                0x0102e31c                I2C_Read_ByteN
                0x0102e3d4                I2C_Write_ByteN
                0x0102e484                HDMIRX_EEPROM0_WriteI2C_Byte
                0x0102e4d4                HDMIRX_EEPROM1_WriteI2C_Byte
                0x0102e524                HDMIRX_EEPROM0_ReadI2C_Byte
                0x0102e574                HDMIRX_EEPROM1_ReadI2C_Byte
 .text          0x0102e5c4      0xca4 obj/main.o
                0x0102e5c4                THDMI_TX_I2S_Start
                0x0102e5f0                THDMI_TX_I2S_Stop
                0x0102e618                THDMI_TX_I2S_Play
                0x0102e6b8                i2s_isr
                0x0102e784                FindVIC
                0x0102e8b8                SetupTxVIC
                0x0102e8fc                VPG_Config
                0x0102e9e4                SetupColorSpace
                0x0102ec9c                button_isr
                0x0102ee60                main
 .text          0x0102f268      0x730 obj/terasic_lib/I2C.o
                0x0102f268                I2C_Open
                0x0102f2bc                I2C_Close
                0x0102f2f8                I2C_Write
                0x0102f3d0                I2C_Read
                0x0102f4d4                I2C_MultipleRead
                0x0102f628                i2c_start
                0x0102f6b0                i2c_stop
                0x0102f728                i2c_write
                0x0102f84c                i2c_read
 .text          0x0102f998      0x184 obj/terasic_lib/debug.o
                0x0102f998                debug_output
                0x0102f9c8                myprintf
                0x0102fa28                myprintf_hexarray
                0x0102faa0                myprintf_dwordarray
 .text          0x0102fb1c      0x3b4 c:/altera/11.1/nios2eds/bin/gnu/h-i686-mingw32/bin/../lib/gcc/nios2-elf/4.1.2/mhw-mulx\libgcc.a(_mul_df.o)
                0x0102fb1c                __muldf3
 .text          0x0102fed0      0x258 c:/altera/11.1/nios2eds/bin/gnu/h-i686-mingw32/bin/../lib/gcc/nios2-elf/4.1.2/mhw-mulx\libgcc.a(_div_df.o)
                0x0102fed0                __divdf3
 .text          0x01030128       0xf8 c:/altera/11.1/nios2eds/bin/gnu/h-i686-mingw32/bin/../lib/gcc/nios2-elf/4.1.2/mhw-mulx\libgcc.a(_si_to_df.o)
                0x01030128                __floatsidf
 .text          0x01030220        0x0 c:/altera/11.1/nios2eds/bin/gnu/h-i686-mingw32/bin/../lib/gcc/nios2-elf/4.1.2/mhw-mulx\libgcc.a(_thenan_df.o)
 .text          0x01030220      0x14c c:/altera/11.1/nios2eds/bin/gnu/h-i686-mingw32/bin/../lib/gcc/nios2-elf/4.1.2/mhw-mulx\libgcc.a(lib2-divmod.o)
                0x0103029c                __divsi3
                0x010302fc                __modsi3
                0x0103035c                __udivsi3
                0x01030364                __umodsi3
 .text          0x0103036c       0x80 c:/altera/11.1/nios2eds/bin/gnu/h-i686-mingw32/bin/../lib/gcc/nios2-elf/4.1.2/mhw-mulx\libgcc.a(_clzsi2.o)
                0x0103036c                __clzsi2
 .text          0x010303ec      0x314 c:/altera/11.1/nios2eds/bin/gnu/h-i686-mingw32/bin/../lib/gcc/nios2-elf/4.1.2/mhw-mulx\libgcc.a(_pack_df.o)
                0x010303ec                __pack_d
 .text          0x01030700      0x138 c:/altera/11.1/nios2eds/bin/gnu/h-i686-mingw32/bin/../lib/gcc/nios2-elf/4.1.2/mhw-mulx\libgcc.a(_unpack_df.o)
                0x01030700                __unpack_d
 .text          0x01030838        0x0 c:/altera/11.1/nios2eds/bin/gnu/h-i686-mingw32/bin/../lib/gcc/nios2-elf/4.1.2/mhw-mulx\libgcc.a(_clz.o)
 .text          0x01030838        0x0 c:/altera/11.1/nios2eds/bin/gnu/h-i686-mingw32/bin/../lib/gcc/nios2-elf/4.1.2/../../../../nios2-elf/lib/mhw-mulx\libsmallc.a(lib_a-impure.o)
 .text          0x01030838       0x20 c:/altera/11.1/nios2eds/bin/gnu/h-i686-mingw32/bin/../lib/gcc/nios2-elf/4.1.2/../../../../nios2-elf/lib/mhw-mulx\libsmallc.a(lib_a-memset.o)
                0x01030838                memset
 .text          0x01030858       0x98 c:/altera/11.1/nios2eds/bin/gnu/h-i686-mingw32/bin/../lib/gcc/nios2-elf/4.1.2/../../../../nios2-elf/lib/mhw-mulx\libsmallc.a(lib_a-printf.o)
                0x01030858                printf
                0x010308ac                _printf_r
 .text          0x010308f0       0x24 c:/altera/11.1/nios2eds/bin/gnu/h-i686-mingw32/bin/../lib/gcc/nios2-elf/4.1.2/../../../../nios2-elf/lib/mhw-mulx\libsmallc.a(lib_a-putchar.o)
                0x010308f0                putchar
                0x0103090c                _putchar_r
 .text          0x01030914       0xa4 c:/altera/11.1/nios2eds/bin/gnu/h-i686-mingw32/bin/../lib/gcc/nios2-elf/4.1.2/../../../../nios2-elf/lib/mhw-mulx\libsmallc.a(lib_a-puts.o)
                0x01030914                _puts_r
                0x010309a4                puts
 .text          0x010309b8       0xf4 c:/altera/11.1/nios2eds/bin/gnu/h-i686-mingw32/bin/../lib/gcc/nios2-elf/4.1.2/../../../../nios2-elf/lib/mhw-mulx\libsmallc.a(lib_a-sprintf.o)
                0x010309b8                sprintf
                0x01030a3c                _sprintf_r
 .text          0x01030aac       0x20 c:/altera/11.1/nios2eds/bin/gnu/h-i686-mingw32/bin/../lib/gcc/nios2-elf/4.1.2/../../../../nios2-elf/lib/mhw-mulx\libsmallc.a(lib_a-strlen.o)
                0x01030aac                strlen
 .text          0x01030acc      0x678 c:/altera/11.1/nios2eds/bin/gnu/h-i686-mingw32/bin/../lib/gcc/nios2-elf/4.1.2/../../../../nios2-elf/lib/mhw-mulx\libsmallc.a(lib_a-vfprintf.o)
                0x01030b4c                ___vfprintf_internal_r
                0x01031120                __vfprintf_internal
 .text          0x01031144       0x10 c:/altera/11.1/nios2eds/bin/gnu/h-i686-mingw32/bin/../lib/gcc/nios2-elf/4.1.2/../../../../nios2-elf/lib/mhw-mulx\libsmallc.a(lib_a-vfprintf_1.o)
                0x01031144                vfprintf
 .text          0x01031154      0x104 c:/altera/11.1/nios2eds/bin/gnu/h-i686-mingw32/bin/../lib/gcc/nios2-elf/4.1.2/../../../../nios2-elf/lib/mhw-mulx\libsmallc.a(lib_a-vsnprintf.o)
                0x01031154                _vsnprintf_r
                0x01031218                vsnprintf
 .text          0x01031258       0xbc c:/altera/11.1/nios2eds/bin/gnu/h-i686-mingw32/bin/../lib/gcc/nios2-elf/4.1.2/../../../../nios2-elf/lib/mhw-mulx\libsmallc.a(lib_a-fvwrite_small_dev.o)
                0x01031258                __sfvwrite_small_dev
 .text          0x01031314       0xb8 c:/altera/11.1/nios2eds/bin/gnu/h-i686-mingw32/bin/../lib/gcc/nios2-elf/4.1.2/../../../../nios2-elf/lib/mhw-mulx\libsmallc.a(lib_a-fvwrite_small_str.o)
                0x01031314                __sfvwrite_small_str
 .text          0x010313cc       0x60 c:/altera/11.1/nios2eds/bin/gnu/h-i686-mingw32/bin/../lib/gcc/nios2-elf/4.1.2/../../../../nios2-elf/lib/mhw-mulx\libsmallc.a(lib_a-memmove.o)
                0x010313cc                memmove
 .text          0x0103142c       0xe4 c:/altera/11.1/nios2eds/bin/gnu/h-i686-mingw32/bin/../lib/gcc/nios2-elf/4.1.2/../../../../nios2-elf/lib/mhw-mulx\libsmallc.a(lib_a-putc.o)
                0x0103142c                putc
                0x0103149c                _putc_r
 .text          0x01031510       0x78 c:/altera/11.1/nios2eds/bin/gnu/h-i686-mingw32/bin/../lib/gcc/nios2-elf/4.1.2/../../../../nios2-elf/lib/mhw-mulx\libsmallc.a(lib_a-writer.o)
                0x01031510                _write_r
 .text          0x01031588        0x0 c:/altera/11.1/nios2eds/bin/gnu/h-i686-mingw32/bin/../lib/gcc/nios2-elf/4.1.2/../../../../nios2-elf/lib/mhw-mulx\libsmallc.a(lib_a-int_errno.o)
 .text          0x01031588      0x1c0 ../TR4_HDMI_TX_RX_bsp/\libhal_bsp.a(alt_irq_register.o)
                0x01031588                alt_irq_register
 .text          0x01031748        0x0 ../TR4_HDMI_TX_RX_bsp/\libhal_bsp.a(alt_irq_vars.o)
 .text          0x01031748       0xec ../TR4_HDMI_TX_RX_bsp/\libhal_bsp.a(alt_load.o)
                0x01031748                alt_load
 .text          0x01031834       0x6c ../TR4_HDMI_TX_RX_bsp/\libhal_bsp.a(alt_main.o)
                0x01031834                alt_main
 .text          0x010318a0      0x1a4 ../TR4_HDMI_TX_RX_bsp/\libhal_bsp.a(alt_tick.o)
                0x010318a0                alt_alarm_stop
                0x01031938                alt_tick
 .text          0x01031a44       0x30 ../TR4_HDMI_TX_RX_bsp/\libhal_bsp.a(alt_usleep.o)
                0x01031a44                usleep
 .text          0x01031a74      0x180 ../TR4_HDMI_TX_RX_bsp/\libhal_bsp.a(alt_write.o)
                0x01031a74                write
 .text          0x01031bf4       0xb0 ../TR4_HDMI_TX_RX_bsp/\libhal_bsp.a(alt_sys_init.o)
                0x01031bf4                alt_irq_init
                0x01031c28                alt_sys_init
 .text          0x01031ca4       0xb0 ../TR4_HDMI_TX_RX_bsp/\libhal_bsp.a(altera_avalon_jtag_uart_fd.o)
                0x01031ca4                altera_avalon_jtag_uart_read_fd
                0x01031cfc                altera_avalon_jtag_uart_write_fd
 .text          0x01031d54      0x104 ../TR4_HDMI_TX_RX_bsp/\libhal_bsp.a(altera_avalon_jtag_uart_read.o)
                0x01031d54                altera_avalon_jtag_uart_read
 .text          0x01031e58       0xa4 ../TR4_HDMI_TX_RX_bsp/\libhal_bsp.a(altera_avalon_jtag_uart_write.o)
                0x01031e58                altera_avalon_jtag_uart_write
 .text          0x01031efc      0x100 ../TR4_HDMI_TX_RX_bsp/\libhal_bsp.a(altera_avalon_timer_sc.o)
                0x01031f6c                alt_avalon_timer_sc_init
 .text          0x01031ffc      0x14c ../TR4_HDMI_TX_RX_bsp/\libhal_bsp.a(alt_busy_sleep.o)
                0x01031ffc                alt_busy_sleep
 .text          0x01032148      0x15c ../TR4_HDMI_TX_RX_bsp/\libhal_bsp.a(alt_close.o)
                0x01032148                close
 .text          0x010322a4       0x1c ../TR4_HDMI_TX_RX_bsp/\libhal_bsp.a(alt_dcache_flush_all.o)
                0x010322a4                alt_dcache_flush_all
 .text          0x010322c0       0x2c ../TR4_HDMI_TX_RX_bsp/\libhal_bsp.a(alt_dev.o)
 .text          0x010322ec      0x114 ../TR4_HDMI_TX_RX_bsp/\libhal_bsp.a(alt_dev_llist_insert.o)
                0x010322ec                alt_dev_llist_insert
 .text          0x01032400       0x64 ../TR4_HDMI_TX_RX_bsp/\libhal_bsp.a(alt_do_ctors.o)
                0x01032400                _do_ctors
 .text          0x01032464       0x64 ../TR4_HDMI_TX_RX_bsp/\libhal_bsp.a(alt_do_dtors.o)
                0x01032464                _do_dtors
 .text          0x010324c8        0x0 ../TR4_HDMI_TX_RX_bsp/\libhal_bsp.a(alt_errno.o)
 .text          0x010324c8       0x30 ../TR4_HDMI_TX_RX_bsp/\libhal_bsp.a(alt_icache_flush_all.o)
                0x010324c8                alt_icache_flush_all
 .text          0x010324f8      0x1d4 ../TR4_HDMI_TX_RX_bsp/\libhal_bsp.a(alt_iic.o)
                0x010324f8                alt_ic_isr_register
                0x01032548                alt_ic_irq_enable
                0x010325e4                alt_ic_irq_disable
                0x01032684                alt_ic_irq_enabled
 .text          0x010326cc       0xf8 ../TR4_HDMI_TX_RX_bsp/\libhal_bsp.a(alt_iic_isr_register.o)
                0x010326cc                alt_iic_isr_register
 .text          0x010327c4      0x13c ../TR4_HDMI_TX_RX_bsp/\libhal_bsp.a(alt_io_redirect.o)
                0x01032888                alt_io_redirect
 .text          0x01032900        0x0 ../TR4_HDMI_TX_RX_bsp/\libhal_bsp.a(alt_irq_entry.o)
 .text          0x01032900        0x0 ../TR4_HDMI_TX_RX_bsp/\libhal_bsp.a(alt_irq_handler.o)
 .text          0x01032900      0x2c4 ../TR4_HDMI_TX_RX_bsp/\libhal_bsp.a(alt_open.o)
                0x010329dc                open
 .text          0x01032bc4       0x60 ../TR4_HDMI_TX_RX_bsp/\libhal_bsp.a(alt_release_fd.o)
                0x01032bc4                alt_release_fd
 .text          0x01032c24       0x20 ../TR4_HDMI_TX_RX_bsp/\libhal_bsp.a(altera_nios2_qsys_irq.o)
                0x01032c24                altera_nios2_qsys_irq_init
 .text          0x01032c44        0x0 ../TR4_HDMI_TX_RX_bsp/\libhal_bsp.a(alt_exception_entry.o)
 .text          0x01032c44       0x94 ../TR4_HDMI_TX_RX_bsp/\libhal_bsp.a(alt_find_dev.o)
                0x01032c44                alt_find_dev
 .text          0x01032cd8      0x120 ../TR4_HDMI_TX_RX_bsp/\libhal_bsp.a(alt_find_file.o)
                0x01032cd8                alt_find_file
 .text          0x01032df8       0xb8 ../TR4_HDMI_TX_RX_bsp/\libhal_bsp.a(alt_get_fd.o)
                0x01032df8                alt_get_fd
 .text          0x01032eb0       0x90 ../TR4_HDMI_TX_RX_bsp/\libhal_bsp.a(alt_icache_flush.o)
                0x01032eb0                alt_icache_flush
 .text          0x01032f40       0x14 c:/altera/11.1/nios2eds/bin/gnu/h-i686-mingw32/bin/../lib/gcc/nios2-elf/4.1.2/../../../../nios2-elf/lib/mhw-mulx\libsmallc.a(lib_a-atexit.o)
                0x01032f40                atexit
 .text          0x01032f54       0x20 c:/altera/11.1/nios2eds/bin/gnu/h-i686-mingw32/bin/../lib/gcc/nios2-elf/4.1.2/../../../../nios2-elf/lib/mhw-mulx\libsmallc.a(lib_a-exit.o)
                0x01032f54                exit
 .text          0x01032f74       0x3c c:/altera/11.1/nios2eds/bin/gnu/h-i686-mingw32/bin/../lib/gcc/nios2-elf/4.1.2/../../../../nios2-elf/lib/mhw-mulx\libsmallc.a(lib_a-memcmp.o)
                0x01032f74                memcmp
 .text          0x01032fb0      0x16c c:/altera/11.1/nios2eds/bin/gnu/h-i686-mingw32/bin/../lib/gcc/nios2-elf/4.1.2/../../../../nios2-elf/lib/mhw-mulx\libsmallc.a(lib_a-__atexit.o)
                0x01032fb0                __register_exitproc
 .text          0x0103311c      0x1c0 c:/altera/11.1/nios2eds/bin/gnu/h-i686-mingw32/bin/../lib/gcc/nios2-elf/4.1.2/../../../../nios2-elf/lib/mhw-mulx\libsmallc.a(lib_a-__call_atexit.o)
                0x01033120                __call_exitprocs
 .text          0x010332dc       0x60 ../TR4_HDMI_TX_RX_bsp/\libhal_bsp.a(alt_exit.o)
                0x0103331c                _exit
 *(.gnu.warning.*)
 *(.fini)
                0x0103333c                PROVIDE (__etext, ABSOLUTE (.))
                0x0103333c                PROVIDE (_etext, ABSOLUTE (.))
                0x0103333c                PROVIDE (etext, ABSOLUTE (.))
 *(.eh_frame_hdr)
                0x0103333c                . = ALIGN (0x4)
                0x0103333c                PROVIDE (__preinit_array_start, ABSOLUTE (.))
 *(.preinit_array)
                0x0103333c                PROVIDE (__preinit_array_end, ABSOLUTE (.))
                0x0103333c                PROVIDE (__init_array_start, ABSOLUTE (.))
 *(.init_array)
                0x0103333c                PROVIDE (__init_array_end, ABSOLUTE (.))
                0x0103333c                PROVIDE (__fini_array_start, ABSOLUTE (.))
 *(.fini_array)
                0x0103333c                PROVIDE (__fini_array_end, ABSOLUTE (.))
 *(.eh_frame)
 *(.gcc_except_table)
 *(.dynamic)
                0x0103333c                PROVIDE (__CTOR_LIST__, ABSOLUTE (.))
 *(.ctors)
 *(SORT(.ctors.*))
 .ctors.65535   0x0103333c        0x4 c:/altera/11.1/nios2eds/bin/gnu/h-i686-mingw32/bin/../lib/gcc/nios2-elf/4.1.2/../../../../nios2-elf/lib/mhw-mulx\libsmallc.a(lib_a-__call_atexit.o)
                0x01033340                PROVIDE (__CTOR_END__, ABSOLUTE (.))
                0x01033340                PROVIDE (__DTOR_LIST__, ABSOLUTE (.))
 *(.dtors)
 *(SORT(.dtors.*))
                0x01033340                PROVIDE (__DTOR_END__, ABSOLUTE (.))
 *(.jcr)
                0x01033340                . = ALIGN (0x4)

.rodata         0x01033340     0x7aec
                0x01033340                PROVIDE (__ram_rodata_start, ABSOLUTE (.))
                0x01033340                . = ALIGN (0x4)
 *(.rodata .rodata.* .gnu.linkonce.r.*)
 .rodata        0x01033340     0x5cdc obj/Beep.o
                0x01033340                szWave
 .rodata        0x0103901c      0x474 obj/HDMI_Lib/HDMI_RX/HDMI_RX.o
                0x0103901c                szDefaultEDID
 .rodata        0x01039490      0xb1c obj/HDMI_Lib/HDMI_RX/it6605.o
 .rodata        0x01039fac       0x70 obj/HDMI_Lib/HDMI_TX/EDID.o
 .rodata        0x0103a01c      0x16c obj/HDMI_Lib/HDMI_TX/HDMI_TX.o
 .rodata        0x0103a188      0x8ac obj/HDMI_Lib/HDMI_TX/it6613_drv.o
 .rodata        0x0103aa34       0x34 obj/HDMI_Lib/HDMI_TX/it6613_sys.o
 .rodata        0x0103aa68       0x84 obj/HDMI_Lib/mcu.o
 .rodata        0x0103aaec      0x1ec obj/main.o
 .rodata        0x0103acd8       0x10 obj/terasic_lib/debug.o
 .rodata        0x0103ace8       0x14 c:/altera/11.1/nios2eds/bin/gnu/h-i686-mingw32/bin/../lib/gcc/nios2-elf/4.1.2/mhw-mulx\libgcc.a(_thenan_df.o)
                0x0103ace8                __thenan_df
 .rodata        0x0103acfc      0x100 c:/altera/11.1/nios2eds/bin/gnu/h-i686-mingw32/bin/../lib/gcc/nios2-elf/4.1.2/mhw-mulx\libgcc.a(_clz.o)
                0x0103acfc                __clz_tab
 .rodata.str1.4
                0x0103adfc        0x4 c:/altera/11.1/nios2eds/bin/gnu/h-i686-mingw32/bin/../lib/gcc/nios2-elf/4.1.2/../../../../nios2-elf/lib/mhw-mulx\libsmallc.a(lib_a-puts.o)
 .rodata        0x0103ae00       0x10 ../TR4_HDMI_TX_RX_bsp/\libhal_bsp.a(alt_main.o)
 .rodata        0x0103ae10       0x10 ../TR4_HDMI_TX_RX_bsp/\libhal_bsp.a(alt_sys_init.o)
 .rodata        0x0103ae20        0xc ../TR4_HDMI_TX_RX_bsp/\libhal_bsp.a(alt_dev.o)
 *(.rodata1)
                0x0103ae2c                . = ALIGN (0x4)
                0x0103ae2c                PROVIDE (__ram_rodata_end, ABSOLUTE (.))
                0x01033340                PROVIDE (__flash_rodata_start, LOADADDR (.rodata))

.rwdata         0x0103ae2c     0x1754 load address 0x0103c580
                0x0103ae2c                PROVIDE (__ram_rwdata_start, ABSOLUTE (.))
                0x0103ae2c                . = ALIGN (0x4)
 *(.got.plt)
 *(.got)
 *(.data1)
 *(.data .data.* .gnu.linkonce.d.*)
 .data          0x0103ae2c        0x0 ../TR4_HDMI_TX_RX_bsp//obj/HAL/src/crt0.o
 .data          0x0103ae2c        0x0 obj/Beep.o
 .data          0x0103ae2c        0x0 obj/HDMI_Lib/HDMI_RX/HDMI_RX.o
 .data          0x0103ae2c      0x934 obj/HDMI_Lib/HDMI_RX/it6605.o
                0x0103ae2c                VStateStr
                0x0103ae50                AStateStr
 .data          0x0103b760        0x0 obj/HDMI_Lib/HDMI_TX/EDID.o
 .data          0x0103b760       0x10 obj/HDMI_Lib/HDMI_TX/HDMI_TX.o
                0x0103b760                InitInstanceData
 .data          0x0103b770        0x0 obj/HDMI_Lib/HDMI_TX/dss_sha.o
 .data          0x0103b770      0x830 obj/HDMI_Lib/HDMI_TX/it6613_drv.o
                0x0103b7b8                bCSCMtx_YUV2RGB_ITU601_16_235
                0x0103b7ca                bCSCMtx_YUV2RGB_ITU601_0_255
                0x0103b7dc                bCSCMtx_YUV2RGB_ITU709_16_235
                0x0103b7ee                bCSCMtx_YUV2RGB_ITU709_0_255
 .data          0x0103bfa0        0x0 obj/HDMI_Lib/HDMI_TX/it6613_sys.o
 .data          0x0103bfa0        0x0 obj/HDMI_Lib/mcu.o
 .data          0x0103bfa0      0x2c0 obj/main.o
                0x0103bfa0                gszVicText
 .data          0x0103c260        0x0 obj/terasic_lib/I2C.o
 .data          0x0103c260        0x0 obj/terasic_lib/debug.o
 .data          0x0103c260        0x0 c:/altera/11.1/nios2eds/bin/gnu/h-i686-mingw32/bin/../lib/gcc/nios2-elf/4.1.2/mhw-mulx\libgcc.a(_mul_df.o)
 .data          0x0103c260        0x0 c:/altera/11.1/nios2eds/bin/gnu/h-i686-mingw32/bin/../lib/gcc/nios2-elf/4.1.2/mhw-mulx\libgcc.a(_div_df.o)
 .data          0x0103c260        0x0 c:/altera/11.1/nios2eds/bin/gnu/h-i686-mingw32/bin/../lib/gcc/nios2-elf/4.1.2/mhw-mulx\libgcc.a(_si_to_df.o)
 .data          0x0103c260        0x0 c:/altera/11.1/nios2eds/bin/gnu/h-i686-mingw32/bin/../lib/gcc/nios2-elf/4.1.2/mhw-mulx\libgcc.a(_thenan_df.o)
 .data          0x0103c260        0x0 c:/altera/11.1/nios2eds/bin/gnu/h-i686-mingw32/bin/../lib/gcc/nios2-elf/4.1.2/mhw-mulx\libgcc.a(lib2-divmod.o)
 .data          0x0103c260        0x0 c:/altera/11.1/nios2eds/bin/gnu/h-i686-mingw32/bin/../lib/gcc/nios2-elf/4.1.2/mhw-mulx\libgcc.a(_clzsi2.o)
 .data          0x0103c260        0x0 c:/altera/11.1/nios2eds/bin/gnu/h-i686-mingw32/bin/../lib/gcc/nios2-elf/4.1.2/mhw-mulx\libgcc.a(_pack_df.o)
 .data          0x0103c260        0x0 c:/altera/11.1/nios2eds/bin/gnu/h-i686-mingw32/bin/../lib/gcc/nios2-elf/4.1.2/mhw-mulx\libgcc.a(_unpack_df.o)
 .data          0x0103c260        0x0 c:/altera/11.1/nios2eds/bin/gnu/h-i686-mingw32/bin/../lib/gcc/nios2-elf/4.1.2/mhw-mulx\libgcc.a(_clz.o)
 .data          0x0103c260       0xe0 c:/altera/11.1/nios2eds/bin/gnu/h-i686-mingw32/bin/../lib/gcc/nios2-elf/4.1.2/../../../../nios2-elf/lib/mhw-mulx\libsmallc.a(lib_a-impure.o)
 .data          0x0103c340        0x0 c:/altera/11.1/nios2eds/bin/gnu/h-i686-mingw32/bin/../lib/gcc/nios2-elf/4.1.2/../../../../nios2-elf/lib/mhw-mulx\libsmallc.a(lib_a-memset.o)
 .data          0x0103c340        0x0 c:/altera/11.1/nios2eds/bin/gnu/h-i686-mingw32/bin/../lib/gcc/nios2-elf/4.1.2/../../../../nios2-elf/lib/mhw-mulx\libsmallc.a(lib_a-printf.o)
 .data          0x0103c340        0x0 c:/altera/11.1/nios2eds/bin/gnu/h-i686-mingw32/bin/../lib/gcc/nios2-elf/4.1.2/../../../../nios2-elf/lib/mhw-mulx\libsmallc.a(lib_a-putchar.o)
 .data          0x0103c340        0x0 c:/altera/11.1/nios2eds/bin/gnu/h-i686-mingw32/bin/../lib/gcc/nios2-elf/4.1.2/../../../../nios2-elf/lib/mhw-mulx\libsmallc.a(lib_a-puts.o)
 .data          0x0103c340        0x0 c:/altera/11.1/nios2eds/bin/gnu/h-i686-mingw32/bin/../lib/gcc/nios2-elf/4.1.2/../../../../nios2-elf/lib/mhw-mulx\libsmallc.a(lib_a-sprintf.o)
 .data          0x0103c340        0x0 c:/altera/11.1/nios2eds/bin/gnu/h-i686-mingw32/bin/../lib/gcc/nios2-elf/4.1.2/../../../../nios2-elf/lib/mhw-mulx\libsmallc.a(lib_a-strlen.o)
 .data          0x0103c340        0x0 c:/altera/11.1/nios2eds/bin/gnu/h-i686-mingw32/bin/../lib/gcc/nios2-elf/4.1.2/../../../../nios2-elf/lib/mhw-mulx\libsmallc.a(lib_a-vfprintf.o)
 .data          0x0103c340        0x0 c:/altera/11.1/nios2eds/bin/gnu/h-i686-mingw32/bin/../lib/gcc/nios2-elf/4.1.2/../../../../nios2-elf/lib/mhw-mulx\libsmallc.a(lib_a-vfprintf_1.o)
 .data          0x0103c340        0x0 c:/altera/11.1/nios2eds/bin/gnu/h-i686-mingw32/bin/../lib/gcc/nios2-elf/4.1.2/../../../../nios2-elf/lib/mhw-mulx\libsmallc.a(lib_a-vsnprintf.o)
 .data          0x0103c340        0x0 c:/altera/11.1/nios2eds/bin/gnu/h-i686-mingw32/bin/../lib/gcc/nios2-elf/4.1.2/../../../../nios2-elf/lib/mhw-mulx\libsmallc.a(lib_a-fvwrite_small_dev.o)
 .data          0x0103c340        0x0 c:/altera/11.1/nios2eds/bin/gnu/h-i686-mingw32/bin/../lib/gcc/nios2-elf/4.1.2/../../../../nios2-elf/lib/mhw-mulx\libsmallc.a(lib_a-fvwrite_small_str.o)
 .data          0x0103c340        0x0 c:/altera/11.1/nios2eds/bin/gnu/h-i686-mingw32/bin/../lib/gcc/nios2-elf/4.1.2/../../../../nios2-elf/lib/mhw-mulx\libsmallc.a(lib_a-memmove.o)
 .data          0x0103c340        0x0 c:/altera/11.1/nios2eds/bin/gnu/h-i686-mingw32/bin/../lib/gcc/nios2-elf/4.1.2/../../../../nios2-elf/lib/mhw-mulx\libsmallc.a(lib_a-putc.o)
 .data          0x0103c340        0x0 c:/altera/11.1/nios2eds/bin/gnu/h-i686-mingw32/bin/../lib/gcc/nios2-elf/4.1.2/../../../../nios2-elf/lib/mhw-mulx\libsmallc.a(lib_a-writer.o)
 .data          0x0103c340        0x0 c:/altera/11.1/nios2eds/bin/gnu/h-i686-mingw32/bin/../lib/gcc/nios2-elf/4.1.2/../../../../nios2-elf/lib/mhw-mulx\libsmallc.a(lib_a-int_errno.o)
 .data          0x0103c340        0x0 ../TR4_HDMI_TX_RX_bsp/\libhal_bsp.a(alt_irq_register.o)
 .data          0x0103c340        0x0 ../TR4_HDMI_TX_RX_bsp/\libhal_bsp.a(alt_irq_vars.o)
 .data          0x0103c340        0x0 ../TR4_HDMI_TX_RX_bsp/\libhal_bsp.a(alt_load.o)
 .data          0x0103c340        0x0 ../TR4_HDMI_TX_RX_bsp/\libhal_bsp.a(alt_main.o)
 .data          0x0103c340        0x0 ../TR4_HDMI_TX_RX_bsp/\libhal_bsp.a(alt_tick.o)
 .data          0x0103c340        0x0 ../TR4_HDMI_TX_RX_bsp/\libhal_bsp.a(alt_usleep.o)
 .data          0x0103c340        0x0 ../TR4_HDMI_TX_RX_bsp/\libhal_bsp.a(alt_write.o)
 .data          0x0103c340       0x2c ../TR4_HDMI_TX_RX_bsp/\libhal_bsp.a(alt_sys_init.o)
 .data          0x0103c36c        0x0 ../TR4_HDMI_TX_RX_bsp/\libhal_bsp.a(altera_avalon_jtag_uart_fd.o)
 .data          0x0103c36c        0x0 ../TR4_HDMI_TX_RX_bsp/\libhal_bsp.a(altera_avalon_jtag_uart_read.o)
 .data          0x0103c36c        0x0 ../TR4_HDMI_TX_RX_bsp/\libhal_bsp.a(altera_avalon_jtag_uart_write.o)
 .data          0x0103c36c        0x0 ../TR4_HDMI_TX_RX_bsp/\libhal_bsp.a(altera_avalon_timer_sc.o)
 .data          0x0103c36c        0x0 ../TR4_HDMI_TX_RX_bsp/\libhal_bsp.a(alt_busy_sleep.o)
 .data          0x0103c36c        0x0 ../TR4_HDMI_TX_RX_bsp/\libhal_bsp.a(alt_close.o)
 .data          0x0103c36c        0x0 ../TR4_HDMI_TX_RX_bsp/\libhal_bsp.a(alt_dcache_flush_all.o)
 .data          0x0103c36c      0x1a8 ../TR4_HDMI_TX_RX_bsp/\libhal_bsp.a(alt_dev.o)
                0x0103c36c                alt_dev_null
                0x0103c394                alt_fd_list
 .data          0x0103c514        0x0 ../TR4_HDMI_TX_RX_bsp/\libhal_bsp.a(alt_dev_llist_insert.o)
 .data          0x0103c514        0x0 ../TR4_HDMI_TX_RX_bsp/\libhal_bsp.a(alt_do_ctors.o)
 .data          0x0103c514        0x0 ../TR4_HDMI_TX_RX_bsp/\libhal_bsp.a(alt_do_dtors.o)
 .data          0x0103c514        0x0 ../TR4_HDMI_TX_RX_bsp/\libhal_bsp.a(alt_errno.o)
 .data          0x0103c514        0x0 ../TR4_HDMI_TX_RX_bsp/\libhal_bsp.a(alt_icache_flush_all.o)
 .data          0x0103c514        0x0 ../TR4_HDMI_TX_RX_bsp/\libhal_bsp.a(alt_iic.o)
 .data          0x0103c514        0x0 ../TR4_HDMI_TX_RX_bsp/\libhal_bsp.a(alt_iic_isr_register.o)
 .data          0x0103c514        0x0 ../TR4_HDMI_TX_RX_bsp/\libhal_bsp.a(alt_io_redirect.o)
 .data          0x0103c514        0x0 ../TR4_HDMI_TX_RX_bsp/\libhal_bsp.a(alt_irq_entry.o)
 .data          0x0103c514        0x0 ../TR4_HDMI_TX_RX_bsp/\libhal_bsp.a(alt_irq_handler.o)
 .data          0x0103c514        0x0 ../TR4_HDMI_TX_RX_bsp/\libhal_bsp.a(alt_open.o)
 .data          0x0103c514        0x0 ../TR4_HDMI_TX_RX_bsp/\libhal_bsp.a(alt_release_fd.o)
 .data          0x0103c514        0x0 ../TR4_HDMI_TX_RX_bsp/\libhal_bsp.a(altera_nios2_qsys_irq.o)
 .data          0x0103c514        0x0 ../TR4_HDMI_TX_RX_bsp/\libhal_bsp.a(alt_exception_entry.o)
 .data          0x0103c514        0x0 ../TR4_HDMI_TX_RX_bsp/\libhal_bsp.a(alt_find_dev.o)
 .data          0x0103c514        0x0 ../TR4_HDMI_TX_RX_bsp/\libhal_bsp.a(alt_find_file.o)
 .data          0x0103c514        0x0 ../TR4_HDMI_TX_RX_bsp/\libhal_bsp.a(alt_get_fd.o)
 .data          0x0103c514        0x0 ../TR4_HDMI_TX_RX_bsp/\libhal_bsp.a(alt_icache_flush.o)
 .data          0x0103c514        0x0 c:/altera/11.1/nios2eds/bin/gnu/h-i686-mingw32/bin/../lib/gcc/nios2-elf/4.1.2/../../../../nios2-elf/lib/mhw-mulx\libsmallc.a(lib_a-atexit.o)
 .data          0x0103c514        0x0 c:/altera/11.1/nios2eds/bin/gnu/h-i686-mingw32/bin/../lib/gcc/nios2-elf/4.1.2/../../../../nios2-elf/lib/mhw-mulx\libsmallc.a(lib_a-exit.o)
 .data          0x0103c514        0x0 c:/altera/11.1/nios2eds/bin/gnu/h-i686-mingw32/bin/../lib/gcc/nios2-elf/4.1.2/../../../../nios2-elf/lib/mhw-mulx\libsmallc.a(lib_a-memcmp.o)
 .data          0x0103c514        0x0 c:/altera/11.1/nios2eds/bin/gnu/h-i686-mingw32/bin/../lib/gcc/nios2-elf/4.1.2/../../../../nios2-elf/lib/mhw-mulx\libsmallc.a(lib_a-__atexit.o)
 .data          0x0103c514        0x0 c:/altera/11.1/nios2eds/bin/gnu/h-i686-mingw32/bin/../lib/gcc/nios2-elf/4.1.2/../../../../nios2-elf/lib/mhw-mulx\libsmallc.a(lib_a-__call_atexit.o)
 .data          0x0103c514        0x0 ../TR4_HDMI_TX_RX_bsp/\libhal_bsp.a(alt_exit.o)
                0x01044514                _gp = ABSOLUTE ((. + 0x8000))
                0x01044514                PROVIDE (gp, _gp)
 *(.rwdata .rwdata.*)
 *(.sdata .sdata.* .gnu.linkonce.s.*)
 .sdata         0x0103c514        0x4 obj/Beep.o
                0x0103c514                nWaveSize
 .sdata         0x0103c518       0x2c obj/HDMI_Lib/HDMI_RX/it6605.o
 .sdata         0x0103c544        0x6 obj/HDMI_Lib/HDMI_TX/it6613_drv.o
 *fill*         0x0103c54a        0x2 00
 .sdata         0x0103c54c        0x4 obj/HDMI_Lib/HDMI_TX/it6613_sys.o
                0x0103c54c                gEnableColorDepth
 .sdata         0x0103c550        0x4 obj/main.o
                0x0103c550                gbPlayTone
 .sdata         0x0103c554        0x8 c:/altera/11.1/nios2eds/bin/gnu/h-i686-mingw32/bin/../lib/gcc/nios2-elf/4.1.2/../../../../nios2-elf/lib/mhw-mulx\libsmallc.a(lib_a-impure.o)
                0x0103c554                _impure_ptr
                0x0103c558                _global_impure_ptr
 .sdata         0x0103c55c        0x4 ../TR4_HDMI_TX_RX_bsp/\libhal_bsp.a(alt_irq_vars.o)
                0x0103c55c                alt_priority_mask
 .sdata         0x0103c560        0x8 ../TR4_HDMI_TX_RX_bsp/\libhal_bsp.a(alt_tick.o)
                0x0103c560                alt_alarm_list
 .sdata         0x0103c568       0x14 ../TR4_HDMI_TX_RX_bsp/\libhal_bsp.a(alt_dev.o)
                0x0103c568                alt_fs_list
                0x0103c570                alt_dev_list
                0x0103c578                alt_max_fd
 .sdata         0x0103c57c        0x4 ../TR4_HDMI_TX_RX_bsp/\libhal_bsp.a(alt_errno.o)
                0x0103c57c                alt_errno
 *(.sdata2 .sdata2.* .gnu.linkonce.s2.*)
                0x0103c580                . = ALIGN (0x4)
                0x0103c580                _edata = ABSOLUTE (.)
                0x0103c580                PROVIDE (edata, ABSOLUTE (.))
                0x0103c580                PROVIDE (__ram_rwdata_end, ABSOLUTE (.))
                0x0103c580                PROVIDE (__flash_rwdata_start, LOADADDR (.rwdata))

.bss            0x0103dcd4      0x64c
                0x0103dcd4                __bss_start = ABSOLUTE (.)
                0x0103dcd4                PROVIDE (__sbss_start, ABSOLUTE (.))
                0x0103dcd4                PROVIDE (___sbss_start, ABSOLUTE (.))
 *(.dynsbss)
 *(.sbss .sbss.* .gnu.linkonce.sb.*)
 .sbss          0x0103dcd4       0x18 obj/HDMI_Lib/HDMI_RX/HDMI_RX.o
 .sbss          0x0103dcec       0x48 obj/HDMI_Lib/HDMI_RX/it6605.o
                0x0103dcec                VState
                0x0103dcf0                AState
                0x0103dd01                bDisableAutoAVMute
                0x0103dd02                bHDCPMode
                0x0103dd04                bIntPOL
 .sbss          0x0103dd34        0x8 obj/HDMI_Lib/HDMI_TX/HDMI_TX.o
                0x0103dd34                TX_HDP
 .sbss          0x0103dd3c        0x9 obj/HDMI_Lib/HDMI_TX/it6613_drv.o
 *fill*         0x0103dd45        0x3 00
 .sbss          0x0103dd48        0x8 obj/HDMI_Lib/HDMI_TX/it6613_sys.o
                0x0103dd48                bChangeMode
                0x0103dd4c                bInputColorMode
                0x0103dd4d                bInputSignalType
                0x0103dd4e                iVideoModeSelect
                0x0103dd4f                bOutputColorMode
 .sbss          0x0103dd50       0x19 obj/HDMI_Lib/HDMI_TX/it6613_sys.o
                0x0103dd50                VideoPixelClock
                0x0103dd54                aspec
                0x0103dd58                Colorimetry
                0x0103dd5c                pixelrep
                0x0103dd60                bHDMIMode
                0x0103dd64                bAudioEnable
                0x0103dd68                VIC
 *fill*         0x0103dd69        0x3 00
 .sbss          0x0103dd6c        0x8 obj/HDMI_Lib/mcu.o
 .sbss          0x0103dd74       0x14 obj/main.o
                0x0103dd74                gDemoMode
                0x0103dd78                gVpgMode
                0x0103dd7c                gVpgColor
 .sbss          0x0103dd88        0x4 c:/altera/11.1/nios2eds/bin/gnu/h-i686-mingw32/bin/../lib/gcc/nios2-elf/4.1.2/../../../../nios2-elf/lib/mhw-mulx\libsmallc.a(lib_a-int_errno.o)
                0x0103dd88                errno
 .sbss          0x0103dd8c        0x4 ../TR4_HDMI_TX_RX_bsp/\libhal_bsp.a(alt_irq_vars.o)
                0x0103dd8c                alt_irq_active
 .sbss          0x0103dd90        0xc ../TR4_HDMI_TX_RX_bsp/\libhal_bsp.a(alt_main.o)
                0x0103dd90                alt_argc
                0x0103dd94                alt_argv
                0x0103dd98                alt_envp
 .sbss          0x0103dd9c        0x8 ../TR4_HDMI_TX_RX_bsp/\libhal_bsp.a(alt_tick.o)
                0x0103dd9c                _alt_tick_rate
                0x0103dda0                _alt_nticks
 *(.sbss2 .sbss2.* .gnu.linkonce.sb2.*)
 *(.scommon)
                0x0103dda4                PROVIDE (__sbss_end, ABSOLUTE (.))
                0x0103dda4                PROVIDE (___sbss_end, ABSOLUTE (.))
 *(.dynbss)
 *(.bss .bss.* .gnu.linkonce.b.*)
 .bss           0x0103dda4        0x0 ../TR4_HDMI_TX_RX_bsp//obj/HAL/src/crt0.o
 .bss           0x0103dda4        0x0 obj/Beep.o
 .bss           0x0103dda4        0x0 obj/HDMI_Lib/HDMI_RX/HDMI_RX.o
 .bss           0x0103dda4       0x6c obj/HDMI_Lib/HDMI_RX/it6605.o
 .bss           0x0103de10        0x0 obj/HDMI_Lib/HDMI_TX/EDID.o
 .bss           0x0103de10        0x0 obj/HDMI_Lib/HDMI_TX/HDMI_TX.o
 .bss           0x0103de10        0x0 obj/HDMI_Lib/HDMI_TX/dss_sha.o
 .bss           0x0103de10      0x1dc obj/HDMI_Lib/HDMI_TX/it6613_drv.o
 .bss           0x0103dfec       0x80 obj/HDMI_Lib/HDMI_TX/it6613_sys.o
 .bss           0x0103e06c        0x0 obj/HDMI_Lib/mcu.o
 .bss           0x0103e06c        0x0 obj/main.o
 .bss           0x0103e06c        0x0 obj/terasic_lib/I2C.o
 .bss           0x0103e06c        0x0 obj/terasic_lib/debug.o
 .bss           0x0103e06c        0x0 c:/altera/11.1/nios2eds/bin/gnu/h-i686-mingw32/bin/../lib/gcc/nios2-elf/4.1.2/mhw-mulx\libgcc.a(_mul_df.o)
 .bss           0x0103e06c        0x0 c:/altera/11.1/nios2eds/bin/gnu/h-i686-mingw32/bin/../lib/gcc/nios2-elf/4.1.2/mhw-mulx\libgcc.a(_div_df.o)
 .bss           0x0103e06c        0x0 c:/altera/11.1/nios2eds/bin/gnu/h-i686-mingw32/bin/../lib/gcc/nios2-elf/4.1.2/mhw-mulx\libgcc.a(_si_to_df.o)
 .bss           0x0103e06c        0x0 c:/altera/11.1/nios2eds/bin/gnu/h-i686-mingw32/bin/../lib/gcc/nios2-elf/4.1.2/mhw-mulx\libgcc.a(_thenan_df.o)
 .bss           0x0103e06c        0x0 c:/altera/11.1/nios2eds/bin/gnu/h-i686-mingw32/bin/../lib/gcc/nios2-elf/4.1.2/mhw-mulx\libgcc.a(lib2-divmod.o)
 .bss           0x0103e06c        0x0 c:/altera/11.1/nios2eds/bin/gnu/h-i686-mingw32/bin/../lib/gcc/nios2-elf/4.1.2/mhw-mulx\libgcc.a(_clzsi2.o)
 .bss           0x0103e06c        0x0 c:/altera/11.1/nios2eds/bin/gnu/h-i686-mingw32/bin/../lib/gcc/nios2-elf/4.1.2/mhw-mulx\libgcc.a(_pack_df.o)
 .bss           0x0103e06c        0x0 c:/altera/11.1/nios2eds/bin/gnu/h-i686-mingw32/bin/../lib/gcc/nios2-elf/4.1.2/mhw-mulx\libgcc.a(_unpack_df.o)
 .bss           0x0103e06c        0x0 c:/altera/11.1/nios2eds/bin/gnu/h-i686-mingw32/bin/../lib/gcc/nios2-elf/4.1.2/mhw-mulx\libgcc.a(_clz.o)
 .bss           0x0103e06c        0x0 c:/altera/11.1/nios2eds/bin/gnu/h-i686-mingw32/bin/../lib/gcc/nios2-elf/4.1.2/../../../../nios2-elf/lib/mhw-mulx\libsmallc.a(lib_a-impure.o)
 .bss           0x0103e06c        0x0 c:/altera/11.1/nios2eds/bin/gnu/h-i686-mingw32/bin/../lib/gcc/nios2-elf/4.1.2/../../../../nios2-elf/lib/mhw-mulx\libsmallc.a(lib_a-memset.o)
 .bss           0x0103e06c        0x0 c:/altera/11.1/nios2eds/bin/gnu/h-i686-mingw32/bin/../lib/gcc/nios2-elf/4.1.2/../../../../nios2-elf/lib/mhw-mulx\libsmallc.a(lib_a-printf.o)
 .bss           0x0103e06c        0x0 c:/altera/11.1/nios2eds/bin/gnu/h-i686-mingw32/bin/../lib/gcc/nios2-elf/4.1.2/../../../../nios2-elf/lib/mhw-mulx\libsmallc.a(lib_a-putchar.o)
 .bss           0x0103e06c        0x0 c:/altera/11.1/nios2eds/bin/gnu/h-i686-mingw32/bin/../lib/gcc/nios2-elf/4.1.2/../../../../nios2-elf/lib/mhw-mulx\libsmallc.a(lib_a-puts.o)
 .bss           0x0103e06c        0x0 c:/altera/11.1/nios2eds/bin/gnu/h-i686-mingw32/bin/../lib/gcc/nios2-elf/4.1.2/../../../../nios2-elf/lib/mhw-mulx\libsmallc.a(lib_a-sprintf.o)
 .bss           0x0103e06c        0x0 c:/altera/11.1/nios2eds/bin/gnu/h-i686-mingw32/bin/../lib/gcc/nios2-elf/4.1.2/../../../../nios2-elf/lib/mhw-mulx\libsmallc.a(lib_a-strlen.o)
 .bss           0x0103e06c        0x0 c:/altera/11.1/nios2eds/bin/gnu/h-i686-mingw32/bin/../lib/gcc/nios2-elf/4.1.2/../../../../nios2-elf/lib/mhw-mulx\libsmallc.a(lib_a-vfprintf.o)
 .bss           0x0103e06c        0x0 c:/altera/11.1/nios2eds/bin/gnu/h-i686-mingw32/bin/../lib/gcc/nios2-elf/4.1.2/../../../../nios2-elf/lib/mhw-mulx\libsmallc.a(lib_a-vfprintf_1.o)
 .bss           0x0103e06c        0x0 c:/altera/11.1/nios2eds/bin/gnu/h-i686-mingw32/bin/../lib/gcc/nios2-elf/4.1.2/../../../../nios2-elf/lib/mhw-mulx\libsmallc.a(lib_a-vsnprintf.o)
 .bss           0x0103e06c        0x0 c:/altera/11.1/nios2eds/bin/gnu/h-i686-mingw32/bin/../lib/gcc/nios2-elf/4.1.2/../../../../nios2-elf/lib/mhw-mulx\libsmallc.a(lib_a-fvwrite_small_dev.o)
 .bss           0x0103e06c        0x0 c:/altera/11.1/nios2eds/bin/gnu/h-i686-mingw32/bin/../lib/gcc/nios2-elf/4.1.2/../../../../nios2-elf/lib/mhw-mulx\libsmallc.a(lib_a-fvwrite_small_str.o)
 .bss           0x0103e06c        0x0 c:/altera/11.1/nios2eds/bin/gnu/h-i686-mingw32/bin/../lib/gcc/nios2-elf/4.1.2/../../../../nios2-elf/lib/mhw-mulx\libsmallc.a(lib_a-memmove.o)
 .bss           0x0103e06c        0x0 c:/altera/11.1/nios2eds/bin/gnu/h-i686-mingw32/bin/../lib/gcc/nios2-elf/4.1.2/../../../../nios2-elf/lib/mhw-mulx\libsmallc.a(lib_a-putc.o)
 .bss           0x0103e06c        0x0 c:/altera/11.1/nios2eds/bin/gnu/h-i686-mingw32/bin/../lib/gcc/nios2-elf/4.1.2/../../../../nios2-elf/lib/mhw-mulx\libsmallc.a(lib_a-writer.o)
 .bss           0x0103e06c        0x0 c:/altera/11.1/nios2eds/bin/gnu/h-i686-mingw32/bin/../lib/gcc/nios2-elf/4.1.2/../../../../nios2-elf/lib/mhw-mulx\libsmallc.a(lib_a-int_errno.o)
 .bss           0x0103e06c        0x0 ../TR4_HDMI_TX_RX_bsp/\libhal_bsp.a(alt_irq_register.o)
 .bss           0x0103e06c        0x0 ../TR4_HDMI_TX_RX_bsp/\libhal_bsp.a(alt_irq_vars.o)
 .bss           0x0103e06c        0x0 ../TR4_HDMI_TX_RX_bsp/\libhal_bsp.a(alt_load.o)
 .bss           0x0103e06c        0x0 ../TR4_HDMI_TX_RX_bsp/\libhal_bsp.a(alt_main.o)
 .bss           0x0103e06c        0x0 ../TR4_HDMI_TX_RX_bsp/\libhal_bsp.a(alt_tick.o)
 .bss           0x0103e06c        0x0 ../TR4_HDMI_TX_RX_bsp/\libhal_bsp.a(alt_usleep.o)
 .bss           0x0103e06c        0x0 ../TR4_HDMI_TX_RX_bsp/\libhal_bsp.a(alt_write.o)
 .bss           0x0103e06c        0x0 ../TR4_HDMI_TX_RX_bsp/\libhal_bsp.a(alt_sys_init.o)
 .bss           0x0103e06c        0x0 ../TR4_HDMI_TX_RX_bsp/\libhal_bsp.a(altera_avalon_jtag_uart_fd.o)
 .bss           0x0103e06c        0x0 ../TR4_HDMI_TX_RX_bsp/\libhal_bsp.a(altera_avalon_jtag_uart_read.o)
 .bss           0x0103e06c        0x0 ../TR4_HDMI_TX_RX_bsp/\libhal_bsp.a(altera_avalon_jtag_uart_write.o)
 .bss           0x0103e06c        0x0 ../TR4_HDMI_TX_RX_bsp/\libhal_bsp.a(altera_avalon_timer_sc.o)
 .bss           0x0103e06c        0x0 ../TR4_HDMI_TX_RX_bsp/\libhal_bsp.a(alt_busy_sleep.o)
 .bss           0x0103e06c        0x0 ../TR4_HDMI_TX_RX_bsp/\libhal_bsp.a(alt_close.o)
 .bss           0x0103e06c        0x0 ../TR4_HDMI_TX_RX_bsp/\libhal_bsp.a(alt_dcache_flush_all.o)
 .bss           0x0103e06c        0x0 ../TR4_HDMI_TX_RX_bsp/\libhal_bsp.a(alt_dev.o)
 .bss           0x0103e06c        0x0 ../TR4_HDMI_TX_RX_bsp/\libhal_bsp.a(alt_dev_llist_insert.o)
 .bss           0x0103e06c        0x0 ../TR4_HDMI_TX_RX_bsp/\libhal_bsp.a(alt_do_ctors.o)
 .bss           0x0103e06c        0x0 ../TR4_HDMI_TX_RX_bsp/\libhal_bsp.a(alt_do_dtors.o)
 .bss           0x0103e06c        0x0 ../TR4_HDMI_TX_RX_bsp/\libhal_bsp.a(alt_errno.o)
 .bss           0x0103e06c        0x0 ../TR4_HDMI_TX_RX_bsp/\libhal_bsp.a(alt_icache_flush_all.o)
 .bss           0x0103e06c        0x0 ../TR4_HDMI_TX_RX_bsp/\libhal_bsp.a(alt_iic.o)
 .bss           0x0103e06c        0x0 ../TR4_HDMI_TX_RX_bsp/\libhal_bsp.a(alt_iic_isr_register.o)
 .bss           0x0103e06c        0x0 ../TR4_HDMI_TX_RX_bsp/\libhal_bsp.a(alt_io_redirect.o)
 .bss           0x0103e06c        0x0 ../TR4_HDMI_TX_RX_bsp/\libhal_bsp.a(alt_irq_entry.o)
 .bss           0x0103e06c        0x0 ../TR4_HDMI_TX_RX_bsp/\libhal_bsp.a(alt_irq_handler.o)
 .bss           0x0103e06c        0x0 ../TR4_HDMI_TX_RX_bsp/\libhal_bsp.a(alt_open.o)
 .bss           0x0103e06c        0x0 ../TR4_HDMI_TX_RX_bsp/\libhal_bsp.a(alt_release_fd.o)
 .bss           0x0103e06c        0x0 ../TR4_HDMI_TX_RX_bsp/\libhal_bsp.a(altera_nios2_qsys_irq.o)
 .bss           0x0103e06c        0x0 ../TR4_HDMI_TX_RX_bsp/\libhal_bsp.a(alt_exception_entry.o)
 .bss           0x0103e06c        0x0 ../TR4_HDMI_TX_RX_bsp/\libhal_bsp.a(alt_find_dev.o)
 .bss           0x0103e06c        0x0 ../TR4_HDMI_TX_RX_bsp/\libhal_bsp.a(alt_find_file.o)
 .bss           0x0103e06c        0x0 ../TR4_HDMI_TX_RX_bsp/\libhal_bsp.a(alt_get_fd.o)
 .bss           0x0103e06c        0x0 ../TR4_HDMI_TX_RX_bsp/\libhal_bsp.a(alt_icache_flush.o)
 .bss           0x0103e06c        0x0 c:/altera/11.1/nios2eds/bin/gnu/h-i686-mingw32/bin/../lib/gcc/nios2-elf/4.1.2/../../../../nios2-elf/lib/mhw-mulx\libsmallc.a(lib_a-atexit.o)
 .bss           0x0103e06c        0x0 c:/altera/11.1/nios2eds/bin/gnu/h-i686-mingw32/bin/../lib/gcc/nios2-elf/4.1.2/../../../../nios2-elf/lib/mhw-mulx\libsmallc.a(lib_a-exit.o)
 .bss           0x0103e06c        0x0 c:/altera/11.1/nios2eds/bin/gnu/h-i686-mingw32/bin/../lib/gcc/nios2-elf/4.1.2/../../../../nios2-elf/lib/mhw-mulx\libsmallc.a(lib_a-memcmp.o)
 .bss           0x0103e06c        0x0 c:/altera/11.1/nios2eds/bin/gnu/h-i686-mingw32/bin/../lib/gcc/nios2-elf/4.1.2/../../../../nios2-elf/lib/mhw-mulx\libsmallc.a(lib_a-__atexit.o)
 .bss           0x0103e06c        0x0 c:/altera/11.1/nios2eds/bin/gnu/h-i686-mingw32/bin/../lib/gcc/nios2-elf/4.1.2/../../../../nios2-elf/lib/mhw-mulx\libsmallc.a(lib_a-__call_atexit.o)
 .bss           0x0103e06c        0x0 ../TR4_HDMI_TX_RX_bsp/\libhal_bsp.a(alt_exit.o)
 *(COMMON)
 COMMON         0x0103e06c       0x10 obj/HDMI_Lib/HDMI_TX/it6613_drv.o
                0x0103e06c                Instance
 COMMON         0x0103e07c      0x118 obj/HDMI_Lib/HDMI_TX/it6613_sys.o
                0x0103e07c                AudioInfo
                0x0103e08c                RxCapability
                0x0103e184                AviInfo
 COMMON         0x0103e194      0x100 ../TR4_HDMI_TX_RX_bsp/\libhal_bsp.a(alt_irq_handler.o)
                0x0103e194                alt_irq
 COMMON         0x0103e294       0x8c c:/altera/11.1/nios2eds/bin/gnu/h-i686-mingw32/bin/../lib/gcc/nios2-elf/4.1.2/../../../../nios2-elf/lib/mhw-mulx\libsmallc.a(lib_a-atexit.o)
                0x0103e294                _atexit0
                0x0103e320                . = ALIGN (0x4)
                0x0103e320                __bss_end = ABSOLUTE (.)

.onchip_memory2
                0x0103e320        0x0
                0x0103e320                PROVIDE (_alt_partition_onchip_memory2_start, ABSOLUTE (.))
 *(.onchip_memory2. onchip_memory2.*)
                0x0103e320                . = ALIGN (0x4)
                0x0103e320                PROVIDE (_alt_partition_onchip_memory2_end, ABSOLUTE (.))
                0x0103e320                _end = ABSOLUTE (.)
                0x0103e320                end = ABSOLUTE (.)
                0x0103e320                __alt_stack_base = ABSOLUTE (.)
                0x0103e320                PROVIDE (_alt_partition_onchip_memory2_load_addr, LOADADDR (.onchip_memory2))

.stab
 *(.stab)

.stabstr
 *(.stabstr)

.stab.excl
 *(.stab.excl)

.stab.exclstr
 *(.stab.exclstr)

.stab.index
 *(.stab.index)

.stab.indexstr
 *(.stab.indexstr)

.comment        0x00000000       0x26
 *(.comment)
 .comment       0x00000000       0x26 obj/Beep.o
                                 0x27 (size before relaxing)
 .comment       0x00000000       0x27 obj/HDMI_Lib/HDMI_RX/HDMI_RX.o
 .comment       0x00000000       0x27 obj/HDMI_Lib/HDMI_RX/it6605.o
 .comment       0x00000000       0x27 obj/HDMI_Lib/HDMI_TX/EDID.o
 .comment       0x00000000       0x27 obj/HDMI_Lib/HDMI_TX/HDMI_TX.o
 .comment       0x00000000       0x27 obj/HDMI_Lib/HDMI_TX/dss_sha.o
 .comment       0x00000000       0x27 obj/HDMI_Lib/HDMI_TX/it6613_drv.o
 .comment       0x00000000       0x27 obj/HDMI_Lib/HDMI_TX/it6613_sys.o
 .comment       0x00000000       0x27 obj/HDMI_Lib/mcu.o
 .comment       0x00000000       0x27 obj/main.o
 .comment       0x00000000       0x27 obj/terasic_lib/I2C.o
 .comment       0x00000000       0x27 obj/terasic_lib/debug.o
 .comment       0x00000000       0x27 c:/altera/11.1/nios2eds/bin/gnu/h-i686-mingw32/bin/../lib/gcc/nios2-elf/4.1.2/mhw-mulx\libgcc.a(_mul_df.o)
 .comment       0x00000000       0x27 c:/altera/11.1/nios2eds/bin/gnu/h-i686-mingw32/bin/../lib/gcc/nios2-elf/4.1.2/mhw-mulx\libgcc.a(_div_df.o)
 .comment       0x00000000       0x27 c:/altera/11.1/nios2eds/bin/gnu/h-i686-mingw32/bin/../lib/gcc/nios2-elf/4.1.2/mhw-mulx\libgcc.a(_si_to_df.o)
 .comment       0x00000000       0x27 c:/altera/11.1/nios2eds/bin/gnu/h-i686-mingw32/bin/../lib/gcc/nios2-elf/4.1.2/mhw-mulx\libgcc.a(_thenan_df.o)
 .comment       0x00000000       0x27 c:/altera/11.1/nios2eds/bin/gnu/h-i686-mingw32/bin/../lib/gcc/nios2-elf/4.1.2/mhw-mulx\libgcc.a(lib2-divmod.o)
 .comment       0x00000000       0x27 c:/altera/11.1/nios2eds/bin/gnu/h-i686-mingw32/bin/../lib/gcc/nios2-elf/4.1.2/mhw-mulx\libgcc.a(_clzsi2.o)
 .comment       0x00000000       0x27 c:/altera/11.1/nios2eds/bin/gnu/h-i686-mingw32/bin/../lib/gcc/nios2-elf/4.1.2/mhw-mulx\libgcc.a(_pack_df.o)
 .comment       0x00000000       0x27 c:/altera/11.1/nios2eds/bin/gnu/h-i686-mingw32/bin/../lib/gcc/nios2-elf/4.1.2/mhw-mulx\libgcc.a(_unpack_df.o)
 .comment       0x00000000       0x27 c:/altera/11.1/nios2eds/bin/gnu/h-i686-mingw32/bin/../lib/gcc/nios2-elf/4.1.2/mhw-mulx\libgcc.a(_clz.o)
 .comment       0x00000000       0x27 c:/altera/11.1/nios2eds/bin/gnu/h-i686-mingw32/bin/../lib/gcc/nios2-elf/4.1.2/../../../../nios2-elf/lib/mhw-mulx\libsmallc.a(lib_a-impure.o)
 .comment       0x00000000       0x27 c:/altera/11.1/nios2eds/bin/gnu/h-i686-mingw32/bin/../lib/gcc/nios2-elf/4.1.2/../../../../nios2-elf/lib/mhw-mulx\libsmallc.a(lib_a-memset.o)
 .comment       0x00000000       0x27 c:/altera/11.1/nios2eds/bin/gnu/h-i686-mingw32/bin/../lib/gcc/nios2-elf/4.1.2/../../../../nios2-elf/lib/mhw-mulx\libsmallc.a(lib_a-printf.o)
 .comment       0x00000000       0x27 c:/altera/11.1/nios2eds/bin/gnu/h-i686-mingw32/bin/../lib/gcc/nios2-elf/4.1.2/../../../../nios2-elf/lib/mhw-mulx\libsmallc.a(lib_a-putchar.o)
 .comment       0x00000000       0x27 c:/altera/11.1/nios2eds/bin/gnu/h-i686-mingw32/bin/../lib/gcc/nios2-elf/4.1.2/../../../../nios2-elf/lib/mhw-mulx\libsmallc.a(lib_a-puts.o)
 .comment       0x00000000       0x27 c:/altera/11.1/nios2eds/bin/gnu/h-i686-mingw32/bin/../lib/gcc/nios2-elf/4.1.2/../../../../nios2-elf/lib/mhw-mulx\libsmallc.a(lib_a-sprintf.o)
 .comment       0x00000000       0x27 c:/altera/11.1/nios2eds/bin/gnu/h-i686-mingw32/bin/../lib/gcc/nios2-elf/4.1.2/../../../../nios2-elf/lib/mhw-mulx\libsmallc.a(lib_a-strlen.o)
 .comment       0x00000000       0x27 c:/altera/11.1/nios2eds/bin/gnu/h-i686-mingw32/bin/../lib/gcc/nios2-elf/4.1.2/../../../../nios2-elf/lib/mhw-mulx\libsmallc.a(lib_a-vfprintf.o)
 .comment       0x00000000       0x27 c:/altera/11.1/nios2eds/bin/gnu/h-i686-mingw32/bin/../lib/gcc/nios2-elf/4.1.2/../../../../nios2-elf/lib/mhw-mulx\libsmallc.a(lib_a-vfprintf_1.o)
 .comment       0x00000000       0x27 c:/altera/11.1/nios2eds/bin/gnu/h-i686-mingw32/bin/../lib/gcc/nios2-elf/4.1.2/../../../../nios2-elf/lib/mhw-mulx\libsmallc.a(lib_a-vsnprintf.o)
 .comment       0x00000000       0x27 c:/altera/11.1/nios2eds/bin/gnu/h-i686-mingw32/bin/../lib/gcc/nios2-elf/4.1.2/../../../../nios2-elf/lib/mhw-mulx\libsmallc.a(lib_a-fvwrite_small_dev.o)
 .comment       0x00000000       0x27 c:/altera/11.1/nios2eds/bin/gnu/h-i686-mingw32/bin/../lib/gcc/nios2-elf/4.1.2/../../../../nios2-elf/lib/mhw-mulx\libsmallc.a(lib_a-fvwrite_small_str.o)
 .comment       0x00000000       0x27 c:/altera/11.1/nios2eds/bin/gnu/h-i686-mingw32/bin/../lib/gcc/nios2-elf/4.1.2/../../../../nios2-elf/lib/mhw-mulx\libsmallc.a(lib_a-memmove.o)
 .comment       0x00000000       0x27 c:/altera/11.1/nios2eds/bin/gnu/h-i686-mingw32/bin/../lib/gcc/nios2-elf/4.1.2/../../../../nios2-elf/lib/mhw-mulx\libsmallc.a(lib_a-putc.o)
 .comment       0x00000000       0x27 c:/altera/11.1/nios2eds/bin/gnu/h-i686-mingw32/bin/../lib/gcc/nios2-elf/4.1.2/../../../../nios2-elf/lib/mhw-mulx\libsmallc.a(lib_a-writer.o)
 .comment       0x00000000       0x27 c:/altera/11.1/nios2eds/bin/gnu/h-i686-mingw32/bin/../lib/gcc/nios2-elf/4.1.2/../../../../nios2-elf/lib/mhw-mulx\libsmallc.a(lib_a-int_errno.o)
 .comment       0x00000000       0x27 ../TR4_HDMI_TX_RX_bsp/\libhal_bsp.a(alt_irq_register.o)
 .comment       0x00000000       0x27 ../TR4_HDMI_TX_RX_bsp/\libhal_bsp.a(alt_irq_vars.o)
 .comment       0x00000000       0x27 ../TR4_HDMI_TX_RX_bsp/\libhal_bsp.a(alt_load.o)
 .comment       0x00000000       0x27 ../TR4_HDMI_TX_RX_bsp/\libhal_bsp.a(alt_main.o)
 .comment       0x00000000       0x27 ../TR4_HDMI_TX_RX_bsp/\libhal_bsp.a(alt_tick.o)
 .comment       0x00000000       0x27 ../TR4_HDMI_TX_RX_bsp/\libhal_bsp.a(alt_usleep.o)
 .comment       0x00000000       0x27 ../TR4_HDMI_TX_RX_bsp/\libhal_bsp.a(alt_write.o)
 .comment       0x00000000       0x27 ../TR4_HDMI_TX_RX_bsp/\libhal_bsp.a(alt_sys_init.o)
 .comment       0x00000000       0x27 ../TR4_HDMI_TX_RX_bsp/\libhal_bsp.a(altera_avalon_jtag_uart_fd.o)
 .comment       0x00000000       0x27 ../TR4_HDMI_TX_RX_bsp/\libhal_bsp.a(altera_avalon_jtag_uart_read.o)
 .comment       0x00000000       0x27 ../TR4_HDMI_TX_RX_bsp/\libhal_bsp.a(altera_avalon_jtag_uart_write.o)
 .comment       0x00000000       0x27 ../TR4_HDMI_TX_RX_bsp/\libhal_bsp.a(altera_avalon_timer_sc.o)
 .comment       0x00000000       0x27 ../TR4_HDMI_TX_RX_bsp/\libhal_bsp.a(alt_busy_sleep.o)
 .comment       0x00000000       0x27 ../TR4_HDMI_TX_RX_bsp/\libhal_bsp.a(alt_close.o)
 .comment       0x00000000       0x27 ../TR4_HDMI_TX_RX_bsp/\libhal_bsp.a(alt_dcache_flush_all.o)
 .comment       0x00000000       0x27 ../TR4_HDMI_TX_RX_bsp/\libhal_bsp.a(alt_dev.o)
 .comment       0x00000000       0x27 ../TR4_HDMI_TX_RX_bsp/\libhal_bsp.a(alt_dev_llist_insert.o)
 .comment       0x00000000       0x27 ../TR4_HDMI_TX_RX_bsp/\libhal_bsp.a(alt_do_ctors.o)
 .comment       0x00000000       0x27 ../TR4_HDMI_TX_RX_bsp/\libhal_bsp.a(alt_do_dtors.o)
 .comment       0x00000000       0x27 ../TR4_HDMI_TX_RX_bsp/\libhal_bsp.a(alt_errno.o)
 .comment       0x00000000       0x27 ../TR4_HDMI_TX_RX_bsp/\libhal_bsp.a(alt_icache_flush_all.o)
 .comment       0x00000000       0x27 ../TR4_HDMI_TX_RX_bsp/\libhal_bsp.a(alt_iic.o)
 .comment       0x00000000       0x27 ../TR4_HDMI_TX_RX_bsp/\libhal_bsp.a(alt_iic_isr_register.o)
 .comment       0x00000000       0x27 ../TR4_HDMI_TX_RX_bsp/\libhal_bsp.a(alt_io_redirect.o)
 .comment       0x00000000       0x27 ../TR4_HDMI_TX_RX_bsp/\libhal_bsp.a(alt_irq_handler.o)
 .comment       0x00000000       0x27 ../TR4_HDMI_TX_RX_bsp/\libhal_bsp.a(alt_open.o)
 .comment       0x00000000       0x27 ../TR4_HDMI_TX_RX_bsp/\libhal_bsp.a(alt_release_fd.o)
 .comment       0x00000000       0x27 ../TR4_HDMI_TX_RX_bsp/\libhal_bsp.a(altera_nios2_qsys_irq.o)
 .comment       0x00000000       0x27 ../TR4_HDMI_TX_RX_bsp/\libhal_bsp.a(alt_find_dev.o)
 .comment       0x00000000       0x27 ../TR4_HDMI_TX_RX_bsp/\libhal_bsp.a(alt_find_file.o)
 .comment       0x00000000       0x27 ../TR4_HDMI_TX_RX_bsp/\libhal_bsp.a(alt_get_fd.o)
 .comment       0x00000000       0x27 ../TR4_HDMI_TX_RX_bsp/\libhal_bsp.a(alt_icache_flush.o)
 .comment       0x00000000       0x27 c:/altera/11.1/nios2eds/bin/gnu/h-i686-mingw32/bin/../lib/gcc/nios2-elf/4.1.2/../../../../nios2-elf/lib/mhw-mulx\libsmallc.a(lib_a-atexit.o)
 .comment       0x00000000       0x27 c:/altera/11.1/nios2eds/bin/gnu/h-i686-mingw32/bin/../lib/gcc/nios2-elf/4.1.2/../../../../nios2-elf/lib/mhw-mulx\libsmallc.a(lib_a-exit.o)
 .comment       0x00000000       0x27 c:/altera/11.1/nios2eds/bin/gnu/h-i686-mingw32/bin/../lib/gcc/nios2-elf/4.1.2/../../../../nios2-elf/lib/mhw-mulx\libsmallc.a(lib_a-memcmp.o)
 .comment       0x00000000       0x27 c:/altera/11.1/nios2eds/bin/gnu/h-i686-mingw32/bin/../lib/gcc/nios2-elf/4.1.2/../../../../nios2-elf/lib/mhw-mulx\libsmallc.a(lib_a-__atexit.o)
 .comment       0x00000000       0x27 c:/altera/11.1/nios2eds/bin/gnu/h-i686-mingw32/bin/../lib/gcc/nios2-elf/4.1.2/../../../../nios2-elf/lib/mhw-mulx\libsmallc.a(lib_a-__call_atexit.o)
 .comment       0x00000000       0x27 ../TR4_HDMI_TX_RX_bsp/\libhal_bsp.a(alt_exit.o)

.debug
 *(.debug)

.line
 *(.line)

.debug_srcinfo
 *(.debug_srcinfo)

.debug_sfnames
 *(.debug_sfnames)

.debug_aranges  0x00000000      0x8f8
 *(.debug_aranges)
 .debug_aranges
                0x00000000       0x28 ../TR4_HDMI_TX_RX_bsp//obj/HAL/src/crt0.o
 .debug_aranges
                0x00000028       0x20 obj/HDMI_Lib/HDMI_RX/HDMI_RX.o
 .debug_aranges
                0x00000048       0x20 obj/HDMI_Lib/HDMI_RX/it6605.o
 .debug_aranges
                0x00000068       0x20 obj/HDMI_Lib/HDMI_TX/EDID.o
 .debug_aranges
                0x00000088       0x20 obj/HDMI_Lib/HDMI_TX/HDMI_TX.o
 .debug_aranges
                0x000000a8       0x20 obj/HDMI_Lib/HDMI_TX/it6613_drv.o
 .debug_aranges
                0x000000c8       0x20 obj/HDMI_Lib/HDMI_TX/it6613_sys.o
 .debug_aranges
                0x000000e8       0x20 obj/HDMI_Lib/mcu.o
 .debug_aranges
                0x00000108       0x20 obj/main.o
 .debug_aranges
                0x00000128       0x20 obj/terasic_lib/I2C.o
 .debug_aranges
                0x00000148       0x20 obj/terasic_lib/debug.o
 .debug_aranges
                0x00000168       0x20 c:/altera/11.1/nios2eds/bin/gnu/h-i686-mingw32/bin/../lib/gcc/nios2-elf/4.1.2/mhw-mulx\libgcc.a(_mul_df.o)
 .debug_aranges
                0x00000188       0x20 c:/altera/11.1/nios2eds/bin/gnu/h-i686-mingw32/bin/../lib/gcc/nios2-elf/4.1.2/mhw-mulx\libgcc.a(_div_df.o)
 .debug_aranges
                0x000001a8       0x20 c:/altera/11.1/nios2eds/bin/gnu/h-i686-mingw32/bin/../lib/gcc/nios2-elf/4.1.2/mhw-mulx\libgcc.a(_si_to_df.o)
 .debug_aranges
                0x000001c8       0x20 c:/altera/11.1/nios2eds/bin/gnu/h-i686-mingw32/bin/../lib/gcc/nios2-elf/4.1.2/mhw-mulx\libgcc.a(lib2-divmod.o)
 .debug_aranges
                0x000001e8       0x20 c:/altera/11.1/nios2eds/bin/gnu/h-i686-mingw32/bin/../lib/gcc/nios2-elf/4.1.2/mhw-mulx\libgcc.a(_clzsi2.o)
 .debug_aranges
                0x00000208       0x20 c:/altera/11.1/nios2eds/bin/gnu/h-i686-mingw32/bin/../lib/gcc/nios2-elf/4.1.2/mhw-mulx\libgcc.a(_pack_df.o)
 .debug_aranges
                0x00000228       0x20 c:/altera/11.1/nios2eds/bin/gnu/h-i686-mingw32/bin/../lib/gcc/nios2-elf/4.1.2/mhw-mulx\libgcc.a(_unpack_df.o)
 .debug_aranges
                0x00000248       0x20 c:/altera/11.1/nios2eds/bin/gnu/h-i686-mingw32/bin/../lib/gcc/nios2-elf/4.1.2/../../../../nios2-elf/lib/mhw-mulx\libsmallc.a(lib_a-memset.o)
 .debug_aranges
                0x00000268       0x20 c:/altera/11.1/nios2eds/bin/gnu/h-i686-mingw32/bin/../lib/gcc/nios2-elf/4.1.2/../../../../nios2-elf/lib/mhw-mulx\libsmallc.a(lib_a-printf.o)
 .debug_aranges
                0x00000288       0x20 c:/altera/11.1/nios2eds/bin/gnu/h-i686-mingw32/bin/../lib/gcc/nios2-elf/4.1.2/../../../../nios2-elf/lib/mhw-mulx\libsmallc.a(lib_a-putchar.o)
 .debug_aranges
                0x000002a8       0x20 c:/altera/11.1/nios2eds/bin/gnu/h-i686-mingw32/bin/../lib/gcc/nios2-elf/4.1.2/../../../../nios2-elf/lib/mhw-mulx\libsmallc.a(lib_a-puts.o)
 .debug_aranges
                0x000002c8       0x20 c:/altera/11.1/nios2eds/bin/gnu/h-i686-mingw32/bin/../lib/gcc/nios2-elf/4.1.2/../../../../nios2-elf/lib/mhw-mulx\libsmallc.a(lib_a-sprintf.o)
 .debug_aranges
                0x000002e8       0x20 c:/altera/11.1/nios2eds/bin/gnu/h-i686-mingw32/bin/../lib/gcc/nios2-elf/4.1.2/../../../../nios2-elf/lib/mhw-mulx\libsmallc.a(lib_a-strlen.o)
 .debug_aranges
                0x00000308       0x20 c:/altera/11.1/nios2eds/bin/gnu/h-i686-mingw32/bin/../lib/gcc/nios2-elf/4.1.2/../../../../nios2-elf/lib/mhw-mulx\libsmallc.a(lib_a-vfprintf.o)
 .debug_aranges
                0x00000328       0x20 c:/altera/11.1/nios2eds/bin/gnu/h-i686-mingw32/bin/../lib/gcc/nios2-elf/4.1.2/../../../../nios2-elf/lib/mhw-mulx\libsmallc.a(lib_a-vfprintf_1.o)
 .debug_aranges
                0x00000348       0x20 c:/altera/11.1/nios2eds/bin/gnu/h-i686-mingw32/bin/../lib/gcc/nios2-elf/4.1.2/../../../../nios2-elf/lib/mhw-mulx\libsmallc.a(lib_a-vsnprintf.o)
 .debug_aranges
                0x00000368       0x20 c:/altera/11.1/nios2eds/bin/gnu/h-i686-mingw32/bin/../lib/gcc/nios2-elf/4.1.2/../../../../nios2-elf/lib/mhw-mulx\libsmallc.a(lib_a-fvwrite_small_dev.o)
 .debug_aranges
                0x00000388       0x20 c:/altera/11.1/nios2eds/bin/gnu/h-i686-mingw32/bin/../lib/gcc/nios2-elf/4.1.2/../../../../nios2-elf/lib/mhw-mulx\libsmallc.a(lib_a-fvwrite_small_str.o)
 .debug_aranges
                0x000003a8       0x20 c:/altera/11.1/nios2eds/bin/gnu/h-i686-mingw32/bin/../lib/gcc/nios2-elf/4.1.2/../../../../nios2-elf/lib/mhw-mulx\libsmallc.a(lib_a-memmove.o)
 .debug_aranges
                0x000003c8       0x20 c:/altera/11.1/nios2eds/bin/gnu/h-i686-mingw32/bin/../lib/gcc/nios2-elf/4.1.2/../../../../nios2-elf/lib/mhw-mulx\libsmallc.a(lib_a-putc.o)
 .debug_aranges
                0x000003e8       0x20 c:/altera/11.1/nios2eds/bin/gnu/h-i686-mingw32/bin/../lib/gcc/nios2-elf/4.1.2/../../../../nios2-elf/lib/mhw-mulx\libsmallc.a(lib_a-writer.o)
 .debug_aranges
                0x00000408       0x20 ../TR4_HDMI_TX_RX_bsp/\libhal_bsp.a(alt_irq_register.o)
 .debug_aranges
                0x00000428       0x20 ../TR4_HDMI_TX_RX_bsp/\libhal_bsp.a(alt_load.o)
 .debug_aranges
                0x00000448       0x20 ../TR4_HDMI_TX_RX_bsp/\libhal_bsp.a(alt_main.o)
 .debug_aranges
                0x00000468       0x20 ../TR4_HDMI_TX_RX_bsp/\libhal_bsp.a(alt_tick.o)
 .debug_aranges
                0x00000488       0x20 ../TR4_HDMI_TX_RX_bsp/\libhal_bsp.a(alt_usleep.o)
 .debug_aranges
                0x000004a8       0x20 ../TR4_HDMI_TX_RX_bsp/\libhal_bsp.a(alt_write.o)
 .debug_aranges
                0x000004c8       0x20 ../TR4_HDMI_TX_RX_bsp/\libhal_bsp.a(alt_sys_init.o)
 .debug_aranges
                0x000004e8       0x20 ../TR4_HDMI_TX_RX_bsp/\libhal_bsp.a(altera_avalon_jtag_uart_fd.o)
 .debug_aranges
                0x00000508       0x20 ../TR4_HDMI_TX_RX_bsp/\libhal_bsp.a(altera_avalon_jtag_uart_read.o)
 .debug_aranges
                0x00000528       0x20 ../TR4_HDMI_TX_RX_bsp/\libhal_bsp.a(altera_avalon_jtag_uart_write.o)
 .debug_aranges
                0x00000548       0x20 ../TR4_HDMI_TX_RX_bsp/\libhal_bsp.a(altera_avalon_timer_sc.o)
 .debug_aranges
                0x00000568       0x20 ../TR4_HDMI_TX_RX_bsp/\libhal_bsp.a(alt_busy_sleep.o)
 .debug_aranges
                0x00000588       0x20 ../TR4_HDMI_TX_RX_bsp/\libhal_bsp.a(alt_close.o)
 .debug_aranges
                0x000005a8       0x20 ../TR4_HDMI_TX_RX_bsp/\libhal_bsp.a(alt_dcache_flush_all.o)
 .debug_aranges
                0x000005c8       0x20 ../TR4_HDMI_TX_RX_bsp/\libhal_bsp.a(alt_dev.o)
 .debug_aranges
                0x000005e8       0x20 ../TR4_HDMI_TX_RX_bsp/\libhal_bsp.a(alt_dev_llist_insert.o)
 .debug_aranges
                0x00000608       0x20 ../TR4_HDMI_TX_RX_bsp/\libhal_bsp.a(alt_do_ctors.o)
 .debug_aranges
                0x00000628       0x20 ../TR4_HDMI_TX_RX_bsp/\libhal_bsp.a(alt_do_dtors.o)
 .debug_aranges
                0x00000648       0x20 ../TR4_HDMI_TX_RX_bsp/\libhal_bsp.a(alt_icache_flush_all.o)
 .debug_aranges
                0x00000668       0x20 ../TR4_HDMI_TX_RX_bsp/\libhal_bsp.a(alt_iic.o)
 .debug_aranges
                0x00000688       0x20 ../TR4_HDMI_TX_RX_bsp/\libhal_bsp.a(alt_iic_isr_register.o)
 .debug_aranges
                0x000006a8       0x20 ../TR4_HDMI_TX_RX_bsp/\libhal_bsp.a(alt_io_redirect.o)
 .debug_aranges
                0x000006c8       0x30 ../TR4_HDMI_TX_RX_bsp/\libhal_bsp.a(alt_irq_entry.o)
 .debug_aranges
                0x000006f8       0x28 ../TR4_HDMI_TX_RX_bsp/\libhal_bsp.a(alt_irq_handler.o)
 .debug_aranges
                0x00000720       0x20 ../TR4_HDMI_TX_RX_bsp/\libhal_bsp.a(alt_open.o)
 .debug_aranges
                0x00000740       0x20 ../TR4_HDMI_TX_RX_bsp/\libhal_bsp.a(alt_release_fd.o)
 .debug_aranges
                0x00000760       0x20 ../TR4_HDMI_TX_RX_bsp/\libhal_bsp.a(altera_nios2_qsys_irq.o)
 .debug_aranges
                0x00000780       0x38 ../TR4_HDMI_TX_RX_bsp/\libhal_bsp.a(alt_exception_entry.o)
 .debug_aranges
                0x000007b8       0x20 ../TR4_HDMI_TX_RX_bsp/\libhal_bsp.a(alt_find_dev.o)
 .debug_aranges
                0x000007d8       0x20 ../TR4_HDMI_TX_RX_bsp/\libhal_bsp.a(alt_find_file.o)
 .debug_aranges
                0x000007f8       0x20 ../TR4_HDMI_TX_RX_bsp/\libhal_bsp.a(alt_get_fd.o)
 .debug_aranges
                0x00000818       0x20 ../TR4_HDMI_TX_RX_bsp/\libhal_bsp.a(alt_icache_flush.o)
 .debug_aranges
                0x00000838       0x20 c:/altera/11.1/nios2eds/bin/gnu/h-i686-mingw32/bin/../lib/gcc/nios2-elf/4.1.2/../../../../nios2-elf/lib/mhw-mulx\libsmallc.a(lib_a-atexit.o)
 .debug_aranges
                0x00000858       0x20 c:/altera/11.1/nios2eds/bin/gnu/h-i686-mingw32/bin/../lib/gcc/nios2-elf/4.1.2/../../../../nios2-elf/lib/mhw-mulx\libsmallc.a(lib_a-exit.o)
 .debug_aranges
                0x00000878       0x20 c:/altera/11.1/nios2eds/bin/gnu/h-i686-mingw32/bin/../lib/gcc/nios2-elf/4.1.2/../../../../nios2-elf/lib/mhw-mulx\libsmallc.a(lib_a-memcmp.o)
 .debug_aranges
                0x00000898       0x20 c:/altera/11.1/nios2eds/bin/gnu/h-i686-mingw32/bin/../lib/gcc/nios2-elf/4.1.2/../../../../nios2-elf/lib/mhw-mulx\libsmallc.a(lib_a-__atexit.o)
 .debug_aranges
                0x000008b8       0x20 c:/altera/11.1/nios2eds/bin/gnu/h-i686-mingw32/bin/../lib/gcc/nios2-elf/4.1.2/../../../../nios2-elf/lib/mhw-mulx\libsmallc.a(lib_a-__call_atexit.o)
 .debug_aranges
                0x000008d8       0x20 ../TR4_HDMI_TX_RX_bsp/\libhal_bsp.a(alt_exit.o)

.debug_pubnames
                0x00000000     0x1dd5
 *(.debug_pubnames)
 .debug_pubnames
                0x00000000       0x2b obj/Beep.o
 .debug_pubnames
                0x0000002b      0x14c obj/HDMI_Lib/HDMI_RX/HDMI_RX.o
 .debug_pubnames
                0x00000177      0x765 obj/HDMI_Lib/HDMI_RX/it6605.o
 .debug_pubnames
                0x000008dc       0x35 obj/HDMI_Lib/HDMI_TX/EDID.o
 .debug_pubnames
                0x00000911      0x1d6 obj/HDMI_Lib/HDMI_TX/HDMI_TX.o
 .debug_pubnames
                0x00000ae7      0x234 obj/HDMI_Lib/HDMI_TX/it6613_drv.o
 .debug_pubnames
                0x00000d1b      0x188 obj/HDMI_Lib/HDMI_TX/it6613_sys.o
 .debug_pubnames
                0x00000ea3      0x29e obj/HDMI_Lib/mcu.o
 .debug_pubnames
                0x00001141       0xfe obj/main.o
 .debug_pubnames
                0x0000123f       0x93 obj/terasic_lib/I2C.o
 .debug_pubnames
                0x000012d2       0x5e obj/terasic_lib/debug.o
 .debug_pubnames
                0x00001330       0x1f c:/altera/11.1/nios2eds/bin/gnu/h-i686-mingw32/bin/../lib/gcc/nios2-elf/4.1.2/mhw-mulx\libgcc.a(_mul_df.o)
 .debug_pubnames
                0x0000134f       0x1f c:/altera/11.1/nios2eds/bin/gnu/h-i686-mingw32/bin/../lib/gcc/nios2-elf/4.1.2/mhw-mulx\libgcc.a(_div_df.o)
 .debug_pubnames
                0x0000136e       0x22 c:/altera/11.1/nios2eds/bin/gnu/h-i686-mingw32/bin/../lib/gcc/nios2-elf/4.1.2/mhw-mulx\libgcc.a(_si_to_df.o)
 .debug_pubnames
                0x00001390       0x22 c:/altera/11.1/nios2eds/bin/gnu/h-i686-mingw32/bin/../lib/gcc/nios2-elf/4.1.2/mhw-mulx\libgcc.a(_thenan_df.o)
 .debug_pubnames
                0x000013b2       0x48 c:/altera/11.1/nios2eds/bin/gnu/h-i686-mingw32/bin/../lib/gcc/nios2-elf/4.1.2/mhw-mulx\libgcc.a(lib2-divmod.o)
 .debug_pubnames
                0x000013fa       0x1f c:/altera/11.1/nios2eds/bin/gnu/h-i686-mingw32/bin/../lib/gcc/nios2-elf/4.1.2/mhw-mulx\libgcc.a(_clzsi2.o)
 .debug_pubnames
                0x00001419       0x1f c:/altera/11.1/nios2eds/bin/gnu/h-i686-mingw32/bin/../lib/gcc/nios2-elf/4.1.2/mhw-mulx\libgcc.a(_pack_df.o)
 .debug_pubnames
                0x00001438       0x21 c:/altera/11.1/nios2eds/bin/gnu/h-i686-mingw32/bin/../lib/gcc/nios2-elf/4.1.2/mhw-mulx\libgcc.a(_unpack_df.o)
 .debug_pubnames
                0x00001459       0x20 c:/altera/11.1/nios2eds/bin/gnu/h-i686-mingw32/bin/../lib/gcc/nios2-elf/4.1.2/mhw-mulx\libgcc.a(_clz.o)
 .debug_pubnames
                0x00001479       0x39 c:/altera/11.1/nios2eds/bin/gnu/h-i686-mingw32/bin/../lib/gcc/nios2-elf/4.1.2/../../../../nios2-elf/lib/mhw-mulx\libsmallc.a(lib_a-impure.o)
 .debug_pubnames
                0x000014b2       0x1d c:/altera/11.1/nios2eds/bin/gnu/h-i686-mingw32/bin/../lib/gcc/nios2-elf/4.1.2/../../../../nios2-elf/lib/mhw-mulx\libsmallc.a(lib_a-memset.o)
 .debug_pubnames
                0x000014cf       0x2b c:/altera/11.1/nios2eds/bin/gnu/h-i686-mingw32/bin/../lib/gcc/nios2-elf/4.1.2/../../../../nios2-elf/lib/mhw-mulx\libsmallc.a(lib_a-printf.o)
 .debug_pubnames
                0x000014fa       0x2d c:/altera/11.1/nios2eds/bin/gnu/h-i686-mingw32/bin/../lib/gcc/nios2-elf/4.1.2/../../../../nios2-elf/lib/mhw-mulx\libsmallc.a(lib_a-putchar.o)
 .debug_pubnames
                0x00001527       0x27 c:/altera/11.1/nios2eds/bin/gnu/h-i686-mingw32/bin/../lib/gcc/nios2-elf/4.1.2/../../../../nios2-elf/lib/mhw-mulx\libsmallc.a(lib_a-puts.o)
 .debug_pubnames
                0x0000154e       0x2d c:/altera/11.1/nios2eds/bin/gnu/h-i686-mingw32/bin/../lib/gcc/nios2-elf/4.1.2/../../../../nios2-elf/lib/mhw-mulx\libsmallc.a(lib_a-sprintf.o)
 .debug_pubnames
                0x0000157b       0x1d c:/altera/11.1/nios2eds/bin/gnu/h-i686-mingw32/bin/../lib/gcc/nios2-elf/4.1.2/../../../../nios2-elf/lib/mhw-mulx\libsmallc.a(lib_a-strlen.o)
 .debug_pubnames
                0x00001598       0x45 c:/altera/11.1/nios2eds/bin/gnu/h-i686-mingw32/bin/../lib/gcc/nios2-elf/4.1.2/../../../../nios2-elf/lib/mhw-mulx\libsmallc.a(lib_a-vfprintf.o)
 .debug_pubnames
                0x000015dd       0x1f c:/altera/11.1/nios2eds/bin/gnu/h-i686-mingw32/bin/../lib/gcc/nios2-elf/4.1.2/../../../../nios2-elf/lib/mhw-mulx\libsmallc.a(lib_a-vfprintf_1.o)
 .debug_pubnames
                0x000015fc       0x31 c:/altera/11.1/nios2eds/bin/gnu/h-i686-mingw32/bin/../lib/gcc/nios2-elf/4.1.2/../../../../nios2-elf/lib/mhw-mulx\libsmallc.a(lib_a-vsnprintf.o)
 .debug_pubnames
                0x0000162d       0x2b c:/altera/11.1/nios2eds/bin/gnu/h-i686-mingw32/bin/../lib/gcc/nios2-elf/4.1.2/../../../../nios2-elf/lib/mhw-mulx\libsmallc.a(lib_a-fvwrite_small_dev.o)
 .debug_pubnames
                0x00001658       0x2b c:/altera/11.1/nios2eds/bin/gnu/h-i686-mingw32/bin/../lib/gcc/nios2-elf/4.1.2/../../../../nios2-elf/lib/mhw-mulx\libsmallc.a(lib_a-fvwrite_small_str.o)
 .debug_pubnames
                0x00001683       0x1e c:/altera/11.1/nios2eds/bin/gnu/h-i686-mingw32/bin/../lib/gcc/nios2-elf/4.1.2/../../../../nios2-elf/lib/mhw-mulx\libsmallc.a(lib_a-memmove.o)
 .debug_pubnames
                0x000016a1       0x27 c:/altera/11.1/nios2eds/bin/gnu/h-i686-mingw32/bin/../lib/gcc/nios2-elf/4.1.2/../../../../nios2-elf/lib/mhw-mulx\libsmallc.a(lib_a-putc.o)
 .debug_pubnames
                0x000016c8       0x1f c:/altera/11.1/nios2eds/bin/gnu/h-i686-mingw32/bin/../lib/gcc/nios2-elf/4.1.2/../../../../nios2-elf/lib/mhw-mulx\libsmallc.a(lib_a-writer.o)
 .debug_pubnames
                0x000016e7       0x1c c:/altera/11.1/nios2eds/bin/gnu/h-i686-mingw32/bin/../lib/gcc/nios2-elf/4.1.2/../../../../nios2-elf/lib/mhw-mulx\libsmallc.a(lib_a-int_errno.o)
 .debug_pubnames
                0x00001703       0x27 ../TR4_HDMI_TX_RX_bsp/\libhal_bsp.a(alt_irq_register.o)
 .debug_pubnames
                0x0000172a       0x3b ../TR4_HDMI_TX_RX_bsp/\libhal_bsp.a(alt_irq_vars.o)
 .debug_pubnames
                0x00001765       0x1f ../TR4_HDMI_TX_RX_bsp/\libhal_bsp.a(alt_load.o)
 .debug_pubnames
                0x00001784       0x46 ../TR4_HDMI_TX_RX_bsp/\libhal_bsp.a(alt_main.o)
 .debug_pubnames
                0x000017ca       0x68 ../TR4_HDMI_TX_RX_bsp/\libhal_bsp.a(alt_tick.o)
 .debug_pubnames
                0x00001832       0x1d ../TR4_HDMI_TX_RX_bsp/\libhal_bsp.a(alt_usleep.o)
 .debug_pubnames
                0x0000184f       0x1c ../TR4_HDMI_TX_RX_bsp/\libhal_bsp.a(alt_write.o)
 .debug_pubnames
                0x0000186b       0x34 ../TR4_HDMI_TX_RX_bsp/\libhal_bsp.a(alt_sys_init.o)
 .debug_pubnames
                0x0000189f       0x5b ../TR4_HDMI_TX_RX_bsp/\libhal_bsp.a(altera_avalon_jtag_uart_fd.o)
 .debug_pubnames
                0x000018fa       0x33 ../TR4_HDMI_TX_RX_bsp/\libhal_bsp.a(altera_avalon_jtag_uart_read.o)
 .debug_pubnames
                0x0000192d       0x34 ../TR4_HDMI_TX_RX_bsp/\libhal_bsp.a(altera_avalon_jtag_uart_write.o)
 .debug_pubnames
                0x00001961       0x2f ../TR4_HDMI_TX_RX_bsp/\libhal_bsp.a(altera_avalon_timer_sc.o)
 .debug_pubnames
                0x00001990       0x25 ../TR4_HDMI_TX_RX_bsp/\libhal_bsp.a(alt_busy_sleep.o)
 .debug_pubnames
                0x000019b5       0x1c ../TR4_HDMI_TX_RX_bsp/\libhal_bsp.a(alt_close.o)
 .debug_pubnames
                0x000019d1       0x2b ../TR4_HDMI_TX_RX_bsp/\libhal_bsp.a(alt_dcache_flush_all.o)
 .debug_pubnames
                0x000019fc       0x63 ../TR4_HDMI_TX_RX_bsp/\libhal_bsp.a(alt_dev.o)
 .debug_pubnames
                0x00001a5f       0x2b ../TR4_HDMI_TX_RX_bsp/\libhal_bsp.a(alt_dev_llist_insert.o)
 .debug_pubnames
                0x00001a8a       0x20 ../TR4_HDMI_TX_RX_bsp/\libhal_bsp.a(alt_do_ctors.o)
 .debug_pubnames
                0x00001aaa       0x20 ../TR4_HDMI_TX_RX_bsp/\libhal_bsp.a(alt_do_dtors.o)
 .debug_pubnames
                0x00001aca       0x20 ../TR4_HDMI_TX_RX_bsp/\libhal_bsp.a(alt_errno.o)
 .debug_pubnames
                0x00001aea       0x2b ../TR4_HDMI_TX_RX_bsp/\libhal_bsp.a(alt_icache_flush_all.o)
 .debug_pubnames
                0x00001b15       0x6e ../TR4_HDMI_TX_RX_bsp/\libhal_bsp.a(alt_iic.o)
 .debug_pubnames
                0x00001b83       0x2b ../TR4_HDMI_TX_RX_bsp/\libhal_bsp.a(alt_iic_isr_register.o)
 .debug_pubnames
                0x00001bae       0x26 ../TR4_HDMI_TX_RX_bsp/\libhal_bsp.a(alt_io_redirect.o)
 .debug_pubnames
                0x00001bd4       0x32 ../TR4_HDMI_TX_RX_bsp/\libhal_bsp.a(alt_irq_handler.o)
 .debug_pubnames
                0x00001c06       0x1b ../TR4_HDMI_TX_RX_bsp/\libhal_bsp.a(alt_open.o)
 .debug_pubnames
                0x00001c21       0x25 ../TR4_HDMI_TX_RX_bsp/\libhal_bsp.a(alt_release_fd.o)
 .debug_pubnames
                0x00001c46       0x31 ../TR4_HDMI_TX_RX_bsp/\libhal_bsp.a(altera_nios2_qsys_irq.o)
 .debug_pubnames
                0x00001c77       0x23 ../TR4_HDMI_TX_RX_bsp/\libhal_bsp.a(alt_find_dev.o)
 .debug_pubnames
                0x00001c9a       0x24 ../TR4_HDMI_TX_RX_bsp/\libhal_bsp.a(alt_find_file.o)
 .debug_pubnames
                0x00001cbe       0x21 ../TR4_HDMI_TX_RX_bsp/\libhal_bsp.a(alt_get_fd.o)
 .debug_pubnames
                0x00001cdf       0x27 ../TR4_HDMI_TX_RX_bsp/\libhal_bsp.a(alt_icache_flush.o)
 .debug_pubnames
                0x00001d06       0x2a c:/altera/11.1/nios2eds/bin/gnu/h-i686-mingw32/bin/../lib/gcc/nios2-elf/4.1.2/../../../../nios2-elf/lib/mhw-mulx\libsmallc.a(lib_a-atexit.o)
 .debug_pubnames
                0x00001d30       0x1b c:/altera/11.1/nios2eds/bin/gnu/h-i686-mingw32/bin/../lib/gcc/nios2-elf/4.1.2/../../../../nios2-elf/lib/mhw-mulx\libsmallc.a(lib_a-exit.o)
 .debug_pubnames
                0x00001d4b       0x1d c:/altera/11.1/nios2eds/bin/gnu/h-i686-mingw32/bin/../lib/gcc/nios2-elf/4.1.2/../../../../nios2-elf/lib/mhw-mulx\libsmallc.a(lib_a-memcmp.o)
 .debug_pubnames
                0x00001d68       0x2a c:/altera/11.1/nios2eds/bin/gnu/h-i686-mingw32/bin/../lib/gcc/nios2-elf/4.1.2/../../../../nios2-elf/lib/mhw-mulx\libsmallc.a(lib_a-__atexit.o)
 .debug_pubnames
                0x00001d92       0x27 c:/altera/11.1/nios2eds/bin/gnu/h-i686-mingw32/bin/../lib/gcc/nios2-elf/4.1.2/../../../../nios2-elf/lib/mhw-mulx\libsmallc.a(lib_a-__call_atexit.o)
 .debug_pubnames
                0x00001db9       0x1c ../TR4_HDMI_TX_RX_bsp/\libhal_bsp.a(alt_exit.o)

.debug_info     0x00000000    0x1a278
 *(.debug_info .gnu.linkonce.wi.*)
 .debug_info    0x00000000       0x7b ../TR4_HDMI_TX_RX_bsp//obj/HAL/src/crt0.o
 .debug_info    0x0000007b       0xe1 obj/Beep.o
 .debug_info    0x0000015c      0xb43 obj/HDMI_Lib/HDMI_RX/HDMI_RX.o
 .debug_info    0x00000c9f     0x25fa obj/HDMI_Lib/HDMI_RX/it6605.o
 .debug_info    0x00003299      0x905 obj/HDMI_Lib/HDMI_TX/EDID.o
 .debug_info    0x00003b9e     0x112b obj/HDMI_Lib/HDMI_TX/HDMI_TX.o
 .debug_info    0x00004cc9      0x1ef obj/HDMI_Lib/HDMI_TX/dss_sha.o
 .debug_info    0x00004eb8     0x2ccf obj/HDMI_Lib/HDMI_TX/it6613_drv.o
 .debug_info    0x00007b87     0x1201 obj/HDMI_Lib/HDMI_TX/it6613_sys.o
 .debug_info    0x00008d88     0x1744 obj/HDMI_Lib/mcu.o
 .debug_info    0x0000a4cc      0xa2b obj/main.o
 .debug_info    0x0000aef7      0x59e obj/terasic_lib/I2C.o
 .debug_info    0x0000b495      0x3c2 obj/terasic_lib/debug.o
 .debug_info    0x0000b857      0x488 c:/altera/11.1/nios2eds/bin/gnu/h-i686-mingw32/bin/../lib/gcc/nios2-elf/4.1.2/mhw-mulx\libgcc.a(_mul_df.o)
 .debug_info    0x0000bcdf      0x39b c:/altera/11.1/nios2eds/bin/gnu/h-i686-mingw32/bin/../lib/gcc/nios2-elf/4.1.2/mhw-mulx\libgcc.a(_div_df.o)
 .debug_info    0x0000c07a      0x218 c:/altera/11.1/nios2eds/bin/gnu/h-i686-mingw32/bin/../lib/gcc/nios2-elf/4.1.2/mhw-mulx\libgcc.a(_si_to_df.o)
 .debug_info    0x0000c292      0x164 c:/altera/11.1/nios2eds/bin/gnu/h-i686-mingw32/bin/../lib/gcc/nios2-elf/4.1.2/mhw-mulx\libgcc.a(_thenan_df.o)
 .debug_info    0x0000c3f6      0x21c c:/altera/11.1/nios2eds/bin/gnu/h-i686-mingw32/bin/../lib/gcc/nios2-elf/4.1.2/mhw-mulx\libgcc.a(lib2-divmod.o)
 .debug_info    0x0000c612      0x130 c:/altera/11.1/nios2eds/bin/gnu/h-i686-mingw32/bin/../lib/gcc/nios2-elf/4.1.2/mhw-mulx\libgcc.a(_clzsi2.o)
 .debug_info    0x0000c742      0x2fc c:/altera/11.1/nios2eds/bin/gnu/h-i686-mingw32/bin/../lib/gcc/nios2-elf/4.1.2/mhw-mulx\libgcc.a(_pack_df.o)
 .debug_info    0x0000ca3e      0x268 c:/altera/11.1/nios2eds/bin/gnu/h-i686-mingw32/bin/../lib/gcc/nios2-elf/4.1.2/mhw-mulx\libgcc.a(_unpack_df.o)
 .debug_info    0x0000cca6       0xc9 c:/altera/11.1/nios2eds/bin/gnu/h-i686-mingw32/bin/../lib/gcc/nios2-elf/4.1.2/mhw-mulx\libgcc.a(_clz.o)
 .debug_info    0x0000cd6f      0x636 c:/altera/11.1/nios2eds/bin/gnu/h-i686-mingw32/bin/../lib/gcc/nios2-elf/4.1.2/../../../../nios2-elf/lib/mhw-mulx\libsmallc.a(lib_a-impure.o)
 .debug_info    0x0000d3a5       0xd7 c:/altera/11.1/nios2eds/bin/gnu/h-i686-mingw32/bin/../lib/gcc/nios2-elf/4.1.2/../../../../nios2-elf/lib/mhw-mulx\libsmallc.a(lib_a-memset.o)
 .debug_info    0x0000d47c      0x6c8 c:/altera/11.1/nios2eds/bin/gnu/h-i686-mingw32/bin/../lib/gcc/nios2-elf/4.1.2/../../../../nios2-elf/lib/mhw-mulx\libsmallc.a(lib_a-printf.o)
 .debug_info    0x0000db44      0x66b c:/altera/11.1/nios2eds/bin/gnu/h-i686-mingw32/bin/../lib/gcc/nios2-elf/4.1.2/../../../../nios2-elf/lib/mhw-mulx\libsmallc.a(lib_a-putchar.o)
 .debug_info    0x0000e1af      0x685 c:/altera/11.1/nios2eds/bin/gnu/h-i686-mingw32/bin/../lib/gcc/nios2-elf/4.1.2/../../../../nios2-elf/lib/mhw-mulx\libsmallc.a(lib_a-puts.o)
 .debug_info    0x0000e834      0x7e7 c:/altera/11.1/nios2eds/bin/gnu/h-i686-mingw32/bin/../lib/gcc/nios2-elf/4.1.2/../../../../nios2-elf/lib/mhw-mulx\libsmallc.a(lib_a-sprintf.o)
 .debug_info    0x0000f01b       0xc2 c:/altera/11.1/nios2eds/bin/gnu/h-i686-mingw32/bin/../lib/gcc/nios2-elf/4.1.2/../../../../nios2-elf/lib/mhw-mulx\libsmallc.a(lib_a-strlen.o)
 .debug_info    0x0000f0dd      0x94c c:/altera/11.1/nios2eds/bin/gnu/h-i686-mingw32/bin/../lib/gcc/nios2-elf/4.1.2/../../../../nios2-elf/lib/mhw-mulx\libsmallc.a(lib_a-vfprintf.o)
 .debug_info    0x0000fa29      0x677 c:/altera/11.1/nios2eds/bin/gnu/h-i686-mingw32/bin/../lib/gcc/nios2-elf/4.1.2/../../../../nios2-elf/lib/mhw-mulx\libsmallc.a(lib_a-vfprintf_1.o)
 .debug_info    0x000100a0      0x7ef c:/altera/11.1/nios2eds/bin/gnu/h-i686-mingw32/bin/../lib/gcc/nios2-elf/4.1.2/../../../../nios2-elf/lib/mhw-mulx\libsmallc.a(lib_a-vsnprintf.o)
 .debug_info    0x0001088f      0x68e c:/altera/11.1/nios2eds/bin/gnu/h-i686-mingw32/bin/../lib/gcc/nios2-elf/4.1.2/../../../../nios2-elf/lib/mhw-mulx\libsmallc.a(lib_a-fvwrite_small_dev.o)
 .debug_info    0x00010f1d      0x75f c:/altera/11.1/nios2eds/bin/gnu/h-i686-mingw32/bin/../lib/gcc/nios2-elf/4.1.2/../../../../nios2-elf/lib/mhw-mulx\libsmallc.a(lib_a-fvwrite_small_str.o)
 .debug_info    0x0001167c      0x102 c:/altera/11.1/nios2eds/bin/gnu/h-i686-mingw32/bin/../lib/gcc/nios2-elf/4.1.2/../../../../nios2-elf/lib/mhw-mulx\libsmallc.a(lib_a-memmove.o)
 .debug_info    0x0001177e      0x6b8 c:/altera/11.1/nios2eds/bin/gnu/h-i686-mingw32/bin/../lib/gcc/nios2-elf/4.1.2/../../../../nios2-elf/lib/mhw-mulx\libsmallc.a(lib_a-putc.o)
 .debug_info    0x00011e36      0x68c c:/altera/11.1/nios2eds/bin/gnu/h-i686-mingw32/bin/../lib/gcc/nios2-elf/4.1.2/../../../../nios2-elf/lib/mhw-mulx\libsmallc.a(lib_a-writer.o)
 .debug_info    0x000124c2       0x8c c:/altera/11.1/nios2eds/bin/gnu/h-i686-mingw32/bin/../lib/gcc/nios2-elf/4.1.2/../../../../nios2-elf/lib/mhw-mulx\libsmallc.a(lib_a-int_errno.o)
 .debug_info    0x0001254e      0x42a ../TR4_HDMI_TX_RX_bsp/\libhal_bsp.a(alt_irq_register.o)
 .debug_info    0x00012978      0x167 ../TR4_HDMI_TX_RX_bsp/\libhal_bsp.a(alt_irq_vars.o)
 .debug_info    0x00012adf      0x28d ../TR4_HDMI_TX_RX_bsp/\libhal_bsp.a(alt_load.o)
 .debug_info    0x00012d6c      0x225 ../TR4_HDMI_TX_RX_bsp/\libhal_bsp.a(alt_main.o)
 .debug_info    0x00012f91      0x3fe ../TR4_HDMI_TX_RX_bsp/\libhal_bsp.a(alt_tick.o)
 .debug_info    0x0001338f      0x168 ../TR4_HDMI_TX_RX_bsp/\libhal_bsp.a(alt_usleep.o)
 .debug_info    0x000134f7      0x693 ../TR4_HDMI_TX_RX_bsp/\libhal_bsp.a(alt_write.o)
 .debug_info    0x00013b8a      0x5c1 ../TR4_HDMI_TX_RX_bsp/\libhal_bsp.a(alt_sys_init.o)
 .debug_info    0x0001414b      0x5b9 ../TR4_HDMI_TX_RX_bsp/\libhal_bsp.a(altera_avalon_jtag_uart_fd.o)
 .debug_info    0x00014704      0x309 ../TR4_HDMI_TX_RX_bsp/\libhal_bsp.a(altera_avalon_jtag_uart_read.o)
 .debug_info    0x00014a0d      0x2e6 ../TR4_HDMI_TX_RX_bsp/\libhal_bsp.a(altera_avalon_jtag_uart_write.o)
 .debug_info    0x00014cf3      0x38b ../TR4_HDMI_TX_RX_bsp/\libhal_bsp.a(altera_avalon_timer_sc.o)
 .debug_info    0x0001507e      0x1ab ../TR4_HDMI_TX_RX_bsp/\libhal_bsp.a(alt_busy_sleep.o)
 .debug_info    0x00015229      0x467 ../TR4_HDMI_TX_RX_bsp/\libhal_bsp.a(alt_close.o)
 .debug_info    0x00015690      0x15c ../TR4_HDMI_TX_RX_bsp/\libhal_bsp.a(alt_dcache_flush_all.o)
 .debug_info    0x000157ec      0x67f ../TR4_HDMI_TX_RX_bsp/\libhal_bsp.a(alt_dev.o)
 .debug_info    0x00015e6b      0x2b7 ../TR4_HDMI_TX_RX_bsp/\libhal_bsp.a(alt_dev_llist_insert.o)
 .debug_info    0x00016122      0x10f ../TR4_HDMI_TX_RX_bsp/\libhal_bsp.a(alt_do_ctors.o)
 .debug_info    0x00016231      0x10e ../TR4_HDMI_TX_RX_bsp/\libhal_bsp.a(alt_do_dtors.o)
 .debug_info    0x0001633f      0x164 ../TR4_HDMI_TX_RX_bsp/\libhal_bsp.a(alt_errno.o)
 .debug_info    0x000164a3      0x15c ../TR4_HDMI_TX_RX_bsp/\libhal_bsp.a(alt_icache_flush_all.o)
 .debug_info    0x000165ff      0x493 ../TR4_HDMI_TX_RX_bsp/\libhal_bsp.a(alt_iic.o)
 .debug_info    0x00016a92      0x314 ../TR4_HDMI_TX_RX_bsp/\libhal_bsp.a(alt_iic_isr_register.o)
 .debug_info    0x00016da6      0x695 ../TR4_HDMI_TX_RX_bsp/\libhal_bsp.a(alt_io_redirect.o)
 .debug_info    0x0001743b       0x84 ../TR4_HDMI_TX_RX_bsp/\libhal_bsp.a(alt_irq_entry.o)
 .debug_info    0x000174bf      0x275 ../TR4_HDMI_TX_RX_bsp/\libhal_bsp.a(alt_irq_handler.o)
 .debug_info    0x00017734      0x525 ../TR4_HDMI_TX_RX_bsp/\libhal_bsp.a(alt_open.o)
 .debug_info    0x00017c59      0x3f2 ../TR4_HDMI_TX_RX_bsp/\libhal_bsp.a(alt_release_fd.o)
 .debug_info    0x0001804b      0x163 ../TR4_HDMI_TX_RX_bsp/\libhal_bsp.a(altera_nios2_qsys_irq.o)
 .debug_info    0x000181ae       0x8a ../TR4_HDMI_TX_RX_bsp/\libhal_bsp.a(alt_exception_entry.o)
 .debug_info    0x00018238      0x418 ../TR4_HDMI_TX_RX_bsp/\libhal_bsp.a(alt_find_dev.o)
 .debug_info    0x00018650      0x41f ../TR4_HDMI_TX_RX_bsp/\libhal_bsp.a(alt_find_file.o)
 .debug_info    0x00018a6f      0x460 ../TR4_HDMI_TX_RX_bsp/\libhal_bsp.a(alt_get_fd.o)
 .debug_info    0x00018ecf      0x1a4 ../TR4_HDMI_TX_RX_bsp/\libhal_bsp.a(alt_icache_flush.o)
 .debug_info    0x00019073      0x186 c:/altera/11.1/nios2eds/bin/gnu/h-i686-mingw32/bin/../lib/gcc/nios2-elf/4.1.2/../../../../nios2-elf/lib/mhw-mulx\libsmallc.a(lib_a-atexit.o)
 .debug_info    0x000191f9       0x9f c:/altera/11.1/nios2eds/bin/gnu/h-i686-mingw32/bin/../lib/gcc/nios2-elf/4.1.2/../../../../nios2-elf/lib/mhw-mulx\libsmallc.a(lib_a-exit.o)
 .debug_info    0x00019298       0xef c:/altera/11.1/nios2eds/bin/gnu/h-i686-mingw32/bin/../lib/gcc/nios2-elf/4.1.2/../../../../nios2-elf/lib/mhw-mulx\libsmallc.a(lib_a-memcmp.o)
 .debug_info    0x00019387      0x68f c:/altera/11.1/nios2eds/bin/gnu/h-i686-mingw32/bin/../lib/gcc/nios2-elf/4.1.2/../../../../nios2-elf/lib/mhw-mulx\libsmallc.a(lib_a-__atexit.o)
 .debug_info    0x00019a16      0x6d5 c:/altera/11.1/nios2eds/bin/gnu/h-i686-mingw32/bin/../lib/gcc/nios2-elf/4.1.2/../../../../nios2-elf/lib/mhw-mulx\libsmallc.a(lib_a-__call_atexit.o)
 .debug_info    0x0001a0eb      0x18d ../TR4_HDMI_TX_RX_bsp/\libhal_bsp.a(alt_exit.o)

.debug_abbrev   0x00000000     0x50fe
 *(.debug_abbrev)
 .debug_abbrev  0x00000000       0x12 ../TR4_HDMI_TX_RX_bsp//obj/HAL/src/crt0.o
 .debug_abbrev  0x00000012       0x5a obj/Beep.o
 .debug_abbrev  0x0000006c      0x205 obj/HDMI_Lib/HDMI_RX/HDMI_RX.o
 .debug_abbrev  0x00000271      0x26f obj/HDMI_Lib/HDMI_RX/it6605.o
 .debug_abbrev  0x000004e0      0x142 obj/HDMI_Lib/HDMI_TX/EDID.o
 .debug_abbrev  0x00000622      0x1e9 obj/HDMI_Lib/HDMI_TX/HDMI_TX.o
 .debug_abbrev  0x0000080b       0x76 obj/HDMI_Lib/HDMI_TX/dss_sha.o
 .debug_abbrev  0x00000881      0x2f5 obj/HDMI_Lib/HDMI_TX/it6613_drv.o
 .debug_abbrev  0x00000b76      0x23d obj/HDMI_Lib/HDMI_TX/it6613_sys.o
 .debug_abbrev  0x00000db3      0x28b obj/HDMI_Lib/mcu.o
 .debug_abbrev  0x0000103e      0x1c3 obj/main.o
 .debug_abbrev  0x00001201       0xe2 obj/terasic_lib/I2C.o
 .debug_abbrev  0x000012e3       0xfa obj/terasic_lib/debug.o
 .debug_abbrev  0x000013dd      0x204 c:/altera/11.1/nios2eds/bin/gnu/h-i686-mingw32/bin/../lib/gcc/nios2-elf/4.1.2/mhw-mulx\libgcc.a(_mul_df.o)
 .debug_abbrev  0x000015e1      0x1e3 c:/altera/11.1/nios2eds/bin/gnu/h-i686-mingw32/bin/../lib/gcc/nios2-elf/4.1.2/mhw-mulx\libgcc.a(_div_df.o)
 .debug_abbrev  0x000017c4      0x13f c:/altera/11.1/nios2eds/bin/gnu/h-i686-mingw32/bin/../lib/gcc/nios2-elf/4.1.2/mhw-mulx\libgcc.a(_si_to_df.o)
 .debug_abbrev  0x00001903       0xba c:/altera/11.1/nios2eds/bin/gnu/h-i686-mingw32/bin/../lib/gcc/nios2-elf/4.1.2/mhw-mulx\libgcc.a(_thenan_df.o)
 .debug_abbrev  0x000019bd       0xe0 c:/altera/11.1/nios2eds/bin/gnu/h-i686-mingw32/bin/../lib/gcc/nios2-elf/4.1.2/mhw-mulx\libgcc.a(lib2-divmod.o)
 .debug_abbrev  0x00001a9d       0xb9 c:/altera/11.1/nios2eds/bin/gnu/h-i686-mingw32/bin/../lib/gcc/nios2-elf/4.1.2/mhw-mulx\libgcc.a(_clzsi2.o)
 .debug_abbrev  0x00001b56      0x1b1 c:/altera/11.1/nios2eds/bin/gnu/h-i686-mingw32/bin/../lib/gcc/nios2-elf/4.1.2/mhw-mulx\libgcc.a(_pack_df.o)
 .debug_abbrev  0x00001d07      0x149 c:/altera/11.1/nios2eds/bin/gnu/h-i686-mingw32/bin/../lib/gcc/nios2-elf/4.1.2/mhw-mulx\libgcc.a(_unpack_df.o)
 .debug_abbrev  0x00001e50       0x61 c:/altera/11.1/nios2eds/bin/gnu/h-i686-mingw32/bin/../lib/gcc/nios2-elf/4.1.2/mhw-mulx\libgcc.a(_clz.o)
 .debug_abbrev  0x00001eb1      0x13f c:/altera/11.1/nios2eds/bin/gnu/h-i686-mingw32/bin/../lib/gcc/nios2-elf/4.1.2/../../../../nios2-elf/lib/mhw-mulx\libsmallc.a(lib_a-impure.o)
 .debug_abbrev  0x00001ff0       0x8b c:/altera/11.1/nios2eds/bin/gnu/h-i686-mingw32/bin/../lib/gcc/nios2-elf/4.1.2/../../../../nios2-elf/lib/mhw-mulx\libsmallc.a(lib_a-memset.o)
 .debug_abbrev  0x0000207b      0x179 c:/altera/11.1/nios2eds/bin/gnu/h-i686-mingw32/bin/../lib/gcc/nios2-elf/4.1.2/../../../../nios2-elf/lib/mhw-mulx\libsmallc.a(lib_a-printf.o)
 .debug_abbrev  0x000021f4      0x158 c:/altera/11.1/nios2eds/bin/gnu/h-i686-mingw32/bin/../lib/gcc/nios2-elf/4.1.2/../../../../nios2-elf/lib/mhw-mulx\libsmallc.a(lib_a-putchar.o)
 .debug_abbrev  0x0000234c      0x180 c:/altera/11.1/nios2eds/bin/gnu/h-i686-mingw32/bin/../lib/gcc/nios2-elf/4.1.2/../../../../nios2-elf/lib/mhw-mulx\libsmallc.a(lib_a-puts.o)
 .debug_abbrev  0x000024cc      0x179 c:/altera/11.1/nios2eds/bin/gnu/h-i686-mingw32/bin/../lib/gcc/nios2-elf/4.1.2/../../../../nios2-elf/lib/mhw-mulx\libsmallc.a(lib_a-sprintf.o)
 .debug_abbrev  0x00002645       0x7a c:/altera/11.1/nios2eds/bin/gnu/h-i686-mingw32/bin/../lib/gcc/nios2-elf/4.1.2/../../../../nios2-elf/lib/mhw-mulx\libsmallc.a(lib_a-strlen.o)
 .debug_abbrev  0x000026bf      0x247 c:/altera/11.1/nios2eds/bin/gnu/h-i686-mingw32/bin/../lib/gcc/nios2-elf/4.1.2/../../../../nios2-elf/lib/mhw-mulx\libsmallc.a(lib_a-vfprintf.o)
 .debug_abbrev  0x00002906      0x163 c:/altera/11.1/nios2eds/bin/gnu/h-i686-mingw32/bin/../lib/gcc/nios2-elf/4.1.2/../../../../nios2-elf/lib/mhw-mulx\libsmallc.a(lib_a-vfprintf_1.o)
 .debug_abbrev  0x00002a69      0x194 c:/altera/11.1/nios2eds/bin/gnu/h-i686-mingw32/bin/../lib/gcc/nios2-elf/4.1.2/../../../../nios2-elf/lib/mhw-mulx\libsmallc.a(lib_a-vsnprintf.o)
 .debug_abbrev  0x00002bfd      0x179 c:/altera/11.1/nios2eds/bin/gnu/h-i686-mingw32/bin/../lib/gcc/nios2-elf/4.1.2/../../../../nios2-elf/lib/mhw-mulx\libsmallc.a(lib_a-fvwrite_small_dev.o)
 .debug_abbrev  0x00002d76      0x184 c:/altera/11.1/nios2eds/bin/gnu/h-i686-mingw32/bin/../lib/gcc/nios2-elf/4.1.2/../../../../nios2-elf/lib/mhw-mulx\libsmallc.a(lib_a-fvwrite_small_str.o)
 .debug_abbrev  0x00002efa       0xa8 c:/altera/11.1/nios2eds/bin/gnu/h-i686-mingw32/bin/../lib/gcc/nios2-elf/4.1.2/../../../../nios2-elf/lib/mhw-mulx\libsmallc.a(lib_a-memmove.o)
 .debug_abbrev  0x00002fa2      0x167 c:/altera/11.1/nios2eds/bin/gnu/h-i686-mingw32/bin/../lib/gcc/nios2-elf/4.1.2/../../../../nios2-elf/lib/mhw-mulx\libsmallc.a(lib_a-putc.o)
 .debug_abbrev  0x00003109      0x16c c:/altera/11.1/nios2eds/bin/gnu/h-i686-mingw32/bin/../lib/gcc/nios2-elf/4.1.2/../../../../nios2-elf/lib/mhw-mulx\libsmallc.a(lib_a-writer.o)
 .debug_abbrev  0x00003275       0x3b c:/altera/11.1/nios2eds/bin/gnu/h-i686-mingw32/bin/../lib/gcc/nios2-elf/4.1.2/../../../../nios2-elf/lib/mhw-mulx\libsmallc.a(lib_a-int_errno.o)
 .debug_abbrev  0x000032b0      0x180 ../TR4_HDMI_TX_RX_bsp/\libhal_bsp.a(alt_irq_register.o)
 .debug_abbrev  0x00003430       0x44 ../TR4_HDMI_TX_RX_bsp/\libhal_bsp.a(alt_irq_vars.o)
 .debug_abbrev  0x00003474       0x88 ../TR4_HDMI_TX_RX_bsp/\libhal_bsp.a(alt_load.o)
 .debug_abbrev  0x000034fc       0xb7 ../TR4_HDMI_TX_RX_bsp/\libhal_bsp.a(alt_main.o)
 .debug_abbrev  0x000035b3      0x150 ../TR4_HDMI_TX_RX_bsp/\libhal_bsp.a(alt_tick.o)
 .debug_abbrev  0x00003703       0x5d ../TR4_HDMI_TX_RX_bsp/\libhal_bsp.a(alt_usleep.o)
 .debug_abbrev  0x00003760      0x100 ../TR4_HDMI_TX_RX_bsp/\libhal_bsp.a(alt_write.o)
 .debug_abbrev  0x00003860      0x121 ../TR4_HDMI_TX_RX_bsp/\libhal_bsp.a(alt_sys_init.o)
 .debug_abbrev  0x00003981       0xcb ../TR4_HDMI_TX_RX_bsp/\libhal_bsp.a(altera_avalon_jtag_uart_fd.o)
 .debug_abbrev  0x00003a4c       0xb6 ../TR4_HDMI_TX_RX_bsp/\libhal_bsp.a(altera_avalon_jtag_uart_read.o)
 .debug_abbrev  0x00003b02       0xb4 ../TR4_HDMI_TX_RX_bsp/\libhal_bsp.a(altera_avalon_jtag_uart_write.o)
 .debug_abbrev  0x00003bb6      0x137 ../TR4_HDMI_TX_RX_bsp/\libhal_bsp.a(altera_avalon_timer_sc.o)
 .debug_abbrev  0x00003ced       0x6c ../TR4_HDMI_TX_RX_bsp/\libhal_bsp.a(alt_busy_sleep.o)
 .debug_abbrev  0x00003d59       0xfb ../TR4_HDMI_TX_RX_bsp/\libhal_bsp.a(alt_close.o)
 .debug_abbrev  0x00003e54       0x3f ../TR4_HDMI_TX_RX_bsp/\libhal_bsp.a(alt_dcache_flush_all.o)
 .debug_abbrev  0x00003e93       0xc7 ../TR4_HDMI_TX_RX_bsp/\libhal_bsp.a(alt_dev.o)
 .debug_abbrev  0x00003f5a       0xf6 ../TR4_HDMI_TX_RX_bsp/\libhal_bsp.a(alt_dev_llist_insert.o)
 .debug_abbrev  0x00004050       0x76 ../TR4_HDMI_TX_RX_bsp/\libhal_bsp.a(alt_do_ctors.o)
 .debug_abbrev  0x000040c6       0x76 ../TR4_HDMI_TX_RX_bsp/\libhal_bsp.a(alt_do_dtors.o)
 .debug_abbrev  0x0000413c       0x5e ../TR4_HDMI_TX_RX_bsp/\libhal_bsp.a(alt_errno.o)
 .debug_abbrev  0x0000419a       0x3f ../TR4_HDMI_TX_RX_bsp/\libhal_bsp.a(alt_icache_flush_all.o)
 .debug_abbrev  0x000041d9      0x134 ../TR4_HDMI_TX_RX_bsp/\libhal_bsp.a(alt_iic.o)
 .debug_abbrev  0x0000430d      0x14e ../TR4_HDMI_TX_RX_bsp/\libhal_bsp.a(alt_iic_isr_register.o)
 .debug_abbrev  0x0000445b       0xf0 ../TR4_HDMI_TX_RX_bsp/\libhal_bsp.a(alt_io_redirect.o)
 .debug_abbrev  0x0000454b       0x12 ../TR4_HDMI_TX_RX_bsp/\libhal_bsp.a(alt_irq_entry.o)
 .debug_abbrev  0x0000455d      0x10c ../TR4_HDMI_TX_RX_bsp/\libhal_bsp.a(alt_irq_handler.o)
 .debug_abbrev  0x00004669      0x112 ../TR4_HDMI_TX_RX_bsp/\libhal_bsp.a(alt_open.o)
 .debug_abbrev  0x0000477b       0xc1 ../TR4_HDMI_TX_RX_bsp/\libhal_bsp.a(alt_release_fd.o)
 .debug_abbrev  0x0000483c       0x3f ../TR4_HDMI_TX_RX_bsp/\libhal_bsp.a(altera_nios2_qsys_irq.o)
 .debug_abbrev  0x0000487b       0x12 ../TR4_HDMI_TX_RX_bsp/\libhal_bsp.a(alt_exception_entry.o)
 .debug_abbrev  0x0000488d       0xcf ../TR4_HDMI_TX_RX_bsp/\libhal_bsp.a(alt_find_dev.o)
 .debug_abbrev  0x0000495c       0xcf ../TR4_HDMI_TX_RX_bsp/\libhal_bsp.a(alt_find_file.o)
 .debug_abbrev  0x00004a2b       0xfb ../TR4_HDMI_TX_RX_bsp/\libhal_bsp.a(alt_get_fd.o)
 .debug_abbrev  0x00004b26       0x7a ../TR4_HDMI_TX_RX_bsp/\libhal_bsp.a(alt_icache_flush.o)
 .debug_abbrev  0x00004ba0       0xc6 c:/altera/11.1/nios2eds/bin/gnu/h-i686-mingw32/bin/../lib/gcc/nios2-elf/4.1.2/../../../../nios2-elf/lib/mhw-mulx\libsmallc.a(lib_a-atexit.o)
 .debug_abbrev  0x00004c66       0x4e c:/altera/11.1/nios2eds/bin/gnu/h-i686-mingw32/bin/../lib/gcc/nios2-elf/4.1.2/../../../../nios2-elf/lib/mhw-mulx\libsmallc.a(lib_a-exit.o)
 .debug_abbrev  0x00004cb4       0x7c c:/altera/11.1/nios2eds/bin/gnu/h-i686-mingw32/bin/../lib/gcc/nios2-elf/4.1.2/../../../../nios2-elf/lib/mhw-mulx\libsmallc.a(lib_a-memcmp.o)
 .debug_abbrev  0x00004d30      0x196 c:/altera/11.1/nios2eds/bin/gnu/h-i686-mingw32/bin/../lib/gcc/nios2-elf/4.1.2/../../../../nios2-elf/lib/mhw-mulx\libsmallc.a(lib_a-__atexit.o)
 .debug_abbrev  0x00004ec6      0x1c6 c:/altera/11.1/nios2eds/bin/gnu/h-i686-mingw32/bin/../lib/gcc/nios2-elf/4.1.2/../../../../nios2-elf/lib/mhw-mulx\libsmallc.a(lib_a-__call_atexit.o)
 .debug_abbrev  0x0000508c       0x72 ../TR4_HDMI_TX_RX_bsp/\libhal_bsp.a(alt_exit.o)

.debug_line     0x00000000    0x12c7f
 *(.debug_line)
 .debug_line    0x00000000       0x6c ../TR4_HDMI_TX_RX_bsp//obj/HAL/src/crt0.o
 .debug_line    0x0000006c       0x4b obj/Beep.o
 .debug_line    0x000000b7      0xa2c obj/HDMI_Lib/HDMI_RX/HDMI_RX.o
 .debug_line    0x00000ae3     0x2c74 obj/HDMI_Lib/HDMI_RX/it6605.o
 .debug_line    0x00003757      0x621 obj/HDMI_Lib/HDMI_TX/EDID.o
 .debug_line    0x00003d78      0x7ee obj/HDMI_Lib/HDMI_TX/HDMI_TX.o
 .debug_line    0x00004566      0x315 obj/HDMI_Lib/HDMI_TX/dss_sha.o
 .debug_line    0x0000487b     0x296b obj/HDMI_Lib/HDMI_TX/it6613_drv.o
 .debug_line    0x000071e6      0xa12 obj/HDMI_Lib/HDMI_TX/it6613_sys.o
 .debug_line    0x00007bf8      0x831 obj/HDMI_Lib/mcu.o
 .debug_line    0x00008429      0x9e6 obj/main.o
 .debug_line    0x00008e0f      0x6b9 obj/terasic_lib/I2C.o
 .debug_line    0x000094c8      0x381 obj/terasic_lib/debug.o
 .debug_line    0x00009849      0x41b c:/altera/11.1/nios2eds/bin/gnu/h-i686-mingw32/bin/../lib/gcc/nios2-elf/4.1.2/mhw-mulx\libgcc.a(_mul_df.o)
 .debug_line    0x00009c64      0x301 c:/altera/11.1/nios2eds/bin/gnu/h-i686-mingw32/bin/../lib/gcc/nios2-elf/4.1.2/mhw-mulx\libgcc.a(_div_df.o)
 .debug_line    0x00009f65      0x175 c:/altera/11.1/nios2eds/bin/gnu/h-i686-mingw32/bin/../lib/gcc/nios2-elf/4.1.2/mhw-mulx\libgcc.a(_si_to_df.o)
 .debug_line    0x0000a0da       0x94 c:/altera/11.1/nios2eds/bin/gnu/h-i686-mingw32/bin/../lib/gcc/nios2-elf/4.1.2/mhw-mulx\libgcc.a(_thenan_df.o)
 .debug_line    0x0000a16e      0x24f c:/altera/11.1/nios2eds/bin/gnu/h-i686-mingw32/bin/../lib/gcc/nios2-elf/4.1.2/mhw-mulx\libgcc.a(lib2-divmod.o)
 .debug_line    0x0000a3bd      0x105 c:/altera/11.1/nios2eds/bin/gnu/h-i686-mingw32/bin/../lib/gcc/nios2-elf/4.1.2/mhw-mulx\libgcc.a(_clzsi2.o)
 .debug_line    0x0000a4c2      0x222 c:/altera/11.1/nios2eds/bin/gnu/h-i686-mingw32/bin/../lib/gcc/nios2-elf/4.1.2/mhw-mulx\libgcc.a(_pack_df.o)
 .debug_line    0x0000a6e4      0x1e4 c:/altera/11.1/nios2eds/bin/gnu/h-i686-mingw32/bin/../lib/gcc/nios2-elf/4.1.2/mhw-mulx\libgcc.a(_unpack_df.o)
 .debug_line    0x0000a8c8       0xaa c:/altera/11.1/nios2eds/bin/gnu/h-i686-mingw32/bin/../lib/gcc/nios2-elf/4.1.2/mhw-mulx\libgcc.a(_clz.o)
 .debug_line    0x0000a972      0x230 c:/altera/11.1/nios2eds/bin/gnu/h-i686-mingw32/bin/../lib/gcc/nios2-elf/4.1.2/../../../../nios2-elf/lib/mhw-mulx\libsmallc.a(lib_a-impure.o)
 .debug_line    0x0000aba2      0x258 c:/altera/11.1/nios2eds/bin/gnu/h-i686-mingw32/bin/../lib/gcc/nios2-elf/4.1.2/../../../../nios2-elf/lib/mhw-mulx\libsmallc.a(lib_a-memset.o)
 .debug_line    0x0000adfa      0x2be c:/altera/11.1/nios2eds/bin/gnu/h-i686-mingw32/bin/../lib/gcc/nios2-elf/4.1.2/../../../../nios2-elf/lib/mhw-mulx\libsmallc.a(lib_a-printf.o)
 .debug_line    0x0000b0b8      0x267 c:/altera/11.1/nios2eds/bin/gnu/h-i686-mingw32/bin/../lib/gcc/nios2-elf/4.1.2/../../../../nios2-elf/lib/mhw-mulx\libsmallc.a(lib_a-putchar.o)
 .debug_line    0x0000b31f      0x2b2 c:/altera/11.1/nios2eds/bin/gnu/h-i686-mingw32/bin/../lib/gcc/nios2-elf/4.1.2/../../../../nios2-elf/lib/mhw-mulx\libsmallc.a(lib_a-puts.o)
 .debug_line    0x0000b5d1      0x365 c:/altera/11.1/nios2eds/bin/gnu/h-i686-mingw32/bin/../lib/gcc/nios2-elf/4.1.2/../../../../nios2-elf/lib/mhw-mulx\libsmallc.a(lib_a-sprintf.o)
 .debug_line    0x0000b936      0x250 c:/altera/11.1/nios2eds/bin/gnu/h-i686-mingw32/bin/../lib/gcc/nios2-elf/4.1.2/../../../../nios2-elf/lib/mhw-mulx\libsmallc.a(lib_a-strlen.o)
 .debug_line    0x0000bb86      0x5db c:/altera/11.1/nios2eds/bin/gnu/h-i686-mingw32/bin/../lib/gcc/nios2-elf/4.1.2/../../../../nios2-elf/lib/mhw-mulx\libsmallc.a(lib_a-vfprintf.o)
 .debug_line    0x0000c161      0x238 c:/altera/11.1/nios2eds/bin/gnu/h-i686-mingw32/bin/../lib/gcc/nios2-elf/4.1.2/../../../../nios2-elf/lib/mhw-mulx\libsmallc.a(lib_a-vfprintf_1.o)
 .debug_line    0x0000c399      0x340 c:/altera/11.1/nios2eds/bin/gnu/h-i686-mingw32/bin/../lib/gcc/nios2-elf/4.1.2/../../../../nios2-elf/lib/mhw-mulx\libsmallc.a(lib_a-vsnprintf.o)
 .debug_line    0x0000c6d9      0x2a9 c:/altera/11.1/nios2eds/bin/gnu/h-i686-mingw32/bin/../lib/gcc/nios2-elf/4.1.2/../../../../nios2-elf/lib/mhw-mulx\libsmallc.a(lib_a-fvwrite_small_dev.o)
 .debug_line    0x0000c982      0x2cf c:/altera/11.1/nios2eds/bin/gnu/h-i686-mingw32/bin/../lib/gcc/nios2-elf/4.1.2/../../../../nios2-elf/lib/mhw-mulx\libsmallc.a(lib_a-fvwrite_small_str.o)
 .debug_line    0x0000cc51      0x294 c:/altera/11.1/nios2eds/bin/gnu/h-i686-mingw32/bin/../lib/gcc/nios2-elf/4.1.2/../../../../nios2-elf/lib/mhw-mulx\libsmallc.a(lib_a-memmove.o)
 .debug_line    0x0000cee5      0x2d2 c:/altera/11.1/nios2eds/bin/gnu/h-i686-mingw32/bin/../lib/gcc/nios2-elf/4.1.2/../../../../nios2-elf/lib/mhw-mulx\libsmallc.a(lib_a-putc.o)
 .debug_line    0x0000d1b7      0x29d c:/altera/11.1/nios2eds/bin/gnu/h-i686-mingw32/bin/../lib/gcc/nios2-elf/4.1.2/../../../../nios2-elf/lib/mhw-mulx\libsmallc.a(lib_a-writer.o)
 .debug_line    0x0000d454      0x1e2 c:/altera/11.1/nios2eds/bin/gnu/h-i686-mingw32/bin/../lib/gcc/nios2-elf/4.1.2/../../../../nios2-elf/lib/mhw-mulx\libsmallc.a(lib_a-int_errno.o)
 .debug_line    0x0000d636      0x2fd ../TR4_HDMI_TX_RX_bsp/\libhal_bsp.a(alt_irq_register.o)
 .debug_line    0x0000d933       0x72 ../TR4_HDMI_TX_RX_bsp/\libhal_bsp.a(alt_irq_vars.o)
 .debug_line    0x0000d9a5      0x211 ../TR4_HDMI_TX_RX_bsp/\libhal_bsp.a(alt_load.o)
 .debug_line    0x0000dbb6      0x2c4 ../TR4_HDMI_TX_RX_bsp/\libhal_bsp.a(alt_main.o)
 .debug_line    0x0000de7a      0x2d6 ../TR4_HDMI_TX_RX_bsp/\libhal_bsp.a(alt_tick.o)
 .debug_line    0x0000e150      0x1f9 ../TR4_HDMI_TX_RX_bsp/\libhal_bsp.a(alt_usleep.o)
 .debug_line    0x0000e349      0x2c3 ../TR4_HDMI_TX_RX_bsp/\libhal_bsp.a(alt_write.o)
 .debug_line    0x0000e60c      0x2c1 ../TR4_HDMI_TX_RX_bsp/\libhal_bsp.a(alt_sys_init.o)
 .debug_line    0x0000e8cd      0x1d4 ../TR4_HDMI_TX_RX_bsp/\libhal_bsp.a(altera_avalon_jtag_uart_fd.o)
 .debug_line    0x0000eaa1      0x33d ../TR4_HDMI_TX_RX_bsp/\libhal_bsp.a(altera_avalon_jtag_uart_read.o)
 .debug_line    0x0000edde      0x2fe ../TR4_HDMI_TX_RX_bsp/\libhal_bsp.a(altera_avalon_jtag_uart_write.o)
 .debug_line    0x0000f0dc      0x2ad ../TR4_HDMI_TX_RX_bsp/\libhal_bsp.a(altera_avalon_timer_sc.o)
 .debug_line    0x0000f389      0x253 ../TR4_HDMI_TX_RX_bsp/\libhal_bsp.a(alt_busy_sleep.o)
 .debug_line    0x0000f5dc      0x293 ../TR4_HDMI_TX_RX_bsp/\libhal_bsp.a(alt_close.o)
 .debug_line    0x0000f86f      0x1af ../TR4_HDMI_TX_RX_bsp/\libhal_bsp.a(alt_dcache_flush_all.o)
 .debug_line    0x0000fa1e      0x24e ../TR4_HDMI_TX_RX_bsp/\libhal_bsp.a(alt_dev.o)
 .debug_line    0x0000fc6c      0x254 ../TR4_HDMI_TX_RX_bsp/\libhal_bsp.a(alt_dev_llist_insert.o)
 .debug_line    0x0000fec0       0x83 ../TR4_HDMI_TX_RX_bsp/\libhal_bsp.a(alt_do_ctors.o)
 .debug_line    0x0000ff43       0x83 ../TR4_HDMI_TX_RX_bsp/\libhal_bsp.a(alt_do_dtors.o)
 .debug_line    0x0000ffc6      0x1a4 ../TR4_HDMI_TX_RX_bsp/\libhal_bsp.a(alt_errno.o)
 .debug_line    0x0001016a      0x1b7 ../TR4_HDMI_TX_RX_bsp/\libhal_bsp.a(alt_icache_flush_all.o)
 .debug_line    0x00010321      0x2c2 ../TR4_HDMI_TX_RX_bsp/\libhal_bsp.a(alt_iic.o)
 .debug_line    0x000105e3      0x243 ../TR4_HDMI_TX_RX_bsp/\libhal_bsp.a(alt_iic_isr_register.o)
 .debug_line    0x00010826      0x2ae ../TR4_HDMI_TX_RX_bsp/\libhal_bsp.a(alt_io_redirect.o)
 .debug_line    0x00010ad4       0x6b ../TR4_HDMI_TX_RX_bsp/\libhal_bsp.a(alt_irq_entry.o)
 .debug_line    0x00010b3f      0x242 ../TR4_HDMI_TX_RX_bsp/\libhal_bsp.a(alt_irq_handler.o)
 .debug_line    0x00010d81      0x2f9 ../TR4_HDMI_TX_RX_bsp/\libhal_bsp.a(alt_open.o)
 .debug_line    0x0001107a       0xed ../TR4_HDMI_TX_RX_bsp/\libhal_bsp.a(alt_release_fd.o)
 .debug_line    0x00011167      0x1c8 ../TR4_HDMI_TX_RX_bsp/\libhal_bsp.a(altera_nios2_qsys_irq.o)
 .debug_line    0x0001132f       0xab ../TR4_HDMI_TX_RX_bsp/\libhal_bsp.a(alt_exception_entry.o)
 .debug_line    0x000113da      0x265 ../TR4_HDMI_TX_RX_bsp/\libhal_bsp.a(alt_find_dev.o)
 .debug_line    0x0001163f      0x276 ../TR4_HDMI_TX_RX_bsp/\libhal_bsp.a(alt_find_file.o)
 .debug_line    0x000118b5      0x291 ../TR4_HDMI_TX_RX_bsp/\libhal_bsp.a(alt_get_fd.o)
 .debug_line    0x00011b46      0x1f3 ../TR4_HDMI_TX_RX_bsp/\libhal_bsp.a(alt_icache_flush.o)
 .debug_line    0x00011d39      0x203 c:/altera/11.1/nios2eds/bin/gnu/h-i686-mingw32/bin/../lib/gcc/nios2-elf/4.1.2/../../../../nios2-elf/lib/mhw-mulx\libsmallc.a(lib_a-atexit.o)
 .debug_line    0x00011f3c      0x223 c:/altera/11.1/nios2eds/bin/gnu/h-i686-mingw32/bin/../lib/gcc/nios2-elf/4.1.2/../../../../nios2-elf/lib/mhw-mulx\libsmallc.a(lib_a-exit.o)
 .debug_line    0x0001215f      0x270 c:/altera/11.1/nios2eds/bin/gnu/h-i686-mingw32/bin/../lib/gcc/nios2-elf/4.1.2/../../../../nios2-elf/lib/mhw-mulx\libsmallc.a(lib_a-memcmp.o)
 .debug_line    0x000123cf      0x350 c:/altera/11.1/nios2eds/bin/gnu/h-i686-mingw32/bin/../lib/gcc/nios2-elf/4.1.2/../../../../nios2-elf/lib/mhw-mulx\libsmallc.a(lib_a-__atexit.o)
 .debug_line    0x0001271f      0x360 c:/altera/11.1/nios2eds/bin/gnu/h-i686-mingw32/bin/../lib/gcc/nios2-elf/4.1.2/../../../../nios2-elf/lib/mhw-mulx\libsmallc.a(lib_a-__call_atexit.o)
 .debug_line    0x00012a7f      0x200 ../TR4_HDMI_TX_RX_bsp/\libhal_bsp.a(alt_exit.o)

.debug_frame    0x00000000     0x2a24
 *(.debug_frame)
 .debug_frame   0x00000000      0x184 obj/HDMI_Lib/HDMI_RX/HDMI_RX.o
 .debug_frame   0x00000184      0xb34 obj/HDMI_Lib/HDMI_RX/it6605.o
 .debug_frame   0x00000cb8       0x64 obj/HDMI_Lib/HDMI_TX/EDID.o
 .debug_frame   0x00000d1c      0x1b8 obj/HDMI_Lib/HDMI_TX/HDMI_TX.o
 .debug_frame   0x00000ed4      0x840 obj/HDMI_Lib/HDMI_TX/it6613_drv.o
 .debug_frame   0x00001714       0x9c obj/HDMI_Lib/HDMI_TX/it6613_sys.o
 .debug_frame   0x000017b0      0x35c obj/HDMI_Lib/mcu.o
 .debug_frame   0x00001b0c      0x12c obj/main.o
 .debug_frame   0x00001c38      0x10c obj/terasic_lib/I2C.o
 .debug_frame   0x00001d44       0x84 obj/terasic_lib/debug.o
 .debug_frame   0x00001dc8       0x3c c:/altera/11.1/nios2eds/bin/gnu/h-i686-mingw32/bin/../lib/gcc/nios2-elf/4.1.2/mhw-mulx\libgcc.a(_mul_df.o)
 .debug_frame   0x00001e04       0x30 c:/altera/11.1/nios2eds/bin/gnu/h-i686-mingw32/bin/../lib/gcc/nios2-elf/4.1.2/mhw-mulx\libgcc.a(_div_df.o)
 .debug_frame   0x00001e34       0x30 c:/altera/11.1/nios2eds/bin/gnu/h-i686-mingw32/bin/../lib/gcc/nios2-elf/4.1.2/mhw-mulx\libgcc.a(_si_to_df.o)
 .debug_frame   0x00001e64       0x70 c:/altera/11.1/nios2eds/bin/gnu/h-i686-mingw32/bin/../lib/gcc/nios2-elf/4.1.2/mhw-mulx\libgcc.a(lib2-divmod.o)
 .debug_frame   0x00001ed4       0x20 c:/altera/11.1/nios2eds/bin/gnu/h-i686-mingw32/bin/../lib/gcc/nios2-elf/4.1.2/mhw-mulx\libgcc.a(_clzsi2.o)
 .debug_frame   0x00001ef4       0x2c c:/altera/11.1/nios2eds/bin/gnu/h-i686-mingw32/bin/../lib/gcc/nios2-elf/4.1.2/mhw-mulx\libgcc.a(_pack_df.o)
 .debug_frame   0x00001f20       0x20 c:/altera/11.1/nios2eds/bin/gnu/h-i686-mingw32/bin/../lib/gcc/nios2-elf/4.1.2/mhw-mulx\libgcc.a(_unpack_df.o)
 .debug_frame   0x00001f40       0x20 c:/altera/11.1/nios2eds/bin/gnu/h-i686-mingw32/bin/../lib/gcc/nios2-elf/4.1.2/../../../../nios2-elf/lib/mhw-mulx\libsmallc.a(lib_a-memset.o)
 .debug_frame   0x00001f60       0x40 c:/altera/11.1/nios2eds/bin/gnu/h-i686-mingw32/bin/../lib/gcc/nios2-elf/4.1.2/../../../../nios2-elf/lib/mhw-mulx\libsmallc.a(lib_a-printf.o)
 .debug_frame   0x00001fa0       0x30 c:/altera/11.1/nios2eds/bin/gnu/h-i686-mingw32/bin/../lib/gcc/nios2-elf/4.1.2/../../../../nios2-elf/lib/mhw-mulx\libsmallc.a(lib_a-putchar.o)
 .debug_frame   0x00001fd0       0x3c c:/altera/11.1/nios2eds/bin/gnu/h-i686-mingw32/bin/../lib/gcc/nios2-elf/4.1.2/../../../../nios2-elf/lib/mhw-mulx\libsmallc.a(lib_a-puts.o)
 .debug_frame   0x0000200c       0x40 c:/altera/11.1/nios2eds/bin/gnu/h-i686-mingw32/bin/../lib/gcc/nios2-elf/4.1.2/../../../../nios2-elf/lib/mhw-mulx\libsmallc.a(lib_a-sprintf.o)
 .debug_frame   0x0000204c       0x20 c:/altera/11.1/nios2eds/bin/gnu/h-i686-mingw32/bin/../lib/gcc/nios2-elf/4.1.2/../../../../nios2-elf/lib/mhw-mulx\libsmallc.a(lib_a-strlen.o)
 .debug_frame   0x0000206c       0x64 c:/altera/11.1/nios2eds/bin/gnu/h-i686-mingw32/bin/../lib/gcc/nios2-elf/4.1.2/../../../../nios2-elf/lib/mhw-mulx\libsmallc.a(lib_a-vfprintf.o)
 .debug_frame   0x000020d0       0x20 c:/altera/11.1/nios2eds/bin/gnu/h-i686-mingw32/bin/../lib/gcc/nios2-elf/4.1.2/../../../../nios2-elf/lib/mhw-mulx\libsmallc.a(lib_a-vfprintf_1.o)
 .debug_frame   0x000020f0       0x44 c:/altera/11.1/nios2eds/bin/gnu/h-i686-mingw32/bin/../lib/gcc/nios2-elf/4.1.2/../../../../nios2-elf/lib/mhw-mulx\libsmallc.a(lib_a-vsnprintf.o)
 .debug_frame   0x00002134       0x30 c:/altera/11.1/nios2eds/bin/gnu/h-i686-mingw32/bin/../lib/gcc/nios2-elf/4.1.2/../../../../nios2-elf/lib/mhw-mulx\libsmallc.a(lib_a-fvwrite_small_dev.o)
 .debug_frame   0x00002164       0x2c c:/altera/11.1/nios2eds/bin/gnu/h-i686-mingw32/bin/../lib/gcc/nios2-elf/4.1.2/../../../../nios2-elf/lib/mhw-mulx\libsmallc.a(lib_a-fvwrite_small_str.o)
 .debug_frame   0x00002190       0x20 c:/altera/11.1/nios2eds/bin/gnu/h-i686-mingw32/bin/../lib/gcc/nios2-elf/4.1.2/../../../../nios2-elf/lib/mhw-mulx\libsmallc.a(lib_a-memmove.o)
 .debug_frame   0x000021b0       0x48 c:/altera/11.1/nios2eds/bin/gnu/h-i686-mingw32/bin/../lib/gcc/nios2-elf/4.1.2/../../../../nios2-elf/lib/mhw-mulx\libsmallc.a(lib_a-putc.o)
 .debug_frame   0x000021f8       0x2c c:/altera/11.1/nios2eds/bin/gnu/h-i686-mingw32/bin/../lib/gcc/nios2-elf/4.1.2/../../../../nios2-elf/lib/mhw-mulx\libsmallc.a(lib_a-writer.o)
 .debug_frame   0x00002224       0x2c ../TR4_HDMI_TX_RX_bsp/\libhal_bsp.a(alt_irq_register.o)
 .debug_frame   0x00002250       0x48 ../TR4_HDMI_TX_RX_bsp/\libhal_bsp.a(alt_load.o)
 .debug_frame   0x00002298       0x2c ../TR4_HDMI_TX_RX_bsp/\libhal_bsp.a(alt_main.o)
 .debug_frame   0x000022c4       0x48 ../TR4_HDMI_TX_RX_bsp/\libhal_bsp.a(alt_tick.o)
 .debug_frame   0x0000230c       0x2c ../TR4_HDMI_TX_RX_bsp/\libhal_bsp.a(alt_usleep.o)
 .debug_frame   0x00002338       0x48 ../TR4_HDMI_TX_RX_bsp/\libhal_bsp.a(alt_write.o)
 .debug_frame   0x00002380       0x64 ../TR4_HDMI_TX_RX_bsp/\libhal_bsp.a(alt_sys_init.o)
 .debug_frame   0x000023e4       0x48 ../TR4_HDMI_TX_RX_bsp/\libhal_bsp.a(altera_avalon_jtag_uart_fd.o)
 .debug_frame   0x0000242c       0x2c ../TR4_HDMI_TX_RX_bsp/\libhal_bsp.a(altera_avalon_jtag_uart_read.o)
 .debug_frame   0x00002458       0x2c ../TR4_HDMI_TX_RX_bsp/\libhal_bsp.a(altera_avalon_jtag_uart_write.o)
 .debug_frame   0x00002484       0x48 ../TR4_HDMI_TX_RX_bsp/\libhal_bsp.a(altera_avalon_timer_sc.o)
 .debug_frame   0x000024cc       0x2c ../TR4_HDMI_TX_RX_bsp/\libhal_bsp.a(alt_busy_sleep.o)
 .debug_frame   0x000024f8       0x48 ../TR4_HDMI_TX_RX_bsp/\libhal_bsp.a(alt_close.o)
 .debug_frame   0x00002540       0x2c ../TR4_HDMI_TX_RX_bsp/\libhal_bsp.a(alt_dcache_flush_all.o)
 .debug_frame   0x0000256c       0x2c ../TR4_HDMI_TX_RX_bsp/\libhal_bsp.a(alt_dev.o)
 .debug_frame   0x00002598       0x48 ../TR4_HDMI_TX_RX_bsp/\libhal_bsp.a(alt_dev_llist_insert.o)
 .debug_frame   0x000025e0       0x2c ../TR4_HDMI_TX_RX_bsp/\libhal_bsp.a(alt_do_ctors.o)
 .debug_frame   0x0000260c       0x2c ../TR4_HDMI_TX_RX_bsp/\libhal_bsp.a(alt_do_dtors.o)
 .debug_frame   0x00002638       0x2c ../TR4_HDMI_TX_RX_bsp/\libhal_bsp.a(alt_icache_flush_all.o)
 .debug_frame   0x00002664       0x80 ../TR4_HDMI_TX_RX_bsp/\libhal_bsp.a(alt_iic.o)
 .debug_frame   0x000026e4       0x2c ../TR4_HDMI_TX_RX_bsp/\libhal_bsp.a(alt_iic_isr_register.o)
 .debug_frame   0x00002710       0x48 ../TR4_HDMI_TX_RX_bsp/\libhal_bsp.a(alt_io_redirect.o)
 .debug_frame   0x00002758       0x2c ../TR4_HDMI_TX_RX_bsp/\libhal_bsp.a(alt_irq_handler.o)
 .debug_frame   0x00002784       0x64 ../TR4_HDMI_TX_RX_bsp/\libhal_bsp.a(alt_open.o)
 .debug_frame   0x000027e8       0x2c ../TR4_HDMI_TX_RX_bsp/\libhal_bsp.a(alt_release_fd.o)
 .debug_frame   0x00002814       0x2c ../TR4_HDMI_TX_RX_bsp/\libhal_bsp.a(altera_nios2_qsys_irq.o)
 .debug_frame   0x00002840       0x2c ../TR4_HDMI_TX_RX_bsp/\libhal_bsp.a(alt_find_dev.o)
 .debug_frame   0x0000286c       0x2c ../TR4_HDMI_TX_RX_bsp/\libhal_bsp.a(alt_find_file.o)
 .debug_frame   0x00002898       0x2c ../TR4_HDMI_TX_RX_bsp/\libhal_bsp.a(alt_get_fd.o)
 .debug_frame   0x000028c4       0x2c ../TR4_HDMI_TX_RX_bsp/\libhal_bsp.a(alt_icache_flush.o)
 .debug_frame   0x000028f0       0x20 c:/altera/11.1/nios2eds/bin/gnu/h-i686-mingw32/bin/../lib/gcc/nios2-elf/4.1.2/../../../../nios2-elf/lib/mhw-mulx\libsmallc.a(lib_a-atexit.o)
 .debug_frame   0x00002910       0x2c c:/altera/11.1/nios2eds/bin/gnu/h-i686-mingw32/bin/../lib/gcc/nios2-elf/4.1.2/../../../../nios2-elf/lib/mhw-mulx\libsmallc.a(lib_a-exit.o)
 .debug_frame   0x0000293c       0x20 c:/altera/11.1/nios2eds/bin/gnu/h-i686-mingw32/bin/../lib/gcc/nios2-elf/4.1.2/../../../../nios2-elf/lib/mhw-mulx\libsmallc.a(lib_a-memcmp.o)
 .debug_frame   0x0000295c       0x34 c:/altera/11.1/nios2eds/bin/gnu/h-i686-mingw32/bin/../lib/gcc/nios2-elf/4.1.2/../../../../nios2-elf/lib/mhw-mulx\libsmallc.a(lib_a-__atexit.o)
 .debug_frame   0x00002990       0x4c c:/altera/11.1/nios2eds/bin/gnu/h-i686-mingw32/bin/../lib/gcc/nios2-elf/4.1.2/../../../../nios2-elf/lib/mhw-mulx\libsmallc.a(lib_a-__call_atexit.o)
 .debug_frame   0x000029dc       0x48 ../TR4_HDMI_TX_RX_bsp/\libhal_bsp.a(alt_exit.o)

.debug_str      0x00000000     0x14e6
 *(.debug_str)
 .debug_str     0x00000000       0x35 obj/HDMI_Lib/HDMI_RX/HDMI_RX.o
 .debug_str     0x00000035       0x83 obj/HDMI_Lib/HDMI_RX/it6605.o
 .debug_str     0x000000b8       0x12 obj/HDMI_Lib/HDMI_TX/EDID.o
 .debug_str     0x000000ca       0x45 obj/HDMI_Lib/HDMI_TX/HDMI_TX.o
 .debug_str     0x0000010f       0x12 obj/HDMI_Lib/HDMI_TX/dss_sha.o
 .debug_str     0x00000121       0xa3 obj/HDMI_Lib/HDMI_TX/it6613_drv.o
 .debug_str     0x000001c4       0x27 obj/HDMI_Lib/HDMI_TX/it6613_sys.o
 .debug_str     0x000001eb       0x40 obj/HDMI_Lib/mcu.o
 .debug_str     0x0000022b       0x1d obj/main.o
 .debug_str     0x00000248       0x45 obj/terasic_lib/I2C.o
 .debug_str     0x0000028d       0x19 obj/terasic_lib/debug.o
 .debug_str     0x000002a6      0x1fc c:/altera/11.1/nios2eds/bin/gnu/h-i686-mingw32/bin/../lib/gcc/nios2-elf/4.1.2/mhw-mulx\libgcc.a(_mul_df.o)
                                0x241 (size before relaxing)
 .debug_str     0x000004a2       0x35 c:/altera/11.1/nios2eds/bin/gnu/h-i686-mingw32/bin/../lib/gcc/nios2-elf/4.1.2/mhw-mulx\libgcc.a(_div_df.o)
                                0x231 (size before relaxing)
 .debug_str     0x000004d7       0x1e c:/altera/11.1/nios2eds/bin/gnu/h-i686-mingw32/bin/../lib/gcc/nios2-elf/4.1.2/mhw-mulx\libgcc.a(_si_to_df.o)
                                0x1de (size before relaxing)
 .debug_str     0x00000000      0x1a3 c:/altera/11.1/nios2eds/bin/gnu/h-i686-mingw32/bin/../lib/gcc/nios2-elf/4.1.2/mhw-mulx\libgcc.a(_thenan_df.o)
 .debug_str     0x000004f5       0xa1 c:/altera/11.1/nios2eds/bin/gnu/h-i686-mingw32/bin/../lib/gcc/nios2-elf/4.1.2/mhw-mulx\libgcc.a(lib2-divmod.o)
                                0x1b4 (size before relaxing)
 .debug_str     0x00000596       0x40 c:/altera/11.1/nios2eds/bin/gnu/h-i686-mingw32/bin/../lib/gcc/nios2-elf/4.1.2/mhw-mulx\libgcc.a(_clzsi2.o)
                                0x17e (size before relaxing)
 .debug_str     0x000005d6       0x10 c:/altera/11.1/nios2eds/bin/gnu/h-i686-mingw32/bin/../lib/gcc/nios2-elf/4.1.2/mhw-mulx\libgcc.a(_pack_df.o)
                                0x206 (size before relaxing)
 .debug_str     0x000005e6        0xb c:/altera/11.1/nios2eds/bin/gnu/h-i686-mingw32/bin/../lib/gcc/nios2-elf/4.1.2/mhw-mulx\libgcc.a(_unpack_df.o)
                                0x1e8 (size before relaxing)
 .debug_str     0x00000000      0x161 c:/altera/11.1/nios2eds/bin/gnu/h-i686-mingw32/bin/../lib/gcc/nios2-elf/4.1.2/mhw-mulx\libgcc.a(_clz.o)
 .debug_str     0x000005f1      0x3a7 c:/altera/11.1/nios2eds/bin/gnu/h-i686-mingw32/bin/../lib/gcc/nios2-elf/4.1.2/../../../../nios2-elf/lib/mhw-mulx\libsmallc.a(lib_a-impure.o)
                                0x45b (size before relaxing)
 .debug_str     0x00000998       0xe0 c:/altera/11.1/nios2eds/bin/gnu/h-i686-mingw32/bin/../lib/gcc/nios2-elf/4.1.2/../../../../nios2-elf/lib/mhw-mulx\libsmallc.a(lib_a-memset.o)
                                0x17c (size before relaxing)
 .debug_str     0x00000a78       0xf0 c:/altera/11.1/nios2eds/bin/gnu/h-i686-mingw32/bin/../lib/gcc/nios2-elf/4.1.2/../../../../nios2-elf/lib/mhw-mulx\libsmallc.a(lib_a-printf.o)
                                0x464 (size before relaxing)
 .debug_str     0x00000b68       0x51 c:/altera/11.1/nios2eds/bin/gnu/h-i686-mingw32/bin/../lib/gcc/nios2-elf/4.1.2/../../../../nios2-elf/lib/mhw-mulx\libsmallc.a(lib_a-putchar.o)
                                0x450 (size before relaxing)
 .debug_str     0x00000bb9       0x48 c:/altera/11.1/nios2eds/bin/gnu/h-i686-mingw32/bin/../lib/gcc/nios2-elf/4.1.2/../../../../nios2-elf/lib/mhw-mulx\libsmallc.a(lib_a-puts.o)
                                0x44e (size before relaxing)
 .debug_str     0x00000c01       0x81 c:/altera/11.1/nios2eds/bin/gnu/h-i686-mingw32/bin/../lib/gcc/nios2-elf/4.1.2/../../../../nios2-elf/lib/mhw-mulx\libsmallc.a(lib_a-sprintf.o)
                                0x497 (size before relaxing)
 .debug_str     0x00000c82       0x45 c:/altera/11.1/nios2eds/bin/gnu/h-i686-mingw32/bin/../lib/gcc/nios2-elf/4.1.2/../../../../nios2-elf/lib/mhw-mulx\libsmallc.a(lib_a-strlen.o)
                                0x182 (size before relaxing)
 .debug_str     0x00000cc7      0x11b c:/altera/11.1/nios2eds/bin/gnu/h-i686-mingw32/bin/../lib/gcc/nios2-elf/4.1.2/../../../../nios2-elf/lib/mhw-mulx\libsmallc.a(lib_a-vfprintf.o)
                                0x560 (size before relaxing)
 .debug_str     0x00000de2       0x4a c:/altera/11.1/nios2eds/bin/gnu/h-i686-mingw32/bin/../lib/gcc/nios2-elf/4.1.2/../../../../nios2-elf/lib/mhw-mulx\libsmallc.a(lib_a-vfprintf_1.o)
                                0x465 (size before relaxing)
 .debug_str     0x00000e2c       0x57 c:/altera/11.1/nios2eds/bin/gnu/h-i686-mingw32/bin/../lib/gcc/nios2-elf/4.1.2/../../../../nios2-elf/lib/mhw-mulx\libsmallc.a(lib_a-vsnprintf.o)
                                0x4a9 (size before relaxing)
 .debug_str     0x00000e83       0x70 c:/altera/11.1/nios2eds/bin/gnu/h-i686-mingw32/bin/../lib/gcc/nios2-elf/4.1.2/../../../../nios2-elf/lib/mhw-mulx\libsmallc.a(lib_a-fvwrite_small_dev.o)
                                0x468 (size before relaxing)
 .debug_str     0x00000ef3       0x5d c:/altera/11.1/nios2eds/bin/gnu/h-i686-mingw32/bin/../lib/gcc/nios2-elf/4.1.2/../../../../nios2-elf/lib/mhw-mulx\libsmallc.a(lib_a-fvwrite_small_str.o)
                                0x485 (size before relaxing)
 .debug_str     0x00000f50       0x60 c:/altera/11.1/nios2eds/bin/gnu/h-i686-mingw32/bin/../lib/gcc/nios2-elf/4.1.2/../../../../nios2-elf/lib/mhw-mulx\libsmallc.a(lib_a-memmove.o)
                                0x197 (size before relaxing)
 .debug_str     0x00000fb0       0x4f c:/altera/11.1/nios2eds/bin/gnu/h-i686-mingw32/bin/../lib/gcc/nios2-elf/4.1.2/../../../../nios2-elf/lib/mhw-mulx\libsmallc.a(lib_a-putc.o)
                                0x453 (size before relaxing)
 .debug_str     0x00000fff       0x4f c:/altera/11.1/nios2eds/bin/gnu/h-i686-mingw32/bin/../lib/gcc/nios2-elf/4.1.2/../../../../nios2-elf/lib/mhw-mulx\libsmallc.a(lib_a-writer.o)
                                0x44f (size before relaxing)
 .debug_str     0x0000104e       0x40 c:/altera/11.1/nios2eds/bin/gnu/h-i686-mingw32/bin/../lib/gcc/nios2-elf/4.1.2/../../../../nios2-elf/lib/mhw-mulx\libsmallc.a(lib_a-int_errno.o)
                                0x175 (size before relaxing)
 .debug_str     0x0000108e       0x21 ../TR4_HDMI_TX_RX_bsp/\libhal_bsp.a(alt_irq_register.o)
 .debug_str     0x000010af       0x12 ../TR4_HDMI_TX_RX_bsp/\libhal_bsp.a(alt_load.o)
 .debug_str     0x000010c1       0x12 ../TR4_HDMI_TX_RX_bsp/\libhal_bsp.a(alt_main.o)
 .debug_str     0x000010d3       0x1a ../TR4_HDMI_TX_RX_bsp/\libhal_bsp.a(alt_tick.o)
 .debug_str     0x000010ed       0x12 ../TR4_HDMI_TX_RX_bsp/\libhal_bsp.a(alt_usleep.o)
 .debug_str     0x000010ff       0x12 ../TR4_HDMI_TX_RX_bsp/\libhal_bsp.a(alt_write.o)
 .debug_str     0x00001111       0x12 ../TR4_HDMI_TX_RX_bsp/\libhal_bsp.a(alt_sys_init.o)
 .debug_str     0x00001123       0x12 ../TR4_HDMI_TX_RX_bsp/\libhal_bsp.a(altera_avalon_jtag_uart_read.o)
 .debug_str     0x00001135       0x12 ../TR4_HDMI_TX_RX_bsp/\libhal_bsp.a(altera_avalon_jtag_uart_write.o)
 .debug_str     0x00001147       0x12 ../TR4_HDMI_TX_RX_bsp/\libhal_bsp.a(altera_avalon_timer_sc.o)
 .debug_str     0x00001159       0x12 ../TR4_HDMI_TX_RX_bsp/\libhal_bsp.a(alt_busy_sleep.o)
 .debug_str     0x0000116b       0x12 ../TR4_HDMI_TX_RX_bsp/\libhal_bsp.a(alt_close.o)
 .debug_str     0x0000117d       0x12 ../TR4_HDMI_TX_RX_bsp/\libhal_bsp.a(alt_dcache_flush_all.o)
 .debug_str     0x0000118f       0x12 ../TR4_HDMI_TX_RX_bsp/\libhal_bsp.a(alt_dev.o)
 .debug_str     0x000011a1       0x12 ../TR4_HDMI_TX_RX_bsp/\libhal_bsp.a(alt_dev_llist_insert.o)
 .debug_str     0x000011b3       0x12 ../TR4_HDMI_TX_RX_bsp/\libhal_bsp.a(alt_errno.o)
 .debug_str     0x000011c5       0x12 ../TR4_HDMI_TX_RX_bsp/\libhal_bsp.a(alt_icache_flush_all.o)
 .debug_str     0x000011d7       0x18 ../TR4_HDMI_TX_RX_bsp/\libhal_bsp.a(alt_iic.o)
 .debug_str     0x000011ef       0x1a ../TR4_HDMI_TX_RX_bsp/\libhal_bsp.a(alt_iic_isr_register.o)
 .debug_str     0x00001209       0x12 ../TR4_HDMI_TX_RX_bsp/\libhal_bsp.a(alt_io_redirect.o)
 .debug_str     0x0000121b       0x12 ../TR4_HDMI_TX_RX_bsp/\libhal_bsp.a(alt_irq_handler.o)
 .debug_str     0x0000122d       0x12 ../TR4_HDMI_TX_RX_bsp/\libhal_bsp.a(alt_open.o)
 .debug_str     0x0000123f       0x12 ../TR4_HDMI_TX_RX_bsp/\libhal_bsp.a(altera_nios2_qsys_irq.o)
 .debug_str     0x00001251       0x12 ../TR4_HDMI_TX_RX_bsp/\libhal_bsp.a(alt_find_dev.o)
 .debug_str     0x00001263       0x12 ../TR4_HDMI_TX_RX_bsp/\libhal_bsp.a(alt_find_file.o)
 .debug_str     0x00001275       0x12 ../TR4_HDMI_TX_RX_bsp/\libhal_bsp.a(alt_get_fd.o)
 .debug_str     0x00001287       0x12 ../TR4_HDMI_TX_RX_bsp/\libhal_bsp.a(alt_icache_flush.o)
 .debug_str     0x00001299       0xd9 c:/altera/11.1/nios2eds/bin/gnu/h-i686-mingw32/bin/../lib/gcc/nios2-elf/4.1.2/../../../../nios2-elf/lib/mhw-mulx\libsmallc.a(lib_a-atexit.o)
                                0x1e3 (size before relaxing)
 .debug_str     0x00001372       0x41 c:/altera/11.1/nios2eds/bin/gnu/h-i686-mingw32/bin/../lib/gcc/nios2-elf/4.1.2/../../../../nios2-elf/lib/mhw-mulx\libsmallc.a(lib_a-exit.o)
                                0x176 (size before relaxing)
 .debug_str     0x000013b3       0x45 c:/altera/11.1/nios2eds/bin/gnu/h-i686-mingw32/bin/../lib/gcc/nios2-elf/4.1.2/../../../../nios2-elf/lib/mhw-mulx\libsmallc.a(lib_a-memcmp.o)
                                0x17c (size before relaxing)
 .debug_str     0x000013f8       0x54 c:/altera/11.1/nios2eds/bin/gnu/h-i686-mingw32/bin/../lib/gcc/nios2-elf/4.1.2/../../../../nios2-elf/lib/mhw-mulx\libsmallc.a(lib_a-__atexit.o)
                                0x465 (size before relaxing)
 .debug_str     0x0000144c       0x7e c:/altera/11.1/nios2eds/bin/gnu/h-i686-mingw32/bin/../lib/gcc/nios2-elf/4.1.2/../../../../nios2-elf/lib/mhw-mulx\libsmallc.a(lib_a-__call_atexit.o)
                                0x48f (size before relaxing)
 .debug_str     0x000014ca       0x1c ../TR4_HDMI_TX_RX_bsp/\libhal_bsp.a(alt_exit.o)

.debug_loc      0x00000000     0x501d
 *(.debug_loc)
 .debug_loc     0x00000000      0x230 obj/HDMI_Lib/HDMI_RX/HDMI_RX.o
 .debug_loc     0x00000230     0x10cc obj/HDMI_Lib/HDMI_RX/it6605.o
 .debug_loc     0x000012fc       0x81 obj/HDMI_Lib/HDMI_TX/EDID.o
 .debug_loc     0x0000137d      0x286 obj/HDMI_Lib/HDMI_TX/HDMI_TX.o
 .debug_loc     0x00001603      0xc6e obj/HDMI_Lib/HDMI_TX/it6613_drv.o
 .debug_loc     0x00002271       0xd7 obj/HDMI_Lib/HDMI_TX/it6613_sys.o
 .debug_loc     0x00002348      0x50a obj/HDMI_Lib/mcu.o
 .debug_loc     0x00002852      0x1af obj/main.o
 .debug_loc     0x00002a01      0x183 obj/terasic_lib/I2C.o
 .debug_loc     0x00002b84       0xad obj/terasic_lib/debug.o
 .debug_loc     0x00002c31      0x346 c:/altera/11.1/nios2eds/bin/gnu/h-i686-mingw32/bin/../lib/gcc/nios2-elf/4.1.2/mhw-mulx\libgcc.a(_mul_df.o)
 .debug_loc     0x00002f77      0x1df c:/altera/11.1/nios2eds/bin/gnu/h-i686-mingw32/bin/../lib/gcc/nios2-elf/4.1.2/mhw-mulx\libgcc.a(_div_df.o)
 .debug_loc     0x00003156       0x9a c:/altera/11.1/nios2eds/bin/gnu/h-i686-mingw32/bin/../lib/gcc/nios2-elf/4.1.2/mhw-mulx\libgcc.a(_si_to_df.o)
 .debug_loc     0x000031f0      0x1d2 c:/altera/11.1/nios2eds/bin/gnu/h-i686-mingw32/bin/../lib/gcc/nios2-elf/4.1.2/mhw-mulx\libgcc.a(lib2-divmod.o)
 .debug_loc     0x000033c2       0x1e c:/altera/11.1/nios2eds/bin/gnu/h-i686-mingw32/bin/../lib/gcc/nios2-elf/4.1.2/mhw-mulx\libgcc.a(_clzsi2.o)
 .debug_loc     0x000033e0      0x184 c:/altera/11.1/nios2eds/bin/gnu/h-i686-mingw32/bin/../lib/gcc/nios2-elf/4.1.2/mhw-mulx\libgcc.a(_pack_df.o)
 .debug_loc     0x00003564       0xe5 c:/altera/11.1/nios2eds/bin/gnu/h-i686-mingw32/bin/../lib/gcc/nios2-elf/4.1.2/mhw-mulx\libgcc.a(_unpack_df.o)
 .debug_loc     0x00003649       0x4f c:/altera/11.1/nios2eds/bin/gnu/h-i686-mingw32/bin/../lib/gcc/nios2-elf/4.1.2/../../../../nios2-elf/lib/mhw-mulx\libsmallc.a(lib_a-memset.o)
 .debug_loc     0x00003698       0x8d c:/altera/11.1/nios2eds/bin/gnu/h-i686-mingw32/bin/../lib/gcc/nios2-elf/4.1.2/../../../../nios2-elf/lib/mhw-mulx\libsmallc.a(lib_a-printf.o)
 .debug_loc     0x00003725       0x44 c:/altera/11.1/nios2eds/bin/gnu/h-i686-mingw32/bin/../lib/gcc/nios2-elf/4.1.2/../../../../nios2-elf/lib/mhw-mulx\libsmallc.a(lib_a-putchar.o)
 .debug_loc     0x00003769       0xa2 c:/altera/11.1/nios2eds/bin/gnu/h-i686-mingw32/bin/../lib/gcc/nios2-elf/4.1.2/../../../../nios2-elf/lib/mhw-mulx\libsmallc.a(lib_a-puts.o)
 .debug_loc     0x0000380b       0xbe c:/altera/11.1/nios2eds/bin/gnu/h-i686-mingw32/bin/../lib/gcc/nios2-elf/4.1.2/../../../../nios2-elf/lib/mhw-mulx\libsmallc.a(lib_a-sprintf.o)
 .debug_loc     0x000038c9       0x1e c:/altera/11.1/nios2eds/bin/gnu/h-i686-mingw32/bin/../lib/gcc/nios2-elf/4.1.2/../../../../nios2-elf/lib/mhw-mulx\libsmallc.a(lib_a-strlen.o)
 .debug_loc     0x000038e7      0x5a9 c:/altera/11.1/nios2eds/bin/gnu/h-i686-mingw32/bin/../lib/gcc/nios2-elf/4.1.2/../../../../nios2-elf/lib/mhw-mulx\libsmallc.a(lib_a-vfprintf.o)
 .debug_loc     0x00003e90       0x39 c:/altera/11.1/nios2eds/bin/gnu/h-i686-mingw32/bin/../lib/gcc/nios2-elf/4.1.2/../../../../nios2-elf/lib/mhw-mulx\libsmallc.a(lib_a-vfprintf_1.o)
 .debug_loc     0x00003ec9      0x1a4 c:/altera/11.1/nios2eds/bin/gnu/h-i686-mingw32/bin/../lib/gcc/nios2-elf/4.1.2/../../../../nios2-elf/lib/mhw-mulx\libsmallc.a(lib_a-vsnprintf.o)
 .debug_loc     0x0000406d      0x162 c:/altera/11.1/nios2eds/bin/gnu/h-i686-mingw32/bin/../lib/gcc/nios2-elf/4.1.2/../../../../nios2-elf/lib/mhw-mulx\libsmallc.a(lib_a-fvwrite_small_dev.o)
 .debug_loc     0x000041cf       0xe1 c:/altera/11.1/nios2eds/bin/gnu/h-i686-mingw32/bin/../lib/gcc/nios2-elf/4.1.2/../../../../nios2-elf/lib/mhw-mulx\libsmallc.a(lib_a-fvwrite_small_str.o)
 .debug_loc     0x000042b0       0x4f c:/altera/11.1/nios2eds/bin/gnu/h-i686-mingw32/bin/../lib/gcc/nios2-elf/4.1.2/../../../../nios2-elf/lib/mhw-mulx\libsmallc.a(lib_a-memmove.o)
 .debug_loc     0x000042ff       0xd4 c:/altera/11.1/nios2eds/bin/gnu/h-i686-mingw32/bin/../lib/gcc/nios2-elf/4.1.2/../../../../nios2-elf/lib/mhw-mulx\libsmallc.a(lib_a-putc.o)
 .debug_loc     0x000043d3       0x97 c:/altera/11.1/nios2eds/bin/gnu/h-i686-mingw32/bin/../lib/gcc/nios2-elf/4.1.2/../../../../nios2-elf/lib/mhw-mulx\libsmallc.a(lib_a-writer.o)
 .debug_loc     0x0000446a       0x2c ../TR4_HDMI_TX_RX_bsp/\libhal_bsp.a(alt_irq_register.o)
 .debug_loc     0x00004496       0x56 ../TR4_HDMI_TX_RX_bsp/\libhal_bsp.a(alt_load.o)
 .debug_loc     0x000044ec       0x2b ../TR4_HDMI_TX_RX_bsp/\libhal_bsp.a(alt_main.o)
 .debug_loc     0x00004517       0x56 ../TR4_HDMI_TX_RX_bsp/\libhal_bsp.a(alt_tick.o)
 .debug_loc     0x0000456d       0x2b ../TR4_HDMI_TX_RX_bsp/\libhal_bsp.a(alt_usleep.o)
 .debug_loc     0x00004598       0x56 ../TR4_HDMI_TX_RX_bsp/\libhal_bsp.a(alt_write.o)
 .debug_loc     0x000045ee       0x81 ../TR4_HDMI_TX_RX_bsp/\libhal_bsp.a(alt_sys_init.o)
 .debug_loc     0x0000466f       0x56 ../TR4_HDMI_TX_RX_bsp/\libhal_bsp.a(altera_avalon_jtag_uart_fd.o)
 .debug_loc     0x000046c5       0x2b ../TR4_HDMI_TX_RX_bsp/\libhal_bsp.a(altera_avalon_jtag_uart_read.o)
 .debug_loc     0x000046f0       0x2b ../TR4_HDMI_TX_RX_bsp/\libhal_bsp.a(altera_avalon_jtag_uart_write.o)
 .debug_loc     0x0000471b       0x56 ../TR4_HDMI_TX_RX_bsp/\libhal_bsp.a(altera_avalon_timer_sc.o)
 .debug_loc     0x00004771       0x2b ../TR4_HDMI_TX_RX_bsp/\libhal_bsp.a(alt_busy_sleep.o)
 .debug_loc     0x0000479c       0x56 ../TR4_HDMI_TX_RX_bsp/\libhal_bsp.a(alt_close.o)
 .debug_loc     0x000047f2       0x2b ../TR4_HDMI_TX_RX_bsp/\libhal_bsp.a(alt_dcache_flush_all.o)
 .debug_loc     0x0000481d       0x2b ../TR4_HDMI_TX_RX_bsp/\libhal_bsp.a(alt_dev.o)
 .debug_loc     0x00004848       0x56 ../TR4_HDMI_TX_RX_bsp/\libhal_bsp.a(alt_dev_llist_insert.o)
 .debug_loc     0x0000489e       0x2b ../TR4_HDMI_TX_RX_bsp/\libhal_bsp.a(alt_do_ctors.o)
 .debug_loc     0x000048c9       0x2b ../TR4_HDMI_TX_RX_bsp/\libhal_bsp.a(alt_do_dtors.o)
 .debug_loc     0x000048f4       0x2b ../TR4_HDMI_TX_RX_bsp/\libhal_bsp.a(alt_icache_flush_all.o)
 .debug_loc     0x0000491f       0xac ../TR4_HDMI_TX_RX_bsp/\libhal_bsp.a(alt_iic.o)
 .debug_loc     0x000049cb       0x2b ../TR4_HDMI_TX_RX_bsp/\libhal_bsp.a(alt_iic_isr_register.o)
 .debug_loc     0x000049f6       0x56 ../TR4_HDMI_TX_RX_bsp/\libhal_bsp.a(alt_io_redirect.o)
 .debug_loc     0x00004a4c       0x2b ../TR4_HDMI_TX_RX_bsp/\libhal_bsp.a(alt_irq_handler.o)
 .debug_loc     0x00004a77       0x81 ../TR4_HDMI_TX_RX_bsp/\libhal_bsp.a(alt_open.o)
 .debug_loc     0x00004af8       0x2b ../TR4_HDMI_TX_RX_bsp/\libhal_bsp.a(alt_release_fd.o)
 .debug_loc     0x00004b23       0x2b ../TR4_HDMI_TX_RX_bsp/\libhal_bsp.a(altera_nios2_qsys_irq.o)
 .debug_loc     0x00004b4e       0x2b ../TR4_HDMI_TX_RX_bsp/\libhal_bsp.a(alt_find_dev.o)
 .debug_loc     0x00004b79       0x2b ../TR4_HDMI_TX_RX_bsp/\libhal_bsp.a(alt_find_file.o)
 .debug_loc     0x00004ba4       0x2b ../TR4_HDMI_TX_RX_bsp/\libhal_bsp.a(alt_get_fd.o)
 .debug_loc     0x00004bcf       0x2b ../TR4_HDMI_TX_RX_bsp/\libhal_bsp.a(alt_icache_flush.o)
 .debug_loc     0x00004bfa       0x1e c:/altera/11.1/nios2eds/bin/gnu/h-i686-mingw32/bin/../lib/gcc/nios2-elf/4.1.2/../../../../nios2-elf/lib/mhw-mulx\libsmallc.a(lib_a-atexit.o)
 .debug_loc     0x00004c18       0x3d c:/altera/11.1/nios2eds/bin/gnu/h-i686-mingw32/bin/../lib/gcc/nios2-elf/4.1.2/../../../../nios2-elf/lib/mhw-mulx\libsmallc.a(lib_a-exit.o)
 .debug_loc     0x00004c55       0x70 c:/altera/11.1/nios2eds/bin/gnu/h-i686-mingw32/bin/../lib/gcc/nios2-elf/4.1.2/../../../../nios2-elf/lib/mhw-mulx\libsmallc.a(lib_a-memcmp.o)
 .debug_loc     0x00004cc5      0x141 c:/altera/11.1/nios2eds/bin/gnu/h-i686-mingw32/bin/../lib/gcc/nios2-elf/4.1.2/../../../../nios2-elf/lib/mhw-mulx\libsmallc.a(lib_a-__atexit.o)
 .debug_loc     0x00004e06      0x1c1 c:/altera/11.1/nios2eds/bin/gnu/h-i686-mingw32/bin/../lib/gcc/nios2-elf/4.1.2/../../../../nios2-elf/lib/mhw-mulx\libsmallc.a(lib_a-__call_atexit.o)
 .debug_loc     0x00004fc7       0x56 ../TR4_HDMI_TX_RX_bsp/\libhal_bsp.a(alt_exit.o)

.debug_macinfo
 *(.debug_macinfo)

.debug_weaknames
 *(.debug_weaknames)

.debug_funcnames
 *(.debug_funcnames)

.debug_typenames
 *(.debug_typenames)

.debug_varnames
 *(.debug_varnames)

.debug_alt_sim_info
                0x00000000       0x50
 *(.debug_alt_sim_info)
 .debug_alt_sim_info
                0x00000000       0x20 ../TR4_HDMI_TX_RX_bsp//obj/HAL/src/crt0.o
 .debug_alt_sim_info
                0x00000020       0x30 ../TR4_HDMI_TX_RX_bsp/\libhal_bsp.a(alt_busy_sleep.o)
                0x01040000                __alt_data_end = 0x1040000
                0x01040000                PROVIDE (__alt_stack_pointer, __alt_data_end)
                0x0103e320                PROVIDE (__alt_stack_limit, __alt_stack_base)
                0x0103e320                PROVIDE (__alt_heap_start, end)
                0x01040000                PROVIDE (__alt_heap_limit, 0x1040000)
OUTPUT(TR4_HDMI_TX_RX.elf elf32-littlenios2)

.debug_ranges   0x00000000      0x278
 .debug_ranges  0x00000000       0x20 ../TR4_HDMI_TX_RX_bsp//obj/HAL/src/crt0.o
 .debug_ranges  0x00000020       0x88 c:/altera/11.1/nios2eds/bin/gnu/h-i686-mingw32/bin/../lib/gcc/nios2-elf/4.1.2/mhw-mulx\libgcc.a(_mul_df.o)
 .debug_ranges  0x000000a8       0x50 c:/altera/11.1/nios2eds/bin/gnu/h-i686-mingw32/bin/../lib/gcc/nios2-elf/4.1.2/mhw-mulx\libgcc.a(_div_df.o)
 .debug_ranges  0x000000f8       0x28 c:/altera/11.1/nios2eds/bin/gnu/h-i686-mingw32/bin/../lib/gcc/nios2-elf/4.1.2/mhw-mulx\libgcc.a(_clzsi2.o)
 .debug_ranges  0x00000120       0x28 c:/altera/11.1/nios2eds/bin/gnu/h-i686-mingw32/bin/../lib/gcc/nios2-elf/4.1.2/mhw-mulx\libgcc.a(_pack_df.o)
 .debug_ranges  0x00000148       0xa8 c:/altera/11.1/nios2eds/bin/gnu/h-i686-mingw32/bin/../lib/gcc/nios2-elf/4.1.2/../../../../nios2-elf/lib/mhw-mulx\libsmallc.a(lib_a-vfprintf.o)
 .debug_ranges  0x000001f0       0x18 c:/altera/11.1/nios2eds/bin/gnu/h-i686-mingw32/bin/../lib/gcc/nios2-elf/4.1.2/../../../../nios2-elf/lib/mhw-mulx\libsmallc.a(lib_a-fvwrite_small_str.o)
 .debug_ranges  0x00000208       0x28 ../TR4_HDMI_TX_RX_bsp/\libhal_bsp.a(alt_irq_entry.o)
 .debug_ranges  0x00000230       0x30 ../TR4_HDMI_TX_RX_bsp/\libhal_bsp.a(alt_exception_entry.o)
 .debug_ranges  0x00000260       0x18 c:/altera/11.1/nios2eds/bin/gnu/h-i686-mingw32/bin/../lib/gcc/nios2-elf/4.1.2/../../../../nios2-elf/lib/mhw-mulx\libsmallc.a(lib_a-__call_atexit.o)
